 jdwp

 Timestamp is ffffffff (Sun Feb  7 06:28:15 2106)

 Preferred load address is 10000000

 Start         Length     Name                   Class
 0001:00000000 000208cfH .text$mn                CODE
 0002:00000000 00000144H .idata$5                DATA
 0002:00000144 00000004H .00cfg                  DATA
 0002:00000148 00000004H .CRT$XCA                DATA
 0002:0000014c 00000004H .CRT$XCZ                DATA
 0002:00000150 00000004H .CRT$XIA                DATA
 0002:00000154 00000004H .CRT$XIZ                DATA
 0002:00000158 00000004H .CRT$XPA                DATA
 0002:0000015c 00000004H .CRT$XPZ                DATA
 0002:00000160 00000004H .CRT$XTA                DATA
 0002:00000164 0000000cH .CRT$XTZ                DATA
 0002:00000168 00000000H .gfids$y                DATA
 0002:00000170 00006a48H .rdata                  DATA
 0002:00006bb8 00000004H .rdata$sxdata           DATA
 0002:00006bbc 00000284H .rdata$zzzdbg           DATA
 0002:00006e40 00000004H .rtc$IAA                DATA
 0002:00006e44 00000004H .rtc$IZZ                DATA
 0002:00006e48 00000004H .rtc$TAA                DATA
 0002:00006e4c 00000004H .rtc$TZZ                DATA
 0002:00006e50 00000090H .xdata$x                DATA
 0002:00006ee0 0000009cH .edata                  DATA
 0002:00006f7c 000000c8H .idata$2                DATA
 0002:00007044 00000014H .idata$3                DATA
 0002:00007058 00000144H .idata$4                DATA
 0002:0000719c 000005aeH .idata$6                DATA
 0003:00000000 00000448H .data                   DATA
 0003:00000448 00000954H .bss                    DATA
 0004:00000000 00000060H .rsrc$01                DATA
 0004:00000060 00000318H .rsrc$02                DATA

  Address         Publics by Value              Rva+Base       Lib:Object

 0000:00000000       ___guard_fids_count        00000000     <absolute>
 0000:00000000       ___hybrid_auxiliary_iat    00000000     <absolute>
 0000:00000000       ___guard_iat_table         00000000     <absolute>
 0000:00000000       ___enclave_config          00000000     <absolute>
 0000:00000000       ___guard_longjmp_table     00000000     <absolute>
 0000:00000000       ___arm64x_redirection_metadata_count 00000000     <absolute>
 0000:00000000       ___arm64x_extra_rfe_table  00000000     <absolute>
 0000:00000000       ___guard_eh_cont_table     00000000     <absolute>
 0000:00000000       ___guard_fids_table        00000000     <absolute>
 0000:00000000       ___hybrid_code_map_count   00000000     <absolute>
 0000:00000000       ___guard_eh_cont_count     00000000     <absolute>
 0000:00000000       ___arm64x_redirection_metadata 00000000     <absolute>
 0000:00000000       ___volatile_metadata       00000000     <absolute>
 0000:00000000       ___guard_iat_count         00000000     <absolute>
 0000:00000000       ___arm64x_extra_rfe_table_size 00000000     <absolute>
 0000:00000000       ___x64_code_ranges_to_entry_points 00000000     <absolute>
 0000:00000000       ___hybrid_code_map         00000000     <absolute>
 0000:00000000       ___AbsoluteZero            00000000     <absolute>
 0000:00000000       ___arm64x_native_entrypoint 00000000     <absolute>
 0000:00000000       ___x64_code_ranges_to_entry_points_count 00000000     <absolute>
 0000:00000000       ___dynamic_value_reloc_table 00000000     <absolute>
 0000:00000000       ___guard_longjmp_count     00000000     <absolute>
 0000:00000001       ___safe_se_handler_count   00000001     <absolute>
 0000:00000100       ___guard_flags             00000100     <absolute>
 0000:00000000       ___ImageBase               10000000     <linker-defined>
 0001:0000270c       _createFrameID             1000370c f   FrameID.obj
 0001:0000272d       _getFrameNumber            1000372d f   FrameID.obj
 0001:00002733       _validateFrameID           10003733 f   FrameID.obj
 0001:0000446d       ___local_stdio_printf_options 1000546d f i SDE.obj
 0001:00004473       __snprintf                 10005473 f i SDE.obj
 0001:0000448d       __vsnprintf                1000548d f i SDE.obj
 0001:000044a8       __vsnprintf_l              100054a8 f i SDE.obj
 0001:000046e8       _convertLineNumberTable    100056e8 f   SDE.obj
 0001:00004c78       _searchAllSourceNames      10005c78 f   SDE.obj
 0001:00004d74       _setGlobalStratumId        10005d74 f   SDE.obj
 0001:00007ae0       ___scrt_stub_for_acrt_thread_detach 10008ae0 f   MSVCRT:ucrt_stubs.obj
 0001:00007ae0       ___acrt_initialize         10008ae0 f   MSVCRT:ucrt_stubs.obj
 0001:00007ae0       ___vcrt_thread_detach      10008ae0 f   MSVCRT:ucrt_stubs.obj
 0001:00007ae0       ___vcrt_uninitialize       10008ae0 f   MSVCRT:ucrt_stubs.obj
 0001:00007ae0       ___acrt_uninitialize       10008ae0 f   MSVCRT:ucrt_stubs.obj
 0001:00007ae0       ___acrt_thread_detach      10008ae0 f   MSVCRT:ucrt_stubs.obj
 0001:00007ae0       ___scrt_stub_for_acrt_initialize 10008ae0 f   MSVCRT:ucrt_stubs.obj
 0001:00007ae0       ___scrt_stub_for_acrt_thread_attach 10008ae0 f   MSVCRT:ucrt_stubs.obj
 0001:00007ae0       ___vcrt_uninitialize_critical 10008ae0 f   MSVCRT:ucrt_stubs.obj
 0001:00007ae0       ___scrt_stub_for_acrt_uninitialize_critical 10008ae0 f   MSVCRT:ucrt_stubs.obj
 0001:00007ae0       ___scrt_stub_for_acrt_uninitialize 10008ae0 f   MSVCRT:ucrt_stubs.obj
 0001:00007ae0       ___vcrt_thread_attach      10008ae0 f   MSVCRT:ucrt_stubs.obj
 0001:00007ae0       ___acrt_thread_attach      10008ae0 f   MSVCRT:ucrt_stubs.obj
 0001:00007ae0       ___vcrt_initialize         10008ae0 f   MSVCRT:ucrt_stubs.obj
 0001:00007ae0       ___acrt_uninitialize_critical 10008ae0 f   MSVCRT:ucrt_stubs.obj
 0001:000083d2       _bagAdd                    100093d2 f   bag.obj
 0001:00008445       _bagCreateBag              10009445 f   bag.obj
 0001:00008493       _bagDeleteAll              10009493 f   bag.obj
 0001:0000849c       _bagDestroyBag             1000949c f   bag.obj
 0001:000084b6       _bagDup                    100094b6 f   bag.obj
 0001:000084ed       _bagEnumerateOver          100094ed f   bag.obj
 0001:00008522       _bagSize                   10009522 f   bag.obj
 0001:00008568       _classTrack_activate       10009568 f   classTrack.obj
 0001:00008598       _classTrack_addPreparedClass 10009598 f   classTrack.obj
 0001:00008760       _classTrack_initialize     10009760 f   classTrack.obj
 0001:000088ac       _classTrack_processUnloads 100098ac f   classTrack.obj
 0001:000088ef       _classTrack_reset          100098ef f   classTrack.obj
 0001:00008a84       _commonRef_compact         10009a84 f   commonRef.obj
 0001:00008b31       _commonRef_idToRef         10009b31 f   commonRef.obj
 0001:00008c3e       _commonRef_idToRef_delete  10009c3e f   commonRef.obj
 0001:00008c56       _commonRef_initialize      10009c56 f   commonRef.obj
 0001:00008c9c       _commonRef_lock            10009c9c f   commonRef.obj
 0001:00008cae       _commonRef_pin             10009cae f   commonRef.obj
 0001:00008d29       _commonRef_pinAll          10009d29 f   commonRef.obj
 0001:00008def       _commonRef_refToID         10009def f   commonRef.obj
 0001:00008e64       _commonRef_release         10009e64 f   commonRef.obj
 0001:00008e9b       _commonRef_releaseMultiple 10009e9b f   commonRef.obj
 0001:00008ed4       _commonRef_reset           10009ed4 f   commonRef.obj
 0001:00008f87       _commonRef_unlock          10009f87 f   commonRef.obj
 0001:00008f99       _commonRef_unpin           10009f99 f   commonRef.obj
 0001:00008ff3       _commonRef_unpinAll        10009ff3 f   commonRef.obj
 0001:00009832       _debugDispatch_getHandler  1000a832 f   debugDispatch.obj
 0001:00009885       _debugDispatch_initialize  1000a885 f   debugDispatch.obj
 0001:0000996c       @_guard_check_icall_nop@4  1000a96c f   MSVCRT:guard_support.obj
 0001:0000996c       _util_reset                1000a96c f   util.obj
 0001:0000996c       _standardHandlers_onDisconnect 1000a96c f   standardHandlers.obj
 0001:0000996c       _stepControl_reset         1000a96c f   stepControl.obj
 0001:0000996c       _debugDispatch_reset       1000a96c f   debugDispatch.obj
 0001:0000996c       _invoker_reset             1000a96c f   invoker.obj
 0001:0000996f       _Agent_OnLoad@12           1000a96f f   debugInit.obj
 0001:00009e33       _Agent_OnUnload@4          1000ae33 f   debugInit.obj
 0001:0000a458       _debugInit_exit            1000b458 f   debugInit.obj
 0001:0000a539       _debugInit_isInitComplete  1000b539 f   debugInit.obj
 0001:0000a53f       _debugInit_launchOnInit    1000b53f f   debugInit.obj
 0001:0000a545       _debugInit_reset           1000b545 f   debugInit.obj
 0001:0000a62f       _debugInit_startDebuggingViaCommand@20 1000b62f f   debugInit.obj
 0001:0000a6bf       _debugInit_suspendOnInit   1000b6bf f   debugInit.obj
 0001:0000a6c5       _debugInit_waitInitComplete 1000b6c5 f   debugInit.obj
 0001:0000a795       _forceExit                 1000b795 f   debugInit.obj
 0001:0000b81c       _debugLoop_initialize      1000c81c f   debugLoop.obj
 0001:0000b82d       _debugLoop_run             1000c82d f   debugLoop.obj
 0001:0000ba78       _debugLoop_sync            1000ca78 f   debugLoop.obj
 0001:0000bccd       __vfprintf_l               1000cccd f i error_messages.obj
 0001:0000bcf1       _do_pause                  1000ccf1 f   error_messages.obj
 0001:0000bd4c       _error_message             1000cd4c f   error_messages.obj
 0001:0000bdc3       _eventText                 1000cdc3 f   error_messages.obj
 0001:0000be8b       _fprintf                   1000ce8b f i error_messages.obj
 0001:0000bea3       _jdiAssertionFailed        1000cea3 f   error_messages.obj
 0001:0000bf61       _jdwpErrorText             1000cf61 f   error_messages.obj
 0001:0000c227       _jvmtiErrorText            1000d227 f   error_messages.obj
 0001:0000c5f1       _print_message             1000d5f1 f   error_messages.obj
 0001:0000c60e       _tty_message               1000d60e f   error_messages.obj
 0001:0000ca3a       _eventFilterRestricted_alloc 1000da3a f   eventFilter.obj
 0001:0000ca7b       _eventFilterRestricted_deinstall 1000da7b f   eventFilter.obj
 0001:0000ca99       _eventFilterRestricted_install 1000da99 f   eventFilter.obj
 0001:0000ca9e       _eventFilterRestricted_isBreakpointInClass 1000da9e f   eventFilter.obj
 0001:0000cad2       _eventFilterRestricted_passesFilter 1000dad2 f   eventFilter.obj
 0001:0000ceca       _eventFilterRestricted_passesUnloadFilter 1000deca f   eventFilter.obj
 0001:0000cfc1       _eventFilter_predictFiltering 1000dfc1 f   eventFilter.obj
 0001:0000d0b6       _eventFilter_setClassExcludeFilter 1000e0b6 f   eventFilter.obj
 0001:0000d0ed       _eventFilter_setClassMatchFilter 1000e0ed f   eventFilter.obj
 0001:0000d124       _eventFilter_setClassOnlyFilter 1000e124 f   eventFilter.obj
 0001:0000d176       _eventFilter_setConditionalFilter 1000e176 f   eventFilter.obj
 0001:0000d1a1       _eventFilter_setCountFilter 1000e1a1 f   eventFilter.obj
 0001:0000d1d9       _eventFilter_setExceptionOnlyFilter 1000e1d9 f   eventFilter.obj
 0001:0000d235       _eventFilter_setFieldOnlyFilter 1000e235 f   eventFilter.obj
 0001:0000d288       _eventFilter_setInstanceOnlyFilter 1000e288 f   eventFilter.obj
 0001:0000d2d0       _eventFilter_setLocationOnlyFilter 1000e2d0 f   eventFilter.obj
 0001:0000d341       _eventFilter_setSourceNameMatchFilter 1000e341 f   eventFilter.obj
 0001:0000d372       _eventFilter_setStepFilter 1000e372 f   eventFilter.obj
 0001:0000d3fc       _eventFilter_setThreadOnlyFilter 1000e3fc f   eventFilter.obj
 0001:0000d59f       _isBreakpointSet           1000e59f f   eventFilter.obj
 0001:0000f92b       _eventHandlerRestricted_iterator 1001092b f   eventHandler.obj
 0001:0000f9b4       _eventHandler_alloc        100109b4 f   eventHandler.obj
 0001:0000f9d5       _eventHandler_allocHandlerID 100109d5 f   eventHandler.obj
 0001:0000f9ff       _eventHandler_createInternalBreakpoint 100109ff f   eventHandler.obj
 0001:0000fa22       _eventHandler_createInternalThreadOnly 10010a22 f   eventHandler.obj
 0001:0000fa3e       _eventHandler_createPermanentInternal 10010a3e f   eventHandler.obj
 0001:0000fa58       _eventHandler_free         10010a58 f   eventHandler.obj
 0001:0000fa81       _eventHandler_freeAll      10010a81 f   eventHandler.obj
 0001:0000facd       _eventHandler_freeByID     10010acd f   eventHandler.obj
 0001:0000fb1a       _eventHandler_freeClassBreakpoints 10010b1a f   eventHandler.obj
 0001:0000fb70       _eventHandler_initialize   10010b70 f   eventHandler.obj
 0001:0000ff97       _eventHandler_installExternal 10010f97 f   eventHandler.obj
 0001:0000ffb3       _eventHandler_lock         10010fb3 f   eventHandler.obj
 0001:0000ffc0       _eventHandler_reset        10010fc0 f   eventHandler.obj
 0001:00010024       _eventHandler_unlock       10011024 f   eventHandler.obj
 0001:00010427       _getMethodClass            10011427 f   eventHandler.obj
 0001:0001091f       _commandLoop_exitVmDeathLockOnError 1001191f f   eventHelper.obj
 0001:00010a47       _commandLoop_sync          10011a47 f   eventHelper.obj
 0001:00010d07       _eventHelper_createEventBag 10011d07 f   eventHelper.obj
 0001:00010d13       _eventHelper_holdEvents    10011d13 f   eventHelper.obj
 0001:00010d3f       _eventHelper_initialize    10011d3f f   eventHelper.obj
 0001:00010db7       _eventHelper_lock          10011db7 f   eventHelper.obj
 0001:00010dd0       _eventHelper_recordClassUnload 10011dd0 f   eventHelper.obj
 0001:00010e41       _eventHelper_recordEvent   10011e41 f   eventHelper.obj
 0001:00010ed4       _eventHelper_recordFrameEvent 10011ed4 f   eventHelper.obj
 0001:00010ffe       _eventHelper_releaseEvents 10011ffe f   eventHelper.obj
 0001:0001102a       _eventHelper_reportEvents  1001202a f   eventHelper.obj
 0001:000110fb       _eventHelper_reportInvokeDone 100120fb f   eventHelper.obj
 0001:00011191       _eventHelper_reportVMInit  10012191 f   eventHelper.obj
 0001:00011228       _eventHelper_reset         10012228 f   eventHelper.obj
 0001:00011262       _eventHelper_suspendThread 10012262 f   eventHelper.obj
 0001:000112f8       _eventHelper_unlock        100122f8 f   eventHelper.obj
 0001:000119bb       _unblockCommandLoop        100129bb f   eventHelper.obj
 0001:00011cde       _dbgsysExec                10012cde f   exec_md.obj
 0001:00011d3e       _inStream_clearError       10012d3e f   inStream.obj
 0001:00011d49       _inStream_command          10012d49 f   inStream.obj
 0001:00011d51       _inStream_destroy          10012d51 f   inStream.obj
 0001:00011d85       _inStream_error            10012d85 f   inStream.obj
 0001:00011d8e       _inStream_id               10012d8e f   inStream.obj
 0001:00011d96       _inStream_init             10012d96 f   inStream.obj
 0001:00011ddb       _inStream_readArrayRef     10012ddb f   inStream.obj
 0001:00011e12       _inStream_readBoolean      10012e12 f   inStream.obj
 0001:00011e44       _inStream_readByte         10012e44 f   inStream.obj
 0001:00011e62       _inStream_readBytes        10012e62 f   inStream.obj
 0001:00011e7b       _inStream_readChar         10012e7b f   inStream.obj
 0001:00011ea4       _inStream_readClassLoaderRef 10012ea4 f   inStream.obj
 0001:00011edb       _inStream_readClassRef     10012edb f   inStream.obj
 0001:00011f10       _inStream_readDouble       10012f10 f   inStream.obj
 0001:00011f3f       _inStream_readMethodID     10012f3f f   inStream.obj
 0001:00011f3f       _inStream_readFieldID      10012f3f f   inStream.obj
 0001:00011f44       _inStream_readFloat        10012f44 f   inStream.obj
 0001:00011f6e       _inStream_readLocation     10012f6e f   inStream.obj
 0001:00011f6e       _inStream_readFrameID      10012f6e f   inStream.obj
 0001:00011f6e       _inStream_readObjectID     10012f6e f   inStream.obj
 0001:00011f73       _inStream_readInt          10012f73 f   inStream.obj
 0001:00011fb4       _inStream_readLong         10012fb4 f   inStream.obj
 0001:00012060       _inStream_readModuleRef    10013060 f   inStream.obj
 0001:00012087       _inStream_readObjectRef    10013087 f   inStream.obj
 0001:000120e2       _inStream_readShort        100130e2 f   inStream.obj
 0001:0001210d       _inStream_readString       1001310d f   inStream.obj
 0001:00012173       _inStream_readStringRef    10013173 f   inStream.obj
 0001:000121aa       _inStream_readThreadGroupRef 100131aa f   inStream.obj
 0001:000121df       _inStream_readThreadRef    100131df f   inStream.obj
 0001:00012214       _inStream_readValue        10013214 f   inStream.obj
 0001:00013636       _invoker_completeInvokeRequest 10014636 f   invoker.obj
 0001:000138f8       _invoker_detach            100148f8 f   invoker.obj
 0001:00013945       _invoker_doInvoke          10014945 f   invoker.obj
 0001:00013b7a       _invoker_enableInvokeRequests 10014b7a f   invoker.obj
 0001:00013c1d       _invoker_initialize        10014c1d f   invoker.obj
 0001:00013c2e       _invoker_isEnabled         10014c2e f   invoker.obj
 0001:00013cd2       _invoker_lock              10014cd2 f   invoker.obj
 0001:00013cdf       _invoker_requestInvoke     10014cdf f   invoker.obj
 0001:00013d77       _invoker_unlock            10014d77 f   invoker.obj
 0001:00013d84       _dbgsysBuildLibName        10014d84 f   linker_md.obj
 0001:00013e16       _dbgsysFindLibraryEntry    10014e16 f   linker_md.obj
 0001:00013e25       _dbgsysGetLastErrorString  10014e25 f   linker_md.obj
 0001:00013ec4       _dbgsysLoadLibrary         10014ec4 f   linker_md.obj
 0001:00013fff       _sprintf                   10014fff f i linker_md.obj
 0001:00014075       _finish_logging            10015075 f   log_messages.obj
 0001:00014155       _log_message_begin         10015155 f   log_messages.obj
 0001:0001416b       _log_message_end           1001516b f   log_messages.obj
 0001:00014298       _setup_logging             10015298 f   log_messages.obj
 0001:00014341       _outStream_destroy         10015341 f   outStream.obj
 0001:00014399       _outStream_error           10015399 f   outStream.obj
 0001:000143a2       _outStream_initCommand     100153a2 f   outStream.obj
 0001:000143cb       _outStream_initReply       100153cb f   outStream.obj
 0001:0001447a       _outStream_sendCommand     1001547a f   outStream.obj
 0001:00014496       _outStream_sendReply       10015496 f   outStream.obj
 0001:000144be       _outStream_setError        100154be f   outStream.obj
 0001:00014512       _outStream_writeBoolean    10015512 f   outStream.obj
 0001:00014530       _outStream_writeByte       10015530 f   outStream.obj
 0001:00014544       _outStream_writeByteArray  10015544 f   outStream.obj
 0001:00014565       _outStream_writeChar       10015565 f   outStream.obj
 0001:00014589       _outStream_writeDouble     10015589 f   outStream.obj
 0001:000145b3       _outStream_writeFieldID    100155b3 f   outStream.obj
 0001:000145b3       _outStream_writeMethodID   100155b3 f   outStream.obj
 0001:000145b8       _outStream_writeFloat      100155b8 f   outStream.obj
 0001:000145e1       _outStream_writeFrameID    100155e1 f   outStream.obj
 0001:000145e1       _outStream_writeLocation   100155e1 f   outStream.obj
 0001:000145f6       _outStream_writeInt        100155f6 f   outStream.obj
 0001:00014635       _outStream_writeLong       10015635 f   outStream.obj
 0001:000146da       _outStream_writeModuleRef  100156da f   outStream.obj
 0001:000146df       _outStream_writeObjectRef  100156df f   outStream.obj
 0001:000148c6       _outStream_writeObjectTag  100158c6 f   outStream.obj
 0001:000148e4       _outStream_writeShort      100158e4 f   outStream.obj
 0001:00014910       _outStream_writeString     10015910 f   outStream.obj
 0001:000149b9       _outStream_writeValue      100159b9 f   outStream.obj
 0001:00014bcf       _componentTypeSignature    10015bcf f   signature.obj
 0001:00014ce1       _convertSignatureToClassname 10015ce1 f   signature.obj
 0001:00014d14       _methodSignature_init      10015d14 f   signature.obj
 0001:00014d4c       _methodSignature_nextArgumentExists 10015d4c f   signature.obj
 0001:00014e1a       _methodSignature_returnTag 10015e1a f   signature.obj
 0001:00014fc0       _standardHandlers_defaultHandler 10015fc0 f   standardHandlers.obj
 0001:0001501c       _standardHandlers_onConnect 1001601c f   standardHandlers.obj
 0001:00015bca       _stepControl_beginStep     10016bca f   stepControl.obj
 0001:00015cf8       _stepControl_clearRequest  10016cf8 f   stepControl.obj
 0001:00015d30       _stepControl_endStep       10016d30 f   stepControl.obj
 0001:00015da2       _stepControl_handleStep    10016da2 f   stepControl.obj
 0001:00016357       _stepControl_initialize    10017357 f   stepControl.obj
 0001:00016368       _stepControl_lock          10017368 f   stepControl.obj
 0001:00016375       _stepControl_resetRequest  10017375 f   stepControl.obj
 0001:0001643e       _stepControl_unlock        1001743e f   stepControl.obj
 0001:0001644b       _stream_encodeDouble       1001744b f   stream.obj
 0001:000164ed       _stream_encodeFloat        100174ed f   stream.obj
 0001:00017db0       _threadControl_addDebugThread 10018db0 f   threadControl.obj
 0001:00017e16       _threadControl_applicationThreadStatus 10018e16 f   threadControl.obj
 0001:00017e9a       _threadControl_clearCLEInfo 10018e9a f   threadControl.obj
 0001:00017ee4       _threadControl_cmpCLEInfo  10018ee4 f   threadControl.obj
 0001:00017f64       _threadControl_currentThread 10018f64 f   threadControl.obj
 0001:00017f96       _threadControl_detachInvokes 10018f96 f   threadControl.obj
 0001:00017fd4       _threadControl_getFrameGeneration 10018fd4 f   threadControl.obj
 0001:00018017       _threadControl_getInstructionStepMode 10019017 f   threadControl.obj
 0001:0001804d       _threadControl_getInvokeRequest 1001904d f   threadControl.obj
 0001:00018083       _threadControl_getStepRequest 10019083 f   threadControl.obj
 0001:000180b9       _threadControl_initialize  100190b9 f   threadControl.obj
 0001:000181e6       _threadControl_interrupt   100191e6 f   threadControl.obj
 0001:0001827c       _threadControl_isDebugThread 1001927c f   threadControl.obj
 0001:000182d5       _threadControl_onConnect   100192d5 f   threadControl.obj
 0001:00018301       _threadControl_onDisconnect 10019301 f   threadControl.obj
 0001:00018347       _threadControl_onEventHandlerEntry 10019347 f   threadControl.obj
 0001:000184a0       _threadControl_onEventHandlerExit 100194a0 f   threadControl.obj
 0001:00018588       _threadControl_onHook      10019588 f   threadControl.obj
 0001:00018678       _threadControl_popFrames   10019678 f   threadControl.obj
 0001:000187f8       _threadControl_reset       100197f8 f   threadControl.obj
 0001:000188c7       _threadControl_resumeAll   100198c7 f   threadControl.obj
 0001:00018956       _threadControl_resumeThread 10019956 f   threadControl.obj
 0001:000189cb       _threadControl_saveCLEInfo 100199cb f   threadControl.obj
 0001:00018a38       _threadControl_setEventMode 10019a38 f   threadControl.obj
 0001:00018afa       _threadControl_setPendingInterrupt 10019afa f   threadControl.obj
 0001:00018b2b       _threadControl_stop        10019b2b f   threadControl.obj
 0001:00018bdc       _threadControl_suspendAll  10019bdc f   threadControl.obj
 0001:00018cbb       _threadControl_suspendCount 10019cbb f   threadControl.obj
 0001:00018d0b       _threadControl_suspendThread 10019d0b f   threadControl.obj
 0001:00019671       _transport_close           1001a671 f   transport.obj
 0001:00019682       _transport_initialize      1001a682 f   transport.obj
 0001:000196ab       _transport_is_open         1001a6ab f   transport.obj
 0001:000196be       _transport_receivePacket   1001a6be f   transport.obj
 0001:00019701       _transport_reset           1001a701 f   transport.obj
 0001:00019739       _transport_sendPacket      1001a739 f   transport.obj
 0001:000197a3       _transport_startTransport  1001a7a3 f   transport.obj
 0001:00019a9e       _transport_waitForConnection 1001aa9e f   transport.obj
 0001:00019bb8       _utf8FromPlatform@16       1001abb8 f   utf_util.obj
 0001:00019cbb       _utf8ToPlatform@16         1001acbb f   utf_util.obj
 0001:00019dbb       _utf8mToUtf8s@16           1001adbb f   utf_util.obj
 0001:00019f52       _utf8mToUtf8sLength@8      1001af52 f   utf_util.obj
 0001:0001a032       _utf8sToUtf8m@16           1001b032 f   utf_util.obj
 0001:0001a17b       _utf8sToUtf8mLength@8      1001b17b f   utf_util.obj
 0001:0001a264       _allClassLoaderClasses     1001b264 f   util.obj
 0001:0001a2c1       _allInterfaces             1001b2c1 f   util.obj
 0001:0001a31e       _allLoadedClasses          1001b31e f   util.obj
 0001:0001a377       _allNestedClasses          1001b377 f   util.obj
 0001:0001a71e       _allThreads                1001b71e f   util.obj
 0001:0001a94e       _classInstanceCounts       1001b94e f   util.obj
 0001:0001aba7       _classInstances            1001bba7 f   util.obj
 0001:0001ad45       _classLoader               1001bd45 f   util.obj
 0001:0001ad98       _classSignature            1001bd98 f   util.obj
 0001:0001ae9d       _classStatus               1001be9d f   util.obj
 0001:0001af3c       _createLocalRefSpace       1001bf3c f   util.obj
 0001:0001b074       _debugMonitorCreate        1001c074 f   util.obj
 0001:0001b10d       _debugMonitorDestroy       1001c10d f   util.obj
 0001:0001b1a2       _debugMonitorEnter         1001c1a2 f   util.obj
 0001:0001b23a       _debugMonitorExit          1001c23a f   util.obj
 0001:0001b2d2       _debugMonitorNotify        1001c2d2 f   util.obj
 0001:0001b36a       _debugMonitorNotifyAll     1001c36a f   util.obj
 0001:0001b402       _debugMonitorTimedWait     1001c402 f   util.obj
 0001:0001b4ae       _debugMonitorWait          1001c4ae f   util.obj
 0001:0001b556       _eventIndex2jdwp           1001c556 f   util.obj
 0001:0001b5b7       _eventIndex2jvmti          1001c5b7 f   util.obj
 0001:0001b619       _eventIndexInit            1001c619 f   util.obj
 0001:0001b6b1       _fieldModifiers            1001c6b1 f   util.obj
 0001:0001b708       _fieldSignature            1001c708 f   util.obj
 0001:0001b96e       _filterDebugThreads        1001c96e f   util.obj
 0001:0001b9a4       _findClass                 1001c9a4 f   util.obj
 0001:0001bbba       _getClassname              1001cbba f   util.obj
 0001:0001bbec       _getEnv                    1001cbec f   util.obj
 0001:0001bc9e       _getMethod                 1001cc9e f   util.obj
 0001:0001c2af       _getSourceDebugExtension   1001d2af f   util.obj
 0001:0001c2fc       _getSpecialJvmti           1001d2fc f   util.obj
 0001:0001c700       _isArray                   1001d700 f   util.obj
 0001:0001c83b       _isClass                   1001d83b f   util.obj
 0001:0001c890       _isClassLoader             1001d890 f   util.obj
 0001:0001c8e5       _isFieldSynthetic          1001d8e5 f   util.obj
 0001:0001c9e3       _isMethodNative            1001d9e3 f   util.obj
 0001:0001ca83       _isMethodObsolete          1001da83 f   util.obj
 0001:0001caef       _isMethodSynthetic         1001daef f   util.obj
 0001:0001cb49       _isObjectTag               1001db49 f   util.obj
 0001:0001cb6f       _isSameObject              1001db6f f   util.obj
 0001:0001cb8c       _isString                  1001db8c f   util.obj
 0001:0001cbe1       _isThread                  1001dbe1 f   util.obj
 0001:0001cc36       _isThreadGroup             1001dc36 f   util.obj
 0001:0001ccea       _jdwp2EventIndex           1001dcea f   util.obj
 0001:0001cdb6       _jvmtiAllocate             1001ddb6 f   util.obj
 0001:0001ce61       _jvmtiDeallocate           1001de61 f   util.obj
 0001:0001cefd       _jvmtiGetCapabilities      1001defd f   util.obj
 0001:0001cf83       _jvmtiMajorVersion         1001df83 f   util.obj
 0001:0001cf91       _jvmtiMicroVersion         1001df91 f   util.obj
 0001:0001cf9a       _jvmtiMinorVersion         1001df9a f   util.obj
 0001:0001d049       _log_debugee_location      1001e049 f   util.obj
 0001:0001d350       _map2jdwpClassStatus       1001e350 f   util.obj
 0001:0001d37f       _map2jdwpError             1001e37f f   util.obj
 0001:0001d64e       _map2jdwpSuspendStatus     1001e64e f   util.obj
 0001:0001d659       _map2jdwpThreadStatus      1001e659 f   util.obj
 0001:0001d697       _map2jvmtiError            1001e697 f   util.obj
 0001:0001d906       _methodClass               1001e906 f   util.obj
 0001:0001d959       _methodLocation            1001e959 f   util.obj
 0001:0001d9aa       _methodModifiers           1001e9aa f   util.obj
 0001:0001d9fd       _methodReturnType          1001e9fd f   util.obj
 0001:0001dae6       _methodSignature           1001eae6 f   util.obj
 0001:0001dd48       _objectReferrers           1001ed48 f   util.obj
 0001:0001dfa7       _referenceTypeTag          1001efa7 f   util.obj
 0001:0001dfcd       _saveGlobalRef             1001efcd f   util.obj
 0001:0001e179       _setAgentPropertyValue     1001f179 f   util.obj
 0001:0001e325       _sharedGetFieldValues      1001f325 f   util.obj
 0001:0001e427       _sharedInvoke              1001f427 f   util.obj
 0001:0001e5c4       _spawnNewThread            1001f5c4 f   util.obj
 0001:0001e8e5       _specificTypeKey           1001f8e5 f   util.obj
 0001:0001eb09       _threadGroupInfo           1001fb09 f   util.obj
 0001:0001eb9b       _tossGlobalRef             1001fb9b f   util.obj
 0001:0001ecca       _uniqueID                  1001fcca f   util.obj
 0001:0001ecd9       _util_initialize           1001fcd9 f   util.obj
 0001:0001f236       _writeCodeLocation         10020236 f   util.obj
 0001:0001f6fd       _writeGenericSignature     100206fd f   util.obj
 0001:0001fb3f       @__security_check_cookie@4 10020b3f f   MSVCRT:secchk.obj
 0001:0001fb94       ___scrt_acquire_startup_lock 10020b94 f   MSVCRT:utility.obj
 0001:0001fbc6       ___scrt_dllmain_after_initialize_c 10020bc6 f   MSVCRT:utility.obj
 0001:0001fbf1       ___scrt_dllmain_before_initialize_c 10020bf1 f   MSVCRT:utility.obj
 0001:0001fbff       ___scrt_dllmain_crt_thread_attach 10020bff f   MSVCRT:utility.obj
 0001:0001fc1e       ___scrt_dllmain_crt_thread_detach 10020c1e f   MSVCRT:utility.obj
 0001:0001fc2b       ___scrt_dllmain_exception_filter 10020c2b f   MSVCRT:utility.obj
 0001:0001fc5f       ___scrt_dllmain_uninitialize_c 10020c5f f   MSVCRT:utility.obj
 0001:0001fc82       ___scrt_dllmain_uninitialize_critical 10020c82 f   MSVCRT:utility.obj
 0001:0001fc8f       ___scrt_initialize_crt     10020c8f f   MSVCRT:utility.obj
 0001:0001fcc8       ___scrt_initialize_onexit_tables 10020cc8 f   MSVCRT:utility.obj
 0001:0001fd4f       ___scrt_is_nonwritable_in_current_image 10020d4f f   MSVCRT:utility.obj
 0001:0001fde3       ___scrt_release_startup_lock 10020de3 f   MSVCRT:utility.obj
 0001:0001fe00       ___scrt_uninitialize_crt   10020e00 f   MSVCRT:utility.obj
 0001:0001fe28       __onexit                   10020e28 f   MSVCRT:utility.obj
 0001:0001fe55       _atexit                    10020e55 f   MSVCRT:utility.obj
 0001:000201aa       __DllMainCRTStartup@12     100211aa f   MSVCRT:dll_dllmain.obj
 0001:000201cd       ___raise_securityfailure   100211cd f   MSVCRT:gs_report.obj
 0001:000201f5       ___report_gsfailure        100211f5 f   MSVCRT:gs_report.obj
 0001:000202ee       ___isa_available_init      100212ee f   MSVCRT:cpu_disp.obj
 0001:000204be       __get_startup_argv_mode    100214be f   MSVCRT:argv_mode.obj
 0001:000204c2       ___scrt_is_ucrt_dll_in_use 100214c2 f   MSVCRT:ucrt_detection.obj
 0001:000204ce       ___scrt_fastfail           100214ce f   MSVCRT:utility_desktop.obj
 0001:000205e8       __crt_debugger_hook        100215e8 f   MSVCRT:utility_desktop.obj
 0001:000205f0       __SEH_prolog4              100215f0 f   MSVCRT:sehprolg4.obj
 0001:00020634       __SEH_epilog4              10021634 f   MSVCRT:sehprolg4.obj
 0001:00020648       __except_handler4          10021648 f   MSVCRT:chandler4gs.obj
 0001:000206c4       ___security_init_cookie    100216c4 f   MSVCRT:gs_support.obj
 0001:0002070f       _DllMain@12                1002170f f   MSVCRT:dll_dllmain_stub.obj
 0001:00020731       ?__scrt_initialize_type_info@@YAXXZ 10021731 f   MSVCRT:tncleanup.obj
 0001:0002073d       ?__scrt_uninitialize_type_info@@YAXXZ 1002173d f   MSVCRT:tncleanup.obj
 0001:00020749       ___local_stdio_scanf_options 10021749 f i MSVCRT:default_local_stdio_options.obj
 0001:0002074f       ___scrt_initialize_default_local_stdio_options 1002174f f   MSVCRT:default_local_stdio_options.obj
 0001:0002076c       ___scrt_get_dyn_tls_init_callback 1002176c f   MSVCRT:dyn_tls_init.obj
 0001:00020772       __RTC_Initialize           10021772 f   MSVCRT:initsect.obj
 0001:0002079e       __RTC_Terminate            1002179e f   MSVCRT:initsect.obj
 0001:000207ca       _IsProcessorFeaturePresent@4 100217ca f   kernel32:KERNEL32.dll
 0001:000207d0       _memset                    100217d0 f   vcruntime:VCRUNTIME140.dll
 0001:000207d6       _longjmp                   100217d6 f   vcruntime:VCRUNTIME140.dll
 0001:000207dc       _memcpy                    100217dc f   vcruntime:VCRUNTIME140.dll
 0001:000207e2       __setjmp3                  100217e2 f   vcruntime:VCRUNTIME140.dll
 0001:000207e8       _strchr                    100217e8 f   vcruntime:VCRUNTIME140.dll
 0001:000207ee       _strrchr                   100217ee f   vcruntime:VCRUNTIME140.dll
 0001:000207f4       __except_handler4_common   100217f4 f   vcruntime:VCRUNTIME140.dll
 0001:000207fa       ___std_type_info_destroy_list 100217fa f   vcruntime:VCRUNTIME140.dll
 0001:00020800       _strcmp                    10021800 f   ucrt:api-ms-win-crt-string-l1-1-0.dll
 0001:00020806       _strlen                    10021806 f   ucrt:api-ms-win-crt-string-l1-1-0.dll
 0001:0002080c       _strcat                    1002180c f   ucrt:api-ms-win-crt-string-l1-1-0.dll
 0001:00020812       _strcpy                    10021812 f   ucrt:api-ms-win-crt-string-l1-1-0.dll
 0001:00020818       __seh_filter_dll           10021818 f   ucrt:api-ms-win-crt-runtime-l1-1-0.dll
 0001:0002081e       __configure_narrow_argv    1002181e f   ucrt:api-ms-win-crt-runtime-l1-1-0.dll
 0001:00020824       __initialize_narrow_environment 10021824 f   ucrt:api-ms-win-crt-runtime-l1-1-0.dll
 0001:0002082a       __initialize_onexit_table  1002182a f   ucrt:api-ms-win-crt-runtime-l1-1-0.dll
 0001:00020830       __register_onexit_function 10021830 f   ucrt:api-ms-win-crt-runtime-l1-1-0.dll
 0001:00020836       __execute_onexit_table     10021836 f   ucrt:api-ms-win-crt-runtime-l1-1-0.dll
 0001:0002083c       __crt_atexit               1002183c f   ucrt:api-ms-win-crt-runtime-l1-1-0.dll
 0001:00020842       __cexit                    10021842 f   ucrt:api-ms-win-crt-runtime-l1-1-0.dll
 0001:00020848       __initterm                 10021848 f   ucrt:api-ms-win-crt-runtime-l1-1-0.dll
 0001:0002084e       __initterm_e               1002184e f   ucrt:api-ms-win-crt-runtime-l1-1-0.dll
 0001:00020854       ___scrt_stub_for_is_c_termination_complete 10021854 f   MSVCRT:ucrt_stubs.obj
 0001:00020854       __is_c_termination_complete 10021854 f   MSVCRT:ucrt_stubs.obj
 0001:00020857       __filter_x86_sse2_floating_point_exception_default 10021857 f   MSVCRT:x86_exception_filter.obj
 0001:00020857       __filter_x86_sse2_floating_point_exception 10021857 f   MSVCRT:x86_exception_filter.obj
 0002:00000000       __imp__Sleep@4             10022000     kernel32:KERNEL32.dll
 0002:00000004       __imp__GetCurrentThreadId@0 10022004     kernel32:KERNEL32.dll
 0002:00000008       __imp__CreateProcessA@40   10022008     kernel32:KERNEL32.dll
 0002:0000000c       __imp__GetLastError@0      1002200c     kernel32:KERNEL32.dll
 0002:00000010       __imp__GetProcAddress@8    10022010     kernel32:KERNEL32.dll
 0002:00000014       __imp__LoadLibraryA@4      10022014     kernel32:KERNEL32.dll
 0002:00000018       __imp__FormatMessageA@28   10022018     kernel32:KERNEL32.dll
 0002:0000001c       __imp__MultiByteToWideChar@24 1002201c     kernel32:KERNEL32.dll
 0002:00000020       __imp__WideCharToMultiByte@32 10022020     kernel32:KERNEL32.dll
 0002:00000024       __imp__GetACP@0            10022024     kernel32:KERNEL32.dll
 0002:00000028       __imp__GetLocaleInfoA@16   10022028     kernel32:KERNEL32.dll
 0002:0000002c       __imp__GetUserDefaultLCID@0 1002202c     kernel32:KERNEL32.dll
 0002:00000030       __imp__UnhandledExceptionFilter@4 10022030     kernel32:KERNEL32.dll
 0002:00000034       __imp__SetUnhandledExceptionFilter@4 10022034     kernel32:KERNEL32.dll
 0002:00000038       __imp__GetCurrentProcess@0 10022038     kernel32:KERNEL32.dll
 0002:0000003c       __imp__TerminateProcess@8  1002203c     kernel32:KERNEL32.dll
 0002:00000040       __imp__IsProcessorFeaturePresent@4 10022040     kernel32:KERNEL32.dll
 0002:00000044       __imp__IsDebuggerPresent@0 10022044     kernel32:KERNEL32.dll
 0002:00000048       __imp__QueryPerformanceCounter@4 10022048     kernel32:KERNEL32.dll
 0002:0000004c       __imp__GetCurrentProcessId@0 1002204c     kernel32:KERNEL32.dll
 0002:00000050       __imp__GetSystemTimeAsFileTime@4 10022050     kernel32:KERNEL32.dll
 0002:00000054       __imp__DisableThreadLibraryCalls@4 10022054     kernel32:KERNEL32.dll
 0002:00000058       __imp__InitializeSListHead@4 10022058     kernel32:KERNEL32.dll
 0002:0000005c       \177KERNEL32_NULL_THUNK_DATA 1002205c     kernel32:KERNEL32.dll
 0002:00000060       __imp__memset              10022060     vcruntime:VCRUNTIME140.dll
 0002:00000064       __imp__longjmp             10022064     vcruntime:VCRUNTIME140.dll
 0002:00000068       __imp__memcpy              10022068     vcruntime:VCRUNTIME140.dll
 0002:0000006c       __imp___setjmp3            1002206c     vcruntime:VCRUNTIME140.dll
 0002:00000070       __imp__strchr              10022070     vcruntime:VCRUNTIME140.dll
 0002:00000074       __imp__strrchr             10022074     vcruntime:VCRUNTIME140.dll
 0002:00000078       __imp___except_handler4_common 10022078     vcruntime:VCRUNTIME140.dll
 0002:0000007c       __imp____std_type_info_destroy_list 1002207c     vcruntime:VCRUNTIME140.dll
 0002:00000080       \177VCRUNTIME140_NULL_THUNK_DATA 10022080     vcruntime:VCRUNTIME140.dll
 0002:00000084       __imp__atol                10022084     ucrt:api-ms-win-crt-convert-l1-1-0.dll
 0002:00000088       __imp__atoi                10022088     ucrt:api-ms-win-crt-convert-l1-1-0.dll
 0002:0000008c       __imp__strtol              1002208c     ucrt:api-ms-win-crt-convert-l1-1-0.dll
 0002:00000090       \177api-ms-win-crt-convert-l1-1-0_NULL_THUNK_DATA 10022090     ucrt:api-ms-win-crt-convert-l1-1-0.dll
 0002:00000094       __imp__getenv              10022094     ucrt:api-ms-win-crt-environment-l1-1-0.dll
 0002:00000098       \177api-ms-win-crt-environment-l1-1-0_NULL_THUNK_DATA 10022098     ucrt:api-ms-win-crt-environment-l1-1-0.dll
 0002:0000009c       __imp___access             1002209c     ucrt:api-ms-win-crt-filesystem-l1-1-0.dll
 0002:000000a0       \177api-ms-win-crt-filesystem-l1-1-0_NULL_THUNK_DATA 100220a0     ucrt:api-ms-win-crt-filesystem-l1-1-0.dll
 0002:000000a4       __imp__malloc              100220a4     ucrt:api-ms-win-crt-heap-l1-1-0.dll
 0002:000000a8       __imp__free                100220a8     ucrt:api-ms-win-crt-heap-l1-1-0.dll
 0002:000000ac       \177api-ms-win-crt-heap-l1-1-0_NULL_THUNK_DATA 100220ac     ucrt:api-ms-win-crt-heap-l1-1-0.dll
 0002:000000b0       __imp__abort               100220b0     ucrt:api-ms-win-crt-runtime-l1-1-0.dll
 0002:000000b4       __imp__getpid              100220b4     ucrt:api-ms-win-crt-runtime-l1-1-0.dll
 0002:000000b4       __imp___getpid             100220b4     ucrt:api-ms-win-crt-runtime-l1-1-0.dll
 0002:000000b8       __imp___errno              100220b8     ucrt:api-ms-win-crt-runtime-l1-1-0.dll
 0002:000000bc       __imp___initterm_e         100220bc     ucrt:api-ms-win-crt-runtime-l1-1-0.dll
 0002:000000c0       __imp__strerror            100220c0     ucrt:api-ms-win-crt-runtime-l1-1-0.dll
 0002:000000c4       __imp___initterm           100220c4     ucrt:api-ms-win-crt-runtime-l1-1-0.dll
 0002:000000c8       __imp__exit                100220c8     ucrt:api-ms-win-crt-runtime-l1-1-0.dll
 0002:000000cc       __imp___cexit              100220cc     ucrt:api-ms-win-crt-runtime-l1-1-0.dll
 0002:000000d0       __imp___crt_atexit         100220d0     ucrt:api-ms-win-crt-runtime-l1-1-0.dll
 0002:000000d4       __imp___execute_onexit_table 100220d4     ucrt:api-ms-win-crt-runtime-l1-1-0.dll
 0002:000000d8       __imp___register_onexit_function 100220d8     ucrt:api-ms-win-crt-runtime-l1-1-0.dll
 0002:000000dc       __imp___initialize_onexit_table 100220dc     ucrt:api-ms-win-crt-runtime-l1-1-0.dll
 0002:000000e0       __imp___initialize_narrow_environment 100220e0     ucrt:api-ms-win-crt-runtime-l1-1-0.dll
 0002:000000e4       __imp___configure_narrow_argv 100220e4     ucrt:api-ms-win-crt-runtime-l1-1-0.dll
 0002:000000e8       __imp___seh_filter_dll     100220e8     ucrt:api-ms-win-crt-runtime-l1-1-0.dll
 0002:000000ec       \177api-ms-win-crt-runtime-l1-1-0_NULL_THUNK_DATA 100220ec     ucrt:api-ms-win-crt-runtime-l1-1-0.dll
 0002:000000f0       __imp__fflush              100220f0     ucrt:api-ms-win-crt-stdio-l1-1-0.dll
 0002:000000f4       __imp____stdio_common_vfprintf 100220f4     ucrt:api-ms-win-crt-stdio-l1-1-0.dll
 0002:000000f8       __imp__fclose              100220f8     ucrt:api-ms-win-crt-stdio-l1-1-0.dll
 0002:000000fc       __imp____acrt_iob_func     100220fc     ucrt:api-ms-win-crt-stdio-l1-1-0.dll
 0002:00000100       __imp__fopen               10022100     ucrt:api-ms-win-crt-stdio-l1-1-0.dll
 0002:00000104       __imp____stdio_common_vsprintf 10022104     ucrt:api-ms-win-crt-stdio-l1-1-0.dll
 0002:00000108       __imp__setvbuf             10022108     ucrt:api-ms-win-crt-stdio-l1-1-0.dll
 0002:0000010c       \177api-ms-win-crt-stdio-l1-1-0_NULL_THUNK_DATA 1002210c     ucrt:api-ms-win-crt-stdio-l1-1-0.dll
 0002:00000110       __imp__strncpy             10022110     ucrt:api-ms-win-crt-string-l1-1-0.dll
 0002:00000114       __imp__strtok_s            10022114     ucrt:api-ms-win-crt-string-l1-1-0.dll
 0002:00000118       __imp__strncmp             10022118     ucrt:api-ms-win-crt-string-l1-1-0.dll
 0002:0000011c       __imp__strlen              1002211c     ucrt:api-ms-win-crt-string-l1-1-0.dll
 0002:00000120       __imp__strcat              10022120     ucrt:api-ms-win-crt-string-l1-1-0.dll
 0002:00000124       __imp__isdigit             10022124     ucrt:api-ms-win-crt-string-l1-1-0.dll
 0002:00000128       __imp__strcmp              10022128     ucrt:api-ms-win-crt-string-l1-1-0.dll
 0002:0000012c       __imp__strcpy              1002212c     ucrt:api-ms-win-crt-string-l1-1-0.dll
 0002:00000130       \177api-ms-win-crt-string-l1-1-0_NULL_THUNK_DATA 10022130     ucrt:api-ms-win-crt-string-l1-1-0.dll
 0002:00000134       __imp___time64             10022134     ucrt:api-ms-win-crt-time-l1-1-0.dll
 0002:00000138       __imp__strftime            10022138     ucrt:api-ms-win-crt-time-l1-1-0.dll
 0002:0000013c       __imp___localtime64        1002213c     ucrt:api-ms-win-crt-time-l1-1-0.dll
 0002:00000140       \177api-ms-win-crt-time-l1-1-0_NULL_THUNK_DATA 10022140     ucrt:api-ms-win-crt-time-l1-1-0.dll
 0002:00000144       ___guard_check_icall_fptr  10022144     MSVCRT:guard_support.obj
 0002:00000148       ___xc_a                    10022148     MSVCRT:initializers.obj
 0002:0000014c       ___xc_z                    1002214c     MSVCRT:initializers.obj
 0002:00000150       ___xi_a                    10022150     MSVCRT:initializers.obj
 0002:00000154       ___xi_z                    10022154     MSVCRT:initializers.obj
 0002:00000158       ___xp_a                    10022158     MSVCRT:initializers.obj
 0002:0000015c       ___xp_z                    1002215c     MSVCRT:initializers.obj
 0002:00000160       ___xt_a                    10022160     MSVCRT:initializers.obj
 0002:00000164       ___xt_z                    10022164     MSVCRT:initializers.obj
 0002:00000170       ??_C@_06MHCOIGNA@Length@   10022170     ArrayReferenceImpl.obj
 0002:00000178       ??_C@_09JHHNDJLP@GetValues@ 10022178     ArrayReferenceImpl.obj
 0002:00000184       ??_C@_09LJDIBICN@SetValues@ 10022184     ArrayReferenceImpl.obj
 0002:00000190       ??_C@_0P@EGNIMIAH@ArrayReference@ 10022190     ArrayReferenceImpl.obj
 0002:000001a0       ??_C@_0BM@KIOODJOG@Tag?5is?5not?5a?5JVM?5basic?5type@ 100221a0     ArrayReferenceImpl.obj
 0002:000001bc       ??_C@_0DG@KNIKPIPG@s?2src?2jdk?4jdwp?4agent?2share?2nati@ 100221bc     ArrayReferenceImpl.obj
 0002:000001f4       ??_C@_0DP@KOAIFEMO@s?2src?2jdk?4jdwp?4agent?2share?2nati@ 100221f4     ArrayReferenceImpl.obj
 0002:00000234       ??_C@_03HBKNMMDM@JNI@      10022234     ArrayReferenceImpl.obj
 0002:00000238       ??_C@_0P@KJGLIDCM@GetArrayLength@ 10022238     ArrayReferenceImpl.obj
 0002:00000248       ??_C@_04DLGOCPFH@?$CFs?$CI?$CJ@ 10022248     ArrayReferenceImpl.obj
 0002:00000250       ??_C@_0BG@DOJPBGJK@GetBooleanArrayRegion@ 10022250     ArrayReferenceImpl.obj
 0002:00000268       ??_C@_0BD@DBCKLPHC@GetByteArrayRegion@ 10022268     ArrayReferenceImpl.obj
 0002:0000027c       ??_C@_0BD@EJLOJIMH@GetCharArrayRegion@ 1002227c     ArrayReferenceImpl.obj
 0002:00000290       ??_C@_0BE@LJPMIBLN@GetShortArrayRegion@ 10022290     ArrayReferenceImpl.obj
 0002:000002a4       ??_C@_0BC@PAFAELMA@GetIntArrayRegion@ 100222a4     ArrayReferenceImpl.obj
 0002:000002b8       ??_C@_0BD@KDOJFBNI@GetLongArrayRegion@ 100222b8     ArrayReferenceImpl.obj
 0002:000002cc       ??_C@_0BE@JEOBKBHM@GetFloatArrayRegion@ 100222cc     ArrayReferenceImpl.obj
 0002:000002e0       ??_C@_0BF@HGGNLGEB@GetDoubleArrayRegion@ 100222e0     ArrayReferenceImpl.obj
 0002:000002f8       ??_C@_0BG@KEKOCCJB@GetObjectArrayElement@ 100222f8     ArrayReferenceImpl.obj
 0002:00000310       ??_C@_0BC@LPILBKGC@ExceptionOccurred@ 10022310     ArrayReferenceImpl.obj
 0002:00000324       ??_C@_0O@EMINCBBD@PopLocalFrame@ 10022324     ArrayReferenceImpl.obj
 0002:00000334       ??_C@_0P@NDOJPFLH@GetObjectClass@ 10022334     ArrayReferenceImpl.obj
 0002:00000344       ??_C@_0P@KFEGKDII@ExceptionClear@ 10022344     ArrayReferenceImpl.obj
 0002:00000354       ??_C@_0BG@MLMJMPNL@SetBooleanArrayRegion@ 10022354     ArrayReferenceImpl.obj
 0002:0000036c       ??_C@_0BD@MLAAIJJK@SetByteArrayRegion@ 1002236c     ArrayReferenceImpl.obj
 0002:00000380       ??_C@_0BD@LDJEKOCP@SetCharArrayRegion@ 10022380     ArrayReferenceImpl.obj
 0002:00000394       ??_C@_0BE@BHNHMBMB@SetShortArrayRegion@ 10022394     ArrayReferenceImpl.obj
 0002:000003a8       ??_C@_0BC@NFFLMANO@SetIntArrayRegion@ 100223a8     ArrayReferenceImpl.obj
 0002:000003bc       ??_C@_0BD@FJMDGHDA@SetLongArrayRegion@ 100223bc     ArrayReferenceImpl.obj
 0002:000003d0       ??_C@_0BE@DKMKOBAA@SetFloatArrayRegion@ 100223d0     ArrayReferenceImpl.obj
 0002:000003e4       ??_C@_0BF@CPHAKABG@SetDoubleArrayRegion@ 100223e4     ArrayReferenceImpl.obj
 0002:000003fc       ??_C@_0BG@FBPIPLNA@SetObjectArrayElement@ 100223fc     ArrayReferenceImpl.obj
 0002:00000414       ??_C@_05MBDEGLCK@ERROR@    10022414     ArrayReferenceImpl.obj
 0002:0000041c       ??_C@_0CG@CDCBEMAB@Invalid?5array?5component?5signatu@ 1002241c     ArrayReferenceImpl.obj
 0002:00000442       ??_C@_00CNPNBAHC@@         10022442     ArrayReferenceImpl.obj
 0002:00000444       ??_C@_0BD@HJCIAOFF@?$CFs?$CI?$CFd?$CJ?3?5?$CFs?5?$FL?$CFs?3?$CFd?$FN@ 10022444     ArrayReferenceImpl.obj
 0002:00000458       ??_C@_01EEMJAFIK@?6@       10022458     ArrayReferenceImpl.obj
 0002:0000045c       ??_C@_0BB@BCMBBBKH@JDWP?5exit?5error?5@ 1002245c     ArrayReferenceImpl.obj
 0002:00000470       ??_C@_0M@LPLNEPAH@NewInstance@ 10022470     ArrayTypeImpl.obj
 0002:0000047c       ??_C@_09MLBOOMFO@ArrayType@ 1002247c     ArrayTypeImpl.obj
 0002:00000488       ??_C@_0DK@KCBNOHN@s?2src?2jdk?4jdwp?4agent?2share?2nati@ 10022488     ArrayTypeImpl.obj
 0002:000004c4       ??_C@_0P@CNKIGBBL@NewObjectArray@ 100224c4     ArrayTypeImpl.obj
 0002:000004d4       ??_C@_0N@NGBLEHOM@NewByteArray@ 100224d4     ArrayTypeImpl.obj
 0002:000004e4       ??_C@_0N@BEEAOHOP@NewCharArray@ 100224e4     ArrayTypeImpl.obj
 0002:000004f4       ??_C@_0O@KEDKGJJM@NewFloatArray@ 100224f4     ArrayTypeImpl.obj
 0002:00000504       ??_C@_0P@DNODLKGI@NewDoubleArray@ 10022504     ArrayTypeImpl.obj
 0002:00000514       ??_C@_0M@PGNBGLNB@NewIntArray@ 10022514     ArrayTypeImpl.obj
 0002:00000520       ??_C@_0N@GNOMHAGO@NewLongArray@ 10022520     ArrayTypeImpl.obj
 0002:00000530       ??_C@_0O@IAEEJHKH@NewShortArray@ 10022530     ArrayTypeImpl.obj
 0002:00000540       ??_C@_0BA@IMLHDFCA@NewBooleanArray@ 10022540     ArrayTypeImpl.obj
 0002:00000550       ??_C@_0P@GEMMHMHN@VisibleClasses@ 10022550     ClassLoaderReferenceImpl.obj
 0002:00000560       ??_C@_0BF@MJJABFGE@ClassLoaderReference@ 10022560     ClassLoaderReferenceImpl.obj
 0002:00000578       ??_C@_0EF@FKFHKPAA@s?2src?2jdk?4jdwp?4agent?2share?2nati@ 10022578     ClassLoaderReferenceImpl.obj
 0002:000005c0       ??_C@_0O@MBFCJPMM@ReflectedType@ 100225c0     ClassObjectReferenceImpl.obj
 0002:000005d0       ??_C@_0BF@IJHAFOFB@ClassObjectReference@ 100225d0     ClassObjectReferenceImpl.obj
 0002:000005e8       ??_C@_0L@HFIGJMAA@Superclass@ 100225e8     ClassTypeImpl.obj
 0002:000005f4       ??_C@_0N@LGIJNKMO@InvokeMethod@ 100225f4     ClassTypeImpl.obj
 0002:00000604       ??_C@_09IAHDNMJ@ClassType@ 10022604     ClassTypeImpl.obj
 0002:00000610       ??_C@_0DK@CPJOGD@s?2src?2jdk?4jdwp?4agent?2share?2nati@ 10022610     ClassTypeImpl.obj
 0002:0000064c       ??_C@_0O@NPFONKNM@GetSuperclass@ 1002264c     ClassTypeImpl.obj
 0002:0000065c       ??_C@_0BF@NBNNHFAL@SetStaticObjectField@ 1002265c     ClassTypeImpl.obj
 0002:00000674       ??_C@_0BD@IANJADAE@SetStaticByteField@ 10022674     ClassTypeImpl.obj
 0002:00000688       ??_C@_0BD@ECICKDAH@SetStaticCharField@ 10022688     ClassTypeImpl.obj
 0002:0000069c       ??_C@_0BE@KCBAKIGK@SetStaticFloatField@ 1002269c     ClassTypeImpl.obj
 0002:000006b0       ??_C@_0BF@MBJGKOHI@SetStaticDoubleField@ 100226b0     ClassTypeImpl.obj
 0002:000006c8       ??_C@_0BC@ENOHANEJ@SetStaticIntField@ 100226c8     ClassTypeImpl.obj
 0002:000006dc       ??_C@_0BD@DLCODEIG@SetStaticLongField@ 100226dc     ClassTypeImpl.obj
 0002:000006f0       ??_C@_0BE@IGGOFGFB@SetStaticShortField@ 100226f0     ClassTypeImpl.obj
 0002:00000704       ??_C@_0BG@DJFBDJKI@SetStaticBooleanField@ 10022704     ClassTypeImpl.obj
 0002:0000071c       ??_C@_0L@CAMDCGEO@SetCommand@ 1002271c     EventRequestImpl.obj
 0002:00000728       ??_C@_0N@NDABFFGD@ClearCommand@ 10022728     EventRequestImpl.obj
 0002:00000738       ??_C@_0BE@IJFBELDD@ClearAllBreakpoints@ 10022738     EventRequestImpl.obj
 0002:0000074c       ??_C@_0N@PGGBGIFJ@EventRequest@ 1002274c     EventRequestImpl.obj
 0002:0000075c       ??_C@_05EPLKDJMH@Field@    1002275c     FieldImpl.obj
 0002:00000764       ??_C@_0O@IHENGMAG@InterfaceType@ 10022764     InterfaceTypeImpl.obj
 0002:00000774       ??_C@_09IPPJBAKB@LineTable@ 10022774     MethodImpl.obj
 0002:00000780       ??_C@_0O@CIFPCEPG@VariableTable@ 10022780     MethodImpl.obj
 0002:00000790       ??_C@_09EAOGBHHA@Bytecodes@ 10022790     MethodImpl.obj
 0002:0000079c       ??_C@_0L@IIIMIJNI@IsObsolete@ 1002279c     MethodImpl.obj
 0002:000007a8       ??_C@_0BK@ILPNHFLA@VariableTableWithGenerics@ 100227a8     MethodImpl.obj
 0002:000007c4       ??_C@_06KPKMBBIM@Method@   100227c4     MethodImpl.obj
 0002:000007cc       ??_C@_0DH@BMAMHHMB@s?2src?2jdk?4jdwp?4agent?2share?2nati@ 100227cc     MethodImpl.obj
 0002:00000804       ??_C@_05HENNLPPN@JVMTI@    10022804     MethodImpl.obj
 0002:0000080c       ??_C@_0BD@MHLEIAPA@GetLineNumberTable@ 1002280c     MethodImpl.obj
 0002:00000820       ??_C@_0BB@ELDBFBNO@GetArgumentsSize@ 10022820     MethodImpl.obj
 0002:00000834       ??_C@_0BG@JNJHMCNH@GetLocalVariableTable@ 10022834     MethodImpl.obj
 0002:0000084c       ??_C@_0N@JCOMJEBO@GetBytecodes@ 1002284c     MethodImpl.obj
 0002:0000085c       ??_C@_07MMGEHGCI@GetName@  1002285c     ModuleReferenceImpl.obj
 0002:00000864       ??_C@_0P@PKAIJGGP@GetClassLoader@ 10022864     ModuleReferenceImpl.obj
 0002:00000874       ??_C@_0BA@OGHCDEJN@ModuleReference@ 10022874     ModuleReferenceImpl.obj
 0002:00000884       ??_C@_0BD@EAPJBIJJ@Ljava?1lang?1Module?$DL@ 10022884     ModuleReferenceImpl.obj
 0002:00000898       ??_C@_0BF@FOHFOJOB@?$CI?$CJLjava?1lang?1String?$DL@ 10022898     ModuleReferenceImpl.obj
 0002:000008b0       ??_C@_07DFBCBEHO@getName@  100228b0     ModuleReferenceImpl.obj
 0002:000008b8       ??_C@_0EA@MKGDLANN@s?2src?2jdk?4jdwp?4agent?2share?2nati@ 100228b8     ModuleReferenceImpl.obj
 0002:000008f8       ??_C@_0BB@FFOMHKKA@CallObjectMethod@ 100228f8     ModuleReferenceImpl.obj
 0002:0000090c       ??_C@_0BC@EDLHHKLL@GetStringUTFChars@ 1002290c     ModuleReferenceImpl.obj
 0002:00000920       ??_C@_0BG@CNECBEKD@ReleaseStringUTFChars@ 10022920     ModuleReferenceImpl.obj
 0002:00000938       ??_C@_0BK@JHGGPLEI@?$CI?$CJLjava?1lang?1ClassLoader?$DL@ 10022938     ModuleReferenceImpl.obj
 0002:00000954       ??_C@_0P@HCMNKIPB@getClassLoader@ 10022954     ModuleReferenceImpl.obj
 0002:00000964       ??_C@_0O@EJIAIJCO@ReferenceType@ 10022964     ObjectReferenceImpl.obj
 0002:00000974       ??_C@_08JLEAJAG@?$DMunused?$DO@ 10022974     ObjectReferenceImpl.obj
 0002:00000980       ??_C@_0M@OFAPJLBC@MonitorInfo@ 10022980     ObjectReferenceImpl.obj
 0002:0000098c       ??_C@_0P@NMHCCJ@InvokeInstance@ 1002298c     ObjectReferenceImpl.obj
 0002:0000099c       ??_C@_0BC@IIMACDIN@DisableCollection@ 1002299c     ObjectReferenceImpl.obj
 0002:000009b0       ??_C@_0BB@MDMHJMHH@EnableCollection@ 100229b0     ObjectReferenceImpl.obj
 0002:000009c4       ??_C@_0M@FOFOOCGH@IsCollected@ 100229c4     ObjectReferenceImpl.obj
 0002:000009d0       ??_C@_0BB@CHKFAPKH@ReferringObjects@ 100229d0     ObjectReferenceImpl.obj
 0002:000009e4       ??_C@_0BA@PPKMBENC@ObjectReference@ 100229e4     ObjectReferenceImpl.obj
 0002:000009f8       ??_C@_0EA@CANAHBDF@s?2src?2jdk?4jdwp?4agent?2share?2nati@ 100229f8     ObjectReferenceImpl.obj
 0002:00000a38       ??_C@_0P@BIEBOGNE@SetObjectField@ 10022a38     ObjectReferenceImpl.obj
 0002:00000a48       ??_C@_0N@IMJNOBAL@SetByteField@ 10022a48     ObjectReferenceImpl.obj
 0002:00000a58       ??_C@_0N@EOMGEBAI@SetCharField@ 10022a58     ObjectReferenceImpl.obj
 0002:00000a68       ??_C@_0O@DCKDPBBJ@SetFloatField@ 10022a68     ObjectReferenceImpl.obj
 0002:00000a78       ??_C@_0P@IAKDNKH@SetDoubleField@ 10022a78     ObjectReferenceImpl.obj
 0002:00000a88       ??_C@_0M@LPBODKIC@SetIntField@ 10022a88     ObjectReferenceImpl.obj
 0002:00000a94       ??_C@_0N@DHGKNGIJ@SetLongField@ 10022a94     ObjectReferenceImpl.obj
 0002:00000aa4       ??_C@_0O@BGNNAPCC@SetShortField@ 10022aa4     ObjectReferenceImpl.obj
 0002:00000ab4       ??_C@_0BA@CPPEGKHO@SetBooleanField@ 10022ab4     ObjectReferenceImpl.obj
 0002:00000ac4       ??_C@_0BG@LNEALOFM@GetObjectMonitorUsage@ 10022ac4     ObjectReferenceImpl.obj
 0002:00000adc       ??_C@_09OLJHFFGC@GetModule@ 10022adc     ReferenceTypeImpl.obj
 0002:00000ae8       ??_C@_0BA@CMEFDKBB@GetConstantPool@ 10022ae8     ReferenceTypeImpl.obj
 0002:00000af8       ??_C@_09GDNFOKKF@Signature@ 10022af8     ReferenceTypeImpl.obj
 0002:00000b04       ??_C@_09KLHEJKNK@Modifiers@ 10022b04     ReferenceTypeImpl.obj
 0002:00000b10       ??_C@_06BFNMHBP@Fields@    10022b10     ReferenceTypeImpl.obj
 0002:00000b18       ??_C@_07OALDEJCP@Methods@  10022b18     ReferenceTypeImpl.obj
 0002:00000b20       ??_C@_0L@CLDEMKOL@SourceFile@ 10022b20     ReferenceTypeImpl.obj
 0002:00000b2c       ??_C@_0M@GJNEEGFC@NestedTypes@ 10022b2c     ReferenceTypeImpl.obj
 0002:00000b38       ??_C@_0P@FHKLENLO@GetClassStatus@ 10022b38     ReferenceTypeImpl.obj
 0002:00000b48       ??_C@_0L@KBICGJBH@Interfaces@ 10022b48     ReferenceTypeImpl.obj
 0002:00000b54       ??_C@_0M@GFAKFENF@ClassObject@ 10022b54     ReferenceTypeImpl.obj
 0002:00000b60       ??_C@_0BF@JDJPNKHD@SourceDebugExtension@ 10022b60     ReferenceTypeImpl.obj
 0002:00000b78       ??_C@_0BF@IKGHKLIB@SignatureWithGeneric@ 10022b78     ReferenceTypeImpl.obj
 0002:00000b90       ??_C@_0BC@MCKDAAHH@FieldsWithGeneric@ 10022b90     ReferenceTypeImpl.obj
 0002:00000ba4       ??_C@_0BD@KPILANFP@MethodsWithGeneric@ 10022ba4     ReferenceTypeImpl.obj
 0002:00000bb8       ??_C@_09FGLEONFO@Instances@ 10022bb8     ReferenceTypeImpl.obj
 0002:00000bc4       ??_C@_0BA@GGCIPEOH@GetClassVersion@ 10022bc4     ReferenceTypeImpl.obj
 0002:00000bd4       ??_C@_0DO@MDHPDAFB@s?2src?2jdk?4jdwp?4agent?2share?2nati@ 10022bd4     ReferenceTypeImpl.obj
 0002:00000c14       ??_C@_0BC@GCIFGINE@GetClassModifiers@ 10022c14     ReferenceTypeImpl.obj
 0002:00000c28       ??_C@_0BA@FAMCEADF@GetClassMethods@ 10022c28     ReferenceTypeImpl.obj
 0002:00000c38       ??_C@_0BH@CNLIIJEM@GetClassVersionNumbers@ 10022c38     ReferenceTypeImpl.obj
 0002:00000c50       ??_C@_0P@KAMMPPGF@GetClassFields@ 10022c50     ReferenceTypeImpl.obj
 0002:00000c60       ??_C@_0BC@NBHLJMHF@GetSourceFileName@ 10022c60     ReferenceTypeImpl.obj
 0002:00000c74       ??_C@_0DA@BMDMENKL@s?2src?2jdk?4jdwp?4agent?2share?2nati@ 10022c74     SDE.obj
 0002:00000ca4       ??_C@_04MKAMAPIC@MISC@     10022ca4     SDE.obj
 0002:00000cac       ??_C@_0CC@FDGBKJLJ@SDE?5is?5re?9ordering?5the?5line?5tab@ 10022cac     SDE.obj
 0002:00000cd0       ??_C@_0DE@CBOCIEPK@bad?5SourceDebugExtension?5syntax@ 10022cd0     SDE.obj
 0002:00000d04       ??_C@_0P@BFDGOIGG@unexpected?5EOF@ 10022d04     SDE.obj
 0002:00000d14       ??_C@_0P@BPOMJGMN@SDE?5line?5table@ 10022d14     SDE.obj
 0002:00000d24       ??_C@_0P@NDLFOGMP@SDE?5file?5table@ 10022d24     SDE.obj
 0002:00000d34       ??_C@_0BC@JMMEOMHE@SDE?5stratum?5table@ 10022d34     SDE.obj
 0002:00000d48       ??_C@_0N@PPNMFI@expected?5?8?3?8@ 10022d48     SDE.obj
 0002:00000d58       ??_C@_04IEJOJGGI@Java@     10022d58     SDE.obj
 0002:00000d60       ??_C@_03EIMPEGPO@Aux@      10022d60     SDE.obj
 0002:00000d64       ??_C@_0N@BMNJHPCI@expected?5?8?$CK?8@ 10022d64     SDE.obj
 0002:00000d74       ??_C@_0N@KAHJKGJC@?$CKterminator?$CK@ 10022d74     SDE.obj
 0002:00000d84       ??_C@_0L@GFPHAPCK@ThisObject@ 10022d84     StackFrameImpl.obj
 0002:00000d90       ??_C@_09MMMKHAHA@PopFrames@ 10022d90     StackFrameImpl.obj
 0002:00000d9c       ??_C@_0L@JHEHPHFN@StackFrame@ 10022d9c     StackFrameImpl.obj
 0002:00000da8       ??_C@_0DL@OGCCGFPD@s?2src?2jdk?4jdwp?4agent?2share?2nati@ 10022da8     StackFrameImpl.obj
 0002:00000de4       ??_C@_0P@CCOLHCFB@GetLocalObject@ 10022de4     StackFrameImpl.obj
 0002:00000df4       ??_C@_0M@OFKPGHNH@GetLocalInt@ 10022df4     StackFrameImpl.obj
 0002:00000e00       ??_C@_0O@BDGHGOEC@GetLocalFloat@ 10022e00     StackFrameImpl.obj
 0002:00000e10       ??_C@_0P@LLJAGJLC@GetLocalDouble@ 10022e10     StackFrameImpl.obj
 0002:00000e20       ??_C@_0N@FDADNLMD@GetLocalLong@ 10022e20     StackFrameImpl.obj
 0002:00000e30       ??_C@_0P@OMPFIIHN@SetLocalObject@ 10022e30     StackFrameImpl.obj
 0002:00000e40       ??_C@_0M@OKLBLBFE@SetLocalInt@ 10022e40     StackFrameImpl.obj
 0002:00000e4c       ??_C@_0O@GMHJNNDF@SetLocalFloat@ 10022e4c     StackFrameImpl.obj
 0002:00000e5c       ??_C@_0P@HFIOJDJO@SetLocalDouble@ 10022e5c     StackFrameImpl.obj
 0002:00000e6c       ??_C@_0N@CHLNBHIP@SetLocalLong@ 10022e6c     StackFrameImpl.obj
 0002:00000e7c       ??_C@_0BB@ECEEEFHG@GetFrameLocation@ 10022e7c     StackFrameImpl.obj
 0002:00000e90       ??_C@_05LPIJGKJ@Value@     10022e90     StringReferenceImpl.obj
 0002:00000e98       ??_C@_0BA@LONLIKLM@StringReference@ 10022e98     StringReferenceImpl.obj
 0002:00000ea8       ??_C@_0EA@PLKIPJLM@s?2src?2jdk?4jdwp?4agent?2share?2nati@ 10022ea8     StringReferenceImpl.obj
 0002:00000ee8       ??_C@_04FABLJDN@Name@      10022ee8     ThreadGroupReferenceImpl.obj
 0002:00000ef0       ??_C@_06EBOPLIP@Parent@    10022ef0     ThreadGroupReferenceImpl.obj
 0002:00000ef8       ??_C@_08IEBJFPPC@Children@ 10022ef8     ThreadGroupReferenceImpl.obj
 0002:00000f04       ??_C@_0BF@HMNGNKAP@ThreadGroupReference@ 10022f04     ThreadGroupReferenceImpl.obj
 0002:00000f20       ??_C@_0EF@COMLBEIJ@s?2src?2jdk?4jdwp?4agent?2share?2nati@ 10022f20     ThreadGroupReferenceImpl.obj
 0002:00000f68       ??_C@_0BH@GAOLNFJO@GetThreadGroupChildren@ 10022f68     ThreadGroupReferenceImpl.obj
 0002:00000f80       ??_C@_0O@OMMMFPCB@GetFrameCount@ 10022f80     ThreadReferenceImpl.obj
 0002:00000f90       ??_C@_07MEGAPLCH@Suspend@  10022f90     ThreadReferenceImpl.obj
 0002:00000f98       ??_C@_06DEPGELNG@Resume@   10022f98     ThreadReferenceImpl.obj
 0002:00000fa0       ??_C@_06PGDKHFME@Status@   10022fa0     ThreadReferenceImpl.obj
 0002:00000fa8       ??_C@_0M@FJLPMLGA@ThreadGroup@ 10022fa8     ThreadReferenceImpl.obj
 0002:00000fb4       ??_C@_06CELCJONF@Frames@   10022fb4     ThreadReferenceImpl.obj
 0002:00000fbc       ??_C@_0O@CIBGJGLJ@OwnedMonitors@ 10022fbc     ThreadReferenceImpl.obj
 0002:00000fcc       ??_C@_0BI@LNCBLBIG@CurrentContendedMonitor@ 10022fcc     ThreadReferenceImpl.obj
 0002:00000fe4       ??_C@_04MOIHHPNJ@Stop@     10022fe4     ThreadReferenceImpl.obj
 0002:00000fec       ??_C@_09JNFEIGJE@Interrupt@ 10022fec     ThreadReferenceImpl.obj
 0002:00000ff8       ??_C@_0N@CJCCJPA@SuspendCount@ 10022ff8     ThreadReferenceImpl.obj
 0002:00001008       ??_C@_0BM@FMMKDMLC@OwnedMonitorsWithStackDepth@ 10023008     ThreadReferenceImpl.obj
 0002:00001024       ??_C@_0BB@OENGDAPG@ForceEarlyReturn@ 10023024     ThreadReferenceImpl.obj
 0002:00001038       ??_C@_0BA@DDHJAEOJ@ThreadReference@ 10023038     ThreadReferenceImpl.obj
 0002:00001048       ??_C@_0EA@KHLCDHFG@s?2src?2jdk?4jdwp?4agent?2share?2nati@ 10023048     ThreadReferenceImpl.obj
 0002:00001088       ??_C@_0O@OMCINHIO@GetThreadInfo@ 10023088     ThreadReferenceImpl.obj
 0002:00001098       ??_C@_0O@HJBPDPBL@GetStackTrace@ 10023098     ThreadReferenceImpl.obj
 0002:000010a8       ??_C@_0BE@CFHIFOK@GetOwnedMonitorInfo@ 100230a8     ThreadReferenceImpl.obj
 0002:000010bc       ??_C@_0BL@FKMDJLON@GetCurrentContendedMonitor@ 100230bc     ThreadReferenceImpl.obj
 0002:000010d8       ??_C@_0BO@KJEKJMBJ@GetOwnedMonitorStackDepthInfo@ 100230d8     ThreadReferenceImpl.obj
 0002:000010f8       ??_C@_0BH@OGPJNGCM@ForceEarlyReturnObject@ 100230f8     ThreadReferenceImpl.obj
 0002:00001110       ??_C@_0BF@GFOCGLCB@ForceEarlyReturnVoid@ 10023110     ThreadReferenceImpl.obj
 0002:00001128       ??_C@_0BE@OOLJADPL@ForceEarlyReturnInt@ 10023128     ThreadReferenceImpl.obj
 0002:0000113c       ??_C@_0BG@GAIJKLLL@ForceEarlyReturnFloat@ 1002313c     ThreadReferenceImpl.obj
 0002:00001154       ??_C@_0BH@HPICMNMP@ForceEarlyReturnDouble@ 10023154     ThreadReferenceImpl.obj
 0002:0000116c       ??_C@_0BF@GBNAKBEE@ForceEarlyReturnLong@ 1002316c     ThreadReferenceImpl.obj
 0002:00001184       ??_C@_0DE@JKJKNCJP@Java?5Debug?5Wire?5Protocol?5?$CIRefer@ 10023184     VirtualMachineImpl.obj
 0002:000011b8       ??_C@_0BA@DLNPNDDE@RedefineClasses@ 100231b8     VirtualMachineImpl.obj
 0002:000011c8       ??_C@_07NGFJPNPN@Version@  100231c8     VirtualMachineImpl.obj
 0002:000011d0       ??_C@_0BE@FBNAKJLP@ClassesForSignature@ 100231d0     VirtualMachineImpl.obj
 0002:000011e4       ??_C@_0L@FHGIJHIB@AllClasses@ 100231e4     VirtualMachineImpl.obj
 0002:000011f0       ??_C@_0O@OOLBCKEI@GetAllThreads@ 100231f0     VirtualMachineImpl.obj
 0002:00001200       ??_C@_0BF@PLHJIAHK@TopLevelThreadGroups@ 10023200     VirtualMachineImpl.obj
 0002:00001218       ??_C@_07HADINEKJ@Dispose@  10023218     VirtualMachineImpl.obj
 0002:00001220       ??_C@_07EMPPKEFJ@IDSizes@  10023220     VirtualMachineImpl.obj
 0002:00001228       ??_C@_06BJLINPHD@DoExit@   10023228     VirtualMachineImpl.obj
 0002:00001230       ??_C@_0N@DNBIJONA@CreateString@ 10023230     VirtualMachineImpl.obj
 0002:00001240       ??_C@_0N@FNJCOOAL@Capabilities@ 10023240     VirtualMachineImpl.obj
 0002:00001250       ??_C@_0L@KKBJMNEN@ClassPaths@ 10023250     VirtualMachineImpl.obj
 0002:0000125c       ??_C@_0P@MLKCHAIH@DisposeObjects@ 1002325c     VirtualMachineImpl.obj
 0002:0000126c       ??_C@_0L@CAGABDAD@HoldEvents@ 1002326c     VirtualMachineImpl.obj
 0002:00001278       ??_C@_0O@IOKPODIB@ReleaseEvents@ 10023278     VirtualMachineImpl.obj
 0002:00001288       ??_C@_0BA@IHAAAKEC@CapabilitiesNew@ 10023288     VirtualMachineImpl.obj
 0002:00001298       ??_C@_0BC@JBKLKNCM@SetDefaultStratum@ 10023298     VirtualMachineImpl.obj
 0002:000012ac       ??_C@_0BG@HDJCDLB@AllClassesWithGeneric@ 100232ac     VirtualMachineImpl.obj
 0002:000012c4       ??_C@_0P@GBGAFJLK@InstanceCounts@ 100232c4     VirtualMachineImpl.obj
 0002:000012d4       ??_C@_0L@KEPNLMPE@AllModules@ 100232d4     VirtualMachineImpl.obj
 0002:000012e0       ??_C@_0P@PELBDMOO@VirtualMachine@ 100232e0     VirtualMachineImpl.obj
 0002:000012f0       ??_C@_09EEKGDCPH@?$DMunknown?$DO@ 100232f0     VirtualMachineImpl.obj
 0002:00001300       ??_C@_0EL@OEBGOINI@?$CFs?5version?5?$CFd?4?$CFd?6JVM?5Debug?5Inte@ 10023300     VirtualMachineImpl.obj
 0002:0000134c       ??_C@_0DP@KCADHKOO@s?2src?2jdk?4jdwp?4agent?2share?2nati@ 1002334c     VirtualMachineImpl.obj
 0002:0000138c       ??_C@_0O@OCFPKCI@GetAllModules@ 1002338c     VirtualMachineImpl.obj
 0002:0000139c       ??_C@_0BD@GPIPONPL@GetTopThreadGroups@ 1002339c     VirtualMachineImpl.obj
 0002:000013b0       ??_C@_09OOFGMMEJ@JNI_FALSE@ 100233b0     VirtualMachineImpl.obj
 0002:000013bc       ??_C@_0N@PHJGBMEP@NewStringUTF@ 100233bc     VirtualMachineImpl.obj
 0002:000013cc       ??_C@_01ICJEACDI@?$DL@     100233cc     VirtualMachineImpl.obj
 0002:000013d0       ??_C@_0DH@GANKBOKD@s?2src?2jdk?4jdwp?4agent?2share?2nati@ 100233d0     classTrack.obj
 0002:00001408       ??_C@_06JAJCHHBC@GetTag@   10023408     classTrack.obj
 0002:00001410       ??_C@_0CI@IMNMNLEM@Unable?5to?5GetTag?5with?5class?5tra@ 10023410     classTrack.obj
 0002:00001438       ??_C@_0BC@PDKPGMNF@tag?5?$DN?$DN?5NOT_TAGGED@ 10023438     classTrack.obj
 0002:0000144c       ??_C@_09CMIIOJHF@signature@ 1002344c     classTrack.obj
 0002:00001458       ??_C@_06DADMPMP@SetTag@    10023458     classTrack.obj
 0002:00001460       ??_C@_0BA@GDHIKEAF@AddCapabilities@ 10023460     classTrack.obj
 0002:00001470       ??_C@_0BC@GAGPFDAP@SetEventCallbacks@ 10023470     classTrack.obj
 0002:00001484       ??_C@_0BJ@MAECPKFO@SetEventNotificationMode@ 10023484     classTrack.obj
 0002:000014a0       ??_C@_0BH@CJDMHCL@Deleted?5class?5tag?5lock@ 100234a0     classTrack.obj
 0002:000014b8       ??_C@_0CJ@MPKHDCCL@Failed?5to?5allocate?5tag?9tracking@ 100234b8     classTrack.obj
 0002:000014e4       ??_C@_0CE@GIKHACIF@Unable?5to?5setup?5ObjectFree?5trac@ 100234e4     classTrack.obj
 0002:00001508       ??_C@_0BF@GLPPHCDA@loaded?5classes?5array@ 10023508     classTrack.obj
 0002:00001520       ??_C@_0DG@IIIEKKMO@s?2src?2jdk?4jdwp?4agent?2share?2nati@ 10023520     commonRef.obj
 0002:00001558       ??_C@_0N@IAAOLNMM@NewGlobalRef@ 10023558     commonRef.obj
 0002:00001568       ??_C@_0BB@DFCJOKMO@NewWeakGlobalRef@ 10023568     commonRef.obj
 0002:0000157c       ??_C@_0BA@HLIPMHMF@DeleteGlobalRef@ 1002357c     commonRef.obj
 0002:0000158c       ??_C@_0BE@BJLAMKFM@DeleteWeakGlobalRef@ 1002358c     commonRef.obj
 0002:000015a0       ??_C@_0BB@EBIINFKL@Freeing?5?$CFd?5?$CI?$CFx?$CJ?6@ 100235a0     commonRef.obj
 0002:000015b4       ??_C@_0BC@GLNEFKOL@RefNode?5count?5?$DM?50@ 100235b4     commonRef.obj
 0002:000015c8       ??_C@_0BN@ODBCKJDJ@JDWP?5Reference?5Table?5Monitor@ 100235c8     commonRef.obj
 0002:000015e8       ??_C@_0M@GAIIKJOJ@NewLocalRef@ 100235e8     commonRef.obj
 0002:000015f4       ??_C@_0P@DFLOMFLG@DeleteLocalRef@ 100235f4     commonRef.obj
 0002:00001604       ??_C@_0DK@LLCGDOIF@s?2src?2jdk?4jdwp?4agent?2share?2nati@ 10023604     debugDispatch.obj
 0002:00001640       ??_C@_0BC@DMLDOBBC@command?5set?5array@ 10023640     debugDispatch.obj
 0002:00001654       ??_C@_0BF@OACBGPIG@?$DMInvalid?5CommandSet?$DO@ 10023654     debugDispatch.obj
 0002:0000166c       ??_C@_0BB@LBJDPCHC@?$DMUnkown?5Command?$DO@ 1002366c     debugDispatch.obj
 0002:00001680       ??_C@_0BC@KIDCJOPK@?$DMInvalid?5Command?$DO@ 10023680     debugDispatch.obj
 0002:00001694       ??_C@_0DG@GNAHAJEF@s?2src?2jdk?4jdwp?4agent?2share?2nati@ 10023694     debugInit.obj
 0002:000016cc       ??_C@_0DI@HJHBDLDN@JDWP?5unable?5to?5configure?5initia@ 100236cc     debugInit.obj
 0002:00001708       ??_C@_0FO@EFFMOFEA@Cannot?5load?5this?5JVM?5TI?5agent?5t@ 10023708     debugInit.obj
 0002:00001768       ??_C@_0BN@FIGCDEN@JDWP?5unable?5to?5load?0?5VM?5died@ 10023768     debugInit.obj
 0002:00001788       ??_C@_03HPEPLPA@JVM@       10023788     debugInit.obj
 0002:0000178c       ??_C@_06CALCCDMF@GetEnv@   1002378c     debugInit.obj
 0002:00001798       ??_C@_0HB@JPGJENBG@JDWP?5unable?5to?5access?5JVMTI?5Ver@ 10023798     debugInit.obj
 0002:00001810       ??_C@_0GO@CPKDKNDM@This?5jdwp?5native?5library?5will?5n@ 10023810     debugInit.obj
 0002:00001880       ??_C@_0L@GCOJPMGE@Onload?3?5?$CFs@ 10023880     debugInit.obj
 0002:0000188c       ??_C@_0BJ@DAFNBFMC@GetPotentialCapabilities@ 1002388c     debugInit.obj
 0002:000018a8       ??_C@_0DI@HGBENBDB@JDWP?5unable?5to?5get?5potential?5JV@ 100238a8     debugInit.obj
 0002:000018e0       ??_C@_0DB@KIBJMMBD@JDWP?5unable?5to?5get?5necessary?5JV@ 100238e0     debugInit.obj
 0002:00001914       ??_C@_0DB@FLBLFKJC@JDWP?5unable?5to?5set?5JVMTI?5event?5@ 10023914     debugInit.obj
 0002:00001948       ??_C@_0N@NKKDPPME@OnLoad?3?5DONE@ 10023948     debugInit.obj
 0002:00001958       ??_C@_02LACNDIPD@CB@       10023958     debugInit.obj
 0002:0000195c       ??_C@_0O@DLFFEAD@cbEarlyVMInit@ 1002395c     debugInit.obj
 0002:0000196c       ??_C@_0BI@BCONGKCA@VM?5dead?5at?5VM_INIT?5time@ 1002396c     debugInit.obj
 0002:00001984       ??_C@_0BC@IFIKOKIP@END?5cbEarlyVMInit@ 10023984     debugInit.obj
 0002:00001998       ??_C@_0BD@IBLDMNIE@DisposeEnvironment@ 10023998     debugInit.obj
 0002:000019ac       ??_C@_0DE@BOJEJHME@JDWP?5unable?5to?5dispose?5of?5JVMTI@ 100239ac     debugInit.obj
 0002:000019e0       ??_C@_0P@DKNEAPGB@cbEarlyVMDeath@ 100239e0     debugInit.obj
 0002:000019f0       ??_C@_0BH@MJOFBADO@VM?5died?5more?5than?5once@ 100239f0     debugInit.obj
 0002:00001a08       ??_C@_0BD@NOFMPPNE@END?5cbEarlyVMDeath@ 10023a08     debugInit.obj
 0002:00001a1c       ??_C@_0BM@IEEFFE@cbEarlyException?3?5thread?$DN?$CFp@ 10023a1c     debugInit.obj
 0002:00001a38       ??_C@_0CD@LICFEBIC@VM?5dead?5at?5initial?5Exception?5ev@ 10023a38     debugInit.obj
 0002:00001a5c       ??_C@_0BK@LELFCHPE@VM?5is?5not?5initialized?5yet@ 10023a5c     debugInit.obj
 0002:00001a78       ??_C@_0CD@IFKJAMDD@Initializing?5on?5uncaught?5except@ 10023a78     debugInit.obj
 0002:00001a9c       ??_C@_0DE@NBANCLO@Checking?5specific?5exception?3?5lo@ 10023a9c     debugInit.obj
 0002:00001ad0       ??_C@_0CD@DGOBNBPB@Initializing?5on?5specific?5except@ 10023ad0     debugInit.obj
 0002:00001af4       ??_C@_0CP@DAAMLOKM@No?5initialization?0?5didn?8t?5find?5@ 10023af4     debugInit.obj
 0002:00001b24       ??_C@_05JCKDCDAK@Throw@    10023b24     debugInit.obj
 0002:00001b2c       ??_C@_0BF@FLBJJJJM@END?5cbEarlyException@ 10023b2c     debugInit.obj
 0002:00001b44       ??_C@_0BF@KCLMNAFK@Begin?5startTransport@ 10023b44     debugInit.obj
 0002:00001b5c       ??_C@_0CP@GLCNJPPL@JDWP?5Transport?5?$CFs?5failed?5to?5ini@ 10023b5c     debugInit.obj
 0002:00001b8c       ??_C@_0BD@KMCJBFOI@End?5startTransport@ 10023b8c     debugInit.obj
 0002:00001ba0       ??_C@_0BP@HFGABHKC@signal?5initialization?5complete@ 10023ba0     debugInit.obj
 0002:00001bc0       ??_C@_0P@CPJAJOGP@UNKNOWN?5REASON@ 10023bc0     debugInit.obj
 0002:00001bd0       ??_C@_0BL@EEDFKGOH@JDWP?5?$CFs?0?5jvmtiError?$DN?$CFs?$CI?$CFd?$CJ@ 10023bd0     debugInit.obj
 0002:00001bec       ??_C@_07CBPKFJFN@JDWP?5?$CFs@ 10023bec     debugInit.obj
 0002:00001bf4       ??_C@_0CG@MHFIMNKE@Can?8t?5call?5JNI?5FatalError?$CINULL?0@ 10023bf4     debugInit.obj
 0002:00001c1c       ??_C@_0O@GBAEPAJL@ERROR?3?5JDWP?3?5@ 10023c1c     debugInit.obj
 0002:00001c2c       ??_C@_0BD@BEMOICGG@Begin?5initialize?$CI?$CJ@ 10023c2c     debugInit.obj
 0002:00001c40       ??_C@_0BN@NHJNNMLF@VM?5dead?5at?5initialize?$CI?$CJ?5time@ 10023c40     debugInit.obj
 0002:00001c60       ??_C@_0CL@FOADKMNE@unable?5to?5disable?5JVMTI?5event?5n@ 10023c60     debugInit.obj
 0002:00001c8c       ??_C@_0CA@LEEFBLBH@unable?5to?5clear?5JVMTI?5callbacks@ 10023c8c     debugInit.obj
 0002:00001cac       ??_C@_0BM@GGAMJPIA@JDWP?5Initialization?5Monitor@ 10023cac     debugInit.obj
 0002:00001cc8       ??_C@_0BK@MDFDHGIG@No?5transports?5initialized@ 10023cc8     debugInit.obj
 0002:00001ce4       ??_C@_0BM@IHKNNPNA@triggering_ei?5?$DN?$DN?5EI_VM_INIT@ 10023ce4     debugInit.obj
 0002:00001d00       ??_C@_0BM@MLOKHCJB@triggering_ei?5?$CB?$DN?5EI_VM_INIT@ 10023d00     debugInit.obj
 0002:00001d1c       ??_C@_0CG@FBKKPEEO@VM?5dead?5before?5initialize?$CI?$CJ?5com@ 10023d1c     debugInit.obj
 0002:00001d44       ??_C@_0BB@FNMNNOIE@End?5initialize?$CI?$CJ@ 10023d44     debugInit.obj
 0002:00001d58       ??_C@_0BM@DDGJDKIN@debugInit_reset?$CI?$CJ?5beginning@ 10023d58     debugInit.obj
 0002:00001d74       ??_C@_0BN@ICEPLJN@debugInit_reset?$CI?$CJ?5completed?4@ 10023d74     debugInit.obj
 0002:00001d98       ??_C@_0EHD@NPDAGEJI@?5?5?5?5?5?5?5?5?5?5?5?5?5?5?5Java?5Debugger?5JD@ 10023d98     debugInit.obj
 0002:00002210       ??_C@_0CEF@LOIFLEGE@Obsolete?5Options?6?9?9?9?9?9?9?9?9?9?9?9?9?9?9@ 10024210     debugInit.obj
 0002:00002458       ??_C@_0GE@PNCPNOJL@JDWP?5Non?9server?5transport?5?$CFs?5mu@ 10024458     debugInit.obj
 0002:000024bc       ??_C@_01IHBHIGKO@?0@       100244bc     debugInit.obj
 0002:000024c0       ??_C@_01EANLCPLP@y@        100244c0     debugInit.obj
 0002:000024c4       ??_C@_01EFFIKLCJ@n@        100244c4     debugInit.obj
 0002:000024c8       ??_C@_04PCJFHION@help@     100244c8     debugInit.obj
 0002:000024d0       ??_C@_0BD@BLCBAGAJ@_JAVA_JDWP_OPTIONS@ 100244d0     debugInit.obj
 0002:000024e4       ??_C@_07FOPBDDAL@options@  100244e4     debugInit.obj
 0002:000024ec       ??_C@_0L@PNFKLIOM@transports@ 100244ec     debugInit.obj
 0002:000024f8       ??_C@_09PBENLGJM@transport@ 100244f8     debugInit.obj
 0002:00002504       ??_C@_07LHEPONKL@address@  10024504     debugInit.obj
 0002:0000250c       ??_C@_0CE@KJBCDAKG@address?5specified?5without?5trans@ 1002450c     debugInit.obj
 0002:00002530       ??_C@_05IDFCDDHI@allow@    10024530     debugInit.obj
 0002:00002538       ??_C@_0CC@DKFOJBDD@allow?5specified?5without?5transpo@ 10024538     debugInit.obj
 0002:0000255c       ??_C@_07DDHNKDGP@timeout@  1002455c     debugInit.obj
 0002:00002564       ??_C@_0CE@KCGGPGKE@timeout?5specified?5without?5trans@ 10024564     debugInit.obj
 0002:00002588       ??_C@_06OAFDKBLG@launch@   10024588     debugInit.obj
 0002:00002590       ??_C@_07JDKNNNFJ@onthrow@  10024590     debugInit.obj
 0002:00002598       ??_C@_06GMEIIFFN@assert@   10024598     debugInit.obj
 0002:000025a0       ??_C@_05FAMCFOJB@fatal@    100245a0     debugInit.obj
 0002:000025a8       ??_C@_05PDJBBECF@pause@    100245a8     debugInit.obj
 0002:000025b0       ??_C@_08JHOBLGK@coredump@  100245b0     debugInit.obj
 0002:000025bc       ??_C@_09NDIDIJNG@errorexit@ 100245bc     debugInit.obj
 0002:000025c8       ??_C@_09KOPDMKB@exitpause@ 100245c8     debugInit.obj
 0002:000025d4       ??_C@_0CO@FJOJNBJC@The?5exitpause?5option?5removed?0?5u@ 100245d4     debugInit.obj
 0002:00002604       ??_C@_08KLNFLELA@precrash@ 10024604     debugInit.obj
 0002:00002610       ??_C@_0CN@FJOGMEJD@The?5precrash?5option?5removed?0?5us@ 10024610     debugInit.obj
 0002:00002640       ??_C@_07HMINABEO@logfile@  10024640     debugInit.obj
 0002:00002648       ??_C@_08KMAEEIGA@logflags@ 10024648     debugInit.obj
 0002:00002654       ??_C@_0L@NDPADBNN@debugflags@ 10024654     debugInit.obj
 0002:00002660       ??_C@_07DNBGJJHB@suspend@  10024660     debugInit.obj
 0002:00002668       ??_C@_06HJHJCKIO@server@   10024668     debugInit.obj
 0002:00002670       ??_C@_06OLFOGHEN@strict@   10024670     debugInit.obj
 0002:00002678       ??_C@_05PMBAOCDH@quiet@    10024678     debugInit.obj
 0002:00002680       ??_C@_0L@EINCANF@onuncaught@ 10024680     debugInit.obj
 0002:0000268c       ??_C@_05HEPNBBMF@mutf8@    1002468c     debugInit.obj
 0002:00002694       ??_C@_08GEPKFJKM@stdalloc@ 10024694     debugInit.obj
 0002:000026a0       ??_C@_06JGBMLDHG@onjcmd@   100246a0     debugInit.obj
 0002:000026a8       ??_C@_0BH@HHOMGJCA@no?5transport?5specified@ 100246a8     debugInit.obj
 0002:000026c0       ??_C@_0DG@LFMJLIEN@multiple?5transports?5are?5not?5sup@ 100246c0     debugInit.obj
 0002:000026f8       ??_C@_0EJ@JJILEHOC@Specify?5launch?$DN?$DMcommand?5line?$DO?5w@ 100246f8     debugInit.obj
 0002:00002744       ??_C@_0CM@MLAKJKDP@Cannot?5combine?5onjcmd?5and?5launc@ 10024744     debugInit.obj
 0002:00002770       ??_C@_0CC@CBAOLJED@Can?5only?5use?5onjcmd?5with?5server@ 10024770     debugInit.obj
 0002:00002794       ??_C@_0P@KGDIDJKL@?9agentlib?3jdwp@ 10024794     debugInit.obj
 0002:000027a4       ??_C@_0CA@PBEIFGCB@JDWP?5option?5syntax?5error?3?5?$CFs?$DN?$CFs@ 100247a4     debugInit.obj
 0002:000027c4       ??_C@_0P@HJPPKHBO@JDWP?5?$CFs?3?5?$CFs?$DN?$CFs@ 100247c4     debugInit.obj
 0002:000027d4       ??_C@_0P@PJFAGLMH@invalid?5option@ 100247d4     debugInit.obj
 0002:000027e4       ??_C@_0BO@EGHMLMKO@Exiting?5with?5error?5?$CFs?$CI?$CFd?$CJ?3?5?$CFs@ 100247e4     debugInit.obj
 0002:00002804       ??_C@_0CK@CLPEKKDE@Dumping?5core?5as?5requested?5by?5co@ 10024804     debugInit.obj
 0002:00002830       ??_C@_0CG@EBFFHEOK@Not?5yet?5initialized?4?5Try?5again?5@ 10024830     debugInit.obj
 0002:00002858       ??_C@_0FF@NOEEBMNP@Starting?5debugging?5via?5jcmd?5was@ 10024858     debugInit.obj
 0002:000028b0       ??_C@_0BD@KBEAEDMA@JDWP?5VM_DEATH?5Lock@ 100248b0     debugLoop.obj
 0002:000028c4       ??_C@_0BI@KEHBCJBK@JDWP?5Command?5Queue?5Lock@ 100248c4     debugLoop.obj
 0002:000028dc       ??_C@_0BE@OJJPFMMB@JDWP?5Command?5Reader@ 100248dc     debugLoop.obj
 0002:000028f0       ??_C@_0DG@PEEBJHLA@s?2src?2jdk?4jdwp?4agent?2share?2nati@ 100248f0     debugLoop.obj
 0002:00002928       ??_C@_0CD@BCFANGIM@Command?5set?5?$CFs?$CI?$CFd?$CJ?0?5command?5?$CFs?$CI@ 10024928     debugLoop.obj
 0002:0000294c       ??_C@_0BE@LPIOKOFH@Begin?5reader?5thread@ 1002494c     debugLoop.obj
 0002:00002960       ??_C@_0FI@EMFENIBI@Received?5jdwpPacket?5with?5flags?5@ 10024960     debugLoop.obj
 0002:000029b8       ??_C@_0BC@PBMDCOFP@End?5reader?5thread@ 100249b8     debugLoop.obj
 0002:000029cc       ??_C@_0M@FFFEEGHJ@packet?5list@ 100249cc     debugLoop.obj
 0002:000029d8       ??_C@_06DIJPEION@?$CFs?$CFs?$CFs@ 100249d8     error_messages.obj
 0002:000029e0       ??_C@_07JHDPBCI@ERROR?3?5@ 100249e0     error_messages.obj
 0002:000029e8       ??_C@_0DL@OBDMDFEC@s?2src?2jdk?4jdwp?4agent?2share?2nati@ 100249e8     error_messages.obj
 0002:00002a24       ??_C@_0BN@HFAPOECE@Requested?5errorexit?$DNy?5exit?$CI?$CJ@ 10024a24     error_messages.obj
 0002:00002a44       ??_C@_0BN@BNMAOKIE@ASSERT?5FAILED?3?5?$CFs?5?3?5?$CFd?5?9?5?$CFs?6@ 10024a44     error_messages.obj
 0002:00002a64       ??_C@_0N@BMIGOGFN@?$CFs?5?3?5?$CFd?5?9?5?$CFs@ 10024a64     error_messages.obj
 0002:00002a74       ??_C@_0BA@HJKPOGGF@ASSERT?5FAILED?3?5@ 10024a74     error_messages.obj
 0002:00002a84       ??_C@_0BB@NAGLCMLI@Assertion?5Failed@ 10024a84     error_messages.obj
 0002:00002a98       ??_C@_0BB@JCNMKLLK@JVMTI_ERROR_NONE@ 10024a98     error_messages.obj
 0002:00002aac       ??_C@_0BL@LDIMKLPH@JVMTI_ERROR_INVALID_THREAD@ 10024aac     error_messages.obj
 0002:00002ac8       ??_C@_0CB@PJFPAIKJ@JVMTI_ERROR_INVALID_THREAD_GROU@ 10024ac8     error_messages.obj
 0002:00002aec       ??_C@_0BN@LLMKHMNF@JVMTI_ERROR_INVALID_PRIORITY@ 10024aec     error_messages.obj
 0002:00002b0c       ??_C@_0CB@MBOFKAGB@JVMTI_ERROR_THREAD_NOT_SUSPENDE@ 10024b0c     error_messages.obj
 0002:00002b30       ??_C@_0BN@FABOLPBI@JVMTI_ERROR_THREAD_SUSPENDED@ 10024b30     error_messages.obj
 0002:00002b50       ??_C@_0BN@FDGNOBJM@JVMTI_ERROR_THREAD_NOT_ALIVE@ 10024b50     error_messages.obj
 0002:00002b70       ??_C@_0BL@GOBIFKNJ@JVMTI_ERROR_INVALID_OBJECT@ 10024b70     error_messages.obj
 0002:00002b8c       ??_C@_0BK@FCMAJPPC@JVMTI_ERROR_INVALID_CLASS@ 10024b8c     error_messages.obj
 0002:00002ba8       ??_C@_0BP@IKLLBKEB@JVMTI_ERROR_CLASS_NOT_PREPARED@ 10024ba8     error_messages.obj
 0002:00002bc8       ??_C@_0BN@KLPPLKG@JVMTI_ERROR_INVALID_METHODID@ 10024bc8     error_messages.obj
 0002:00002be8       ??_C@_0BN@BCEKOKND@JVMTI_ERROR_INVALID_LOCATION@ 10024be8     error_messages.obj
 0002:00002c08       ??_C@_0BM@DFDGPME@JVMTI_ERROR_INVALID_FIELDID@ 10024c08     error_messages.obj
 0002:00002c24       ??_C@_0BL@NELIEPEC@JVMTI_ERROR_NO_MORE_FRAMES@ 10024c24     error_messages.obj
 0002:00002c40       ??_C@_0BJ@BDBECFDM@JVMTI_ERROR_OPAQUE_FRAME@ 10024c40     error_messages.obj
 0002:00002c5c       ??_C@_0BK@MIIFNLOB@JVMTI_ERROR_TYPE_MISMATCH@ 10024c5c     error_messages.obj
 0002:00002c78       ??_C@_0BJ@HPCAOILC@JVMTI_ERROR_INVALID_SLOT@ 10024c78     error_messages.obj
 0002:00002c94       ??_C@_0BG@CHILOPNI@JVMTI_ERROR_DUPLICATE@ 10024c94     error_messages.obj
 0002:00002cac       ??_C@_0BG@DIEMLHKM@JVMTI_ERROR_NOT_FOUND@ 10024cac     error_messages.obj
 0002:00002cc4       ??_C@_0BM@NHMCKHOB@JVMTI_ERROR_INVALID_MONITOR@ 10024cc4     error_messages.obj
 0002:00002ce0       ??_C@_0BO@PPEDAJGL@JVMTI_ERROR_NOT_MONITOR_OWNER@ 10024ce0     error_messages.obj
 0002:00002d00       ??_C@_0BG@FCAIPEID@JVMTI_ERROR_INTERRUPT@ 10024d00     error_messages.obj
 0002:00002d18       ??_C@_0CB@EGDBNKOI@JVMTI_ERROR_INVALID_CLASS_FORMA@ 10024d18     error_messages.obj
 0002:00002d3c       ??_C@_0CG@DGKOGIAL@JVMTI_ERROR_CIRCULAR_CLASS_DEFI@ 10024d3c     error_messages.obj
 0002:00002d64       ??_C@_0BP@ICEALPKC@JVMTI_ERROR_FAILS_VERIFICATION@ 10024d64     error_messages.obj
 0002:00002d84       ??_C@_0DC@JDACLMIO@JVMTI_ERROR_UNSUPPORTED_REDEFIN@ 10024d84     error_messages.obj
 0002:00002db8       ??_C@_0DE@GKDKNOMJ@JVMTI_ERROR_UNSUPPORTED_REDEFIN@ 10024db8     error_messages.obj
 0002:00002dec       ??_C@_0BO@LAFKIOG@JVMTI_ERROR_INVALID_TYPESTATE@ 10024dec     error_messages.obj
 0002:00002e0c       ??_C@_0DH@INDGCLLB@JVMTI_ERROR_UNSUPPORTED_REDEFIN@ 10024e0c     error_messages.obj
 0002:00002e44       ??_C@_0DE@NHEOMMGI@JVMTI_ERROR_UNSUPPORTED_REDEFIN@ 10024e44     error_messages.obj
 0002:00002e78       ??_C@_0CA@EKPNJOEP@JVMTI_ERROR_UNSUPPORTED_VERSION@ 10024e78     error_messages.obj
 0002:00002e98       ??_C@_0BN@OFFMAHHL@JVMTI_ERROR_NAMES_DONT_MATCH@ 10024e98     error_messages.obj
 0002:00002eb8       ??_C@_0DN@HHBBLAKE@JVMTI_ERROR_UNSUPPORTED_REDEFIN@ 10024eb8     error_messages.obj
 0002:00002ef8       ??_C@_0DO@HMBGBGNA@JVMTI_ERROR_UNSUPPORTED_REDEFIN@ 10024ef8     error_messages.obj
 0002:00002f38       ??_C@_0BK@CANILEHF@JVMTI_ERROR_NOT_AVAILABLE@ 10024f38     error_messages.obj
 0002:00002f54       ??_C@_0CE@INJKMEFK@JVMTI_ERROR_MUST_POSSESS_CAPABI@ 10024f54     error_messages.obj
 0002:00002f78       ??_C@_0BJ@LBFPFPDM@JVMTI_ERROR_NULL_POINTER@ 10024f78     error_messages.obj
 0002:00002f94       ??_C@_0BP@CHJPNNEM@JVMTI_ERROR_ABSENT_INFORMATION@ 10024f94     error_messages.obj
 0002:00002fb4       ??_C@_0BP@OMFMNLC@JVMTI_ERROR_INVALID_EVENT_TYPE@ 10024fb4     error_messages.obj
 0002:00002fd4       ??_C@_0BN@BIBNPHHO@JVMTI_ERROR_ILLEGAL_ARGUMENT@ 10024fd4     error_messages.obj
 0002:00002ff4       ??_C@_0BK@PMKCFHAE@JVMTI_ERROR_OUT_OF_MEMORY@ 10024ff4     error_messages.obj
 0002:00003010       ??_C@_0BK@NNJBDMNB@JVMTI_ERROR_ACCESS_DENIED@ 10025010     error_messages.obj
 0002:0000302c       ??_C@_0BI@GHECLMNC@JVMTI_ERROR_WRONG_PHASE@ 1002502c     error_messages.obj
 0002:00003044       ??_C@_0BF@OLIHJOII@JVMTI_ERROR_INTERNAL@ 10025044     error_messages.obj
 0002:0000305c       ??_C@_0BO@EOHGKJHI@JVMTI_ERROR_UNATTACHED_THREAD@ 1002505c     error_messages.obj
 0002:0000307c       ??_C@_0CA@LKHFDACL@JVMTI_ERROR_INVALID_ENVIRONMENT@ 1002507c     error_messages.obj
 0002:0000309c       ??_C@_0BF@KCDLAD@AGENT_ERROR_INTERNAL@ 1002509c     error_messages.obj
 0002:000030b4       ??_C@_0BE@KFGADCIM@AGENT_ERROR_VM_DEAD@ 100250b4     error_messages.obj
 0002:000030c8       ??_C@_0BH@IOOMLCPK@AGENT_ERROR_NO_JNI_ENV@ 100250c8     error_messages.obj
 0002:000030e0       ??_C@_0BK@OHNBOEAB@AGENT_ERROR_JNI_EXCEPTION@ 100250e0     error_messages.obj
 0002:000030fc       ??_C@_0BL@HHHLGBCJ@AGENT_ERROR_JVMTI_INTERNAL@ 100250fc     error_messages.obj
 0002:00003118       ??_C@_0BK@DOAJMAC@AGENT_ERROR_JDWP_INTERNAL@ 10025118     error_messages.obj
 0002:00003134       ??_C@_0BO@HMIKBJDH@AGENT_ERROR_NOT_CURRENT_FRAME@ 10025134     error_messages.obj
 0002:00003154       ??_C@_0BK@MDCNJBJM@AGENT_ERROR_OUT_OF_MEMORY@ 10025154     error_messages.obj
 0002:00003170       ??_C@_0BI@OCBNFCC@AGENT_ERROR_INVALID_TAG@ 10025170     error_messages.obj
 0002:00003188       ??_C@_0BN@PEANMDOB@AGENT_ERROR_ALREADY_INVOKING@ 10025188     error_messages.obj
 0002:000031a8       ??_C@_0BK@HKJFNPFH@AGENT_ERROR_INVALID_INDEX@ 100251a8     error_messages.obj
 0002:000031c4       ??_C@_0BL@BMIJGCKP@AGENT_ERROR_INVALID_LENGTH@ 100251c4     error_messages.obj
 0002:000031e0       ??_C@_0BL@JGHDGIGP@AGENT_ERROR_INVALID_STRING@ 100251e0     error_messages.obj
 0002:000031fc       ??_C@_0CB@GJDCCCGC@AGENT_ERROR_INVALID_CLASS_LOADE@ 100251fc     error_messages.obj
 0002:00003220       ??_C@_0BK@FILGLGGH@AGENT_ERROR_INVALID_ARRAY@ 10025220     error_messages.obj
 0002:0000323c       ??_C@_0BL@FDPHKKDB@AGENT_ERROR_TRANSPORT_LOAD@ 1002523c     error_messages.obj
 0002:00003258       ??_C@_0BL@GHHKABMN@AGENT_ERROR_TRANSPORT_INIT@ 10025258     error_messages.obj
 0002:00003274       ??_C@_0BK@JFFMLFLM@AGENT_ERROR_NATIVE_METHOD@ 10025274     error_messages.obj
 0002:00003290       ??_C@_0BK@KOCLEFJG@AGENT_ERROR_INVALID_COUNT@ 10025290     error_messages.obj
 0002:000032ac       ??_C@_0BM@LDFIPDCL@AGENT_ERROR_INVALID_FRAMEID@ 100252ac     error_messages.obj
 0002:000032c8       ??_C@_0BJ@ILJPBKJK@AGENT_ERROR_NULL_POINTER@ 100252c8     error_messages.obj
 0002:000032e4       ??_C@_0BN@LLKPAHA@AGENT_ERROR_ILLEGAL_ARGUMENT@ 100252e4     error_messages.obj
 0002:00003304       ??_C@_0BL@ENGHDPEH@AGENT_ERROR_INVALID_THREAD@ 10025304     error_messages.obj
 0002:00003320       ??_C@_0BP@OCCGGDI@AGENT_ERROR_INVALID_EVENT_TYPE@ 10025320     error_messages.obj
 0002:00003340       ??_C@_0BL@JAPDMOGJ@AGENT_ERROR_INVALID_OBJECT@ 10025340     error_messages.obj
 0002:0000335c       ??_C@_0BL@CKFDNLPC@AGENT_ERROR_NO_MORE_FRAMES@ 1002535c     error_messages.obj
 0002:00003378       ??_C@_0O@LFPPCNKG@ERROR_unknown@ 10025378     error_messages.obj
 0002:00003388       ??_C@_0P@KOMKCNJP@EI_SINGLE_STEP@ 10025388     error_messages.obj
 0002:00003398       ??_C@_0O@PLAPKDL@EI_BREAKPOINT@ 10025398     error_messages.obj
 0002:000033a8       ??_C@_0N@PGOIKMFF@EI_FRAME_POP@ 100253a8     error_messages.obj
 0002:000033b8       ??_C@_0N@CEKAFBCB@EI_EXCEPTION@ 100253b8     error_messages.obj
 0002:000033c8       ??_C@_0BA@EJAFLEFO@EI_THREAD_START@ 100253c8     error_messages.obj
 0002:000033d8       ??_C@_0O@GJFHOBHI@EI_THREAD_END@ 100253d8     error_messages.obj
 0002:000033e8       ??_C@_0BB@FOCFHABH@EI_CLASS_PREPARE@ 100253e8     error_messages.obj
 0002:000033fc       ??_C@_0O@BCBJODOG@EI_CLASS_LOAD@ 100253fc     error_messages.obj
 0002:0000340c       ??_C@_0BA@DBHDLMCN@EI_FIELD_ACCESS@ 1002540c     error_messages.obj
 0002:0000341c       ??_C@_0BG@BKOJDIGF@EI_FIELD_MODIFICATION@ 1002541c     error_messages.obj
 0002:00003434       ??_C@_0BD@IMHNDJNF@EI_EXCEPTION_CATCH@ 10025434     error_messages.obj
 0002:00003448       ??_C@_0BA@BMAHDEKG@EI_METHOD_ENTRY@ 10025448     error_messages.obj
 0002:00003458       ??_C@_0P@EODELCOH@EI_METHOD_EXIT@ 10025458     error_messages.obj
 0002:00003468       ??_C@_0L@DINKDGIA@EI_VM_INIT@ 10025468     error_messages.obj
 0002:00003474       ??_C@_0M@NLNKJGDL@EI_VM_DEATH@ 10025474     error_messages.obj
 0002:00003480       ??_C@_0N@FJNDECKL@EI_GC_FINISH@ 10025480     error_messages.obj
 0002:00003490       ??_C@_0O@MBFGOMME@EVENT_unknown@ 10025490     error_messages.obj
 0002:000034a0       ??_C@_04OKGDLNCL@NONE@     100254a0     error_messages.obj
 0002:000034a8       ??_C@_0P@JCGOCJJM@INVALID_THREAD@ 100254a8     error_messages.obj
 0002:000034b8       ??_C@_0BF@BFLDLBKG@INVALID_THREAD_GROUP@ 100254b8     error_messages.obj
 0002:000034d0       ??_C@_0BB@DOHFANFH@INVALID_PRIORITY@ 100254d0     error_messages.obj
 0002:000034e4       ??_C@_0BF@CNAJBJGO@THREAD_NOT_SUSPENDED@ 100254e4     error_messages.obj
 0002:000034fc       ??_C@_0BB@NFKBMOJK@THREAD_SUSPENDED@ 100254fc     error_messages.obj
 0002:00003510       ??_C@_0P@EPPKNILC@INVALID_OBJECT@ 10025510     error_messages.obj
 0002:00003520       ??_C@_0O@ELGEBMG@INVALID_CLASS@ 10025520     error_messages.obj
 0002:00003530       ??_C@_0BD@KEAMCEJN@CLASS_NOT_PREPARED@ 10025530     error_messages.obj
 0002:00003544       ??_C@_0BB@IPAAIKCE@INVALID_METHODID@ 10025544     error_messages.obj
 0002:00003558       ??_C@_0BB@JHPFJLFB@INVALID_LOCATION@ 10025558     error_messages.obj
 0002:0000356c       ??_C@_0BA@NJBCDFJG@INVALID_FIELDID@ 1002556c     error_messages.obj
 0002:0000357c       ??_C@_0BA@KCIGPBGB@INVALID_FRAMEID@ 1002557c     error_messages.obj
 0002:0000358c       ??_C@_0P@PFFKMNCJ@NO_MORE_FRAMES@ 1002558c     error_messages.obj
 0002:0000359c       ??_C@_0N@NGAODCAJ@OPAQUE_FRAME@ 1002559c     error_messages.obj
 0002:000035ac       ??_C@_0BC@JIBCMOEK@NOT_CURRENT_FRAME@ 100255ac     error_messages.obj
 0002:000035c0       ??_C@_0O@JOPDAFNF@TYPE_MISMATCH@ 100255c0     error_messages.obj
 0002:000035d0       ??_C@_0N@LKDKPPIH@INVALID_SLOT@ 100255d0     error_messages.obj
 0002:000035e0       ??_C@_09JHHLKDOI@DUPLICATE@ 100255e0     error_messages.obj
 0002:000035ec       ??_C@_09IILMPLJM@NOT_FOUND@ 100255ec     error_messages.obj
 0002:000035f8       ??_C@_0BA@NIDPNLD@INVALID_MONITOR@ 100255f8     error_messages.obj
 0002:00003608       ??_C@_0BC@PMHAFEBG@NOT_MONITOR_OWNER@ 10025608     error_messages.obj
 0002:0000361c       ??_C@_09OCPILILD@INTERRUPT@ 1002561c     error_messages.obj
 0002:00003628       ??_C@_0BF@KKNNGDOH@INVALID_CLASS_FORMAT@ 10025628     error_messages.obj
 0002:00003640       ??_C@_0BK@IGLHGLOO@CIRCULAR_CLASS_DEFINITION@ 10025640     error_messages.obj
 0002:0000365c       ??_C@_0BD@KMPHIBHO@FAILS_VERIFICATION@ 1002565c     error_messages.obj
 0002:00003670       ??_C@_0BL@PPBPAAJH@ADD_METHOD_NOT_IMPLEMENTED@ 10025670     error_messages.obj
 0002:0000368c       ??_C@_0BO@EMGJAAKO@SCHEMA_CHANGE_NOT_IMPLEMENTED@ 1002568c     error_messages.obj
 0002:000036ac       ??_C@_0BC@IDGPFJL@INVALID_TYPESTATE@ 100256ac     error_messages.obj
 0002:000036c0       ??_C@_0CB@DMMJDFBN@HIERARCHY_CHANGE_NOT_IMPLEMENTE@ 100256c0     error_messages.obj
 0002:000036e4       ??_C@_0BO@EGGEGIDF@DELETE_METHOD_NOT_IMPLEMENTED@ 100256e4     error_messages.obj
 0002:00003704       ??_C@_0BE@MFLGLHIO@UNSUPPORTED_VERSION@ 10025704     error_messages.obj
 0002:00003718       ??_C@_0BB@GAODHGPJ@NAMES_DONT_MATCH@ 10025718     error_messages.obj
 0002:0000372c       ??_C@_0CH@NAGMIHMO@CLASS_MODIFIERS_CHANGE_NOT_IMPL@ 1002572c     error_messages.obj
 0002:00003754       ??_C@_0CI@BOHKDDHK@METHOD_MODIFIERS_CHANGE_NOT_IMP@ 10025754     error_messages.obj
 0002:0000377c       ??_C@_0CH@LDPJIDCO@CLASS_ATTRIBUTE_CHANGE_NOT_IMPL@ 1002577c     error_messages.obj
 0002:000037a4       ??_C@_0BA@PIOOPNBD@NOT_IMPLEMENTED@ 100257a4     error_messages.obj
 0002:000037b4       ??_C@_0N@HEEFEIAJ@NULL_POINTER@ 100257b4     error_messages.obj
 0002:000037c4       ??_C@_0BD@JCIODJA@ABSENT_INFORMATION@ 100257c4     error_messages.obj
 0002:000037d8       ??_C@_0BD@CAHCPDGO@INVALID_EVENT_TYPE@ 100257d8     error_messages.obj
 0002:000037ec       ??_C@_0BB@JNKCIGPM@ILLEGAL_ARGUMENT@ 100257ec     error_messages.obj
 0002:00003800       ??_C@_0O@KKNEIJDA@OUT_OF_MEMORY@ 10025800     error_messages.obj
 0002:00003810       ??_C@_0O@ILOHOCOF@ACCESS_DENIED@ 10025810     error_messages.obj
 0002:00003820       ??_C@_07DFGEEPDM@VM_DEAD@  10025820     error_messages.obj
 0002:00003828       ??_C@_08MLFDIMPC@INTERNAL@ 10025828     error_messages.obj
 0002:00003834       ??_C@_0BC@ENEFPEAF@UNATTACHED_THREAD@ 10025834     error_messages.obj
 0002:00003848       ??_C@_0M@NLBJDGPL@INVALID_TAG@ 10025848     error_messages.obj
 0002:00003854       ??_C@_0BB@GCBFLFGN@ALREADY_INVOKING@ 10025854     error_messages.obj
 0002:00003868       ??_C@_0O@BDGMMHPL@INVALID_INDEX@ 10025868     error_messages.obj
 0002:00003878       ??_C@_0P@MDIAHEHE@INVALID_LENGTH@ 10025878     error_messages.obj
 0002:00003888       ??_C@_0P@EJHKHOLE@INVALID_STRING@ 10025888     error_messages.obj
 0002:00003898       ??_C@_0BF@FLGJBCL@INVALID_CLASS_LOADER@ 10025898     error_messages.obj
 0002:000038b0       ??_C@_0O@DBEPKOML@INVALID_ARRAY@ 100258b0     error_messages.obj
 0002:000038c0       ??_C@_0P@IMPOLMOK@TRANSPORT_LOAD@ 100258c0     error_messages.obj
 0002:000038d0       ??_C@_0P@LIHDBHBG@TRANSPORT_INIT@ 100258d0     error_messages.obj
 0002:000038e0       ??_C@_0O@PMKFKNBA@NATIVE_METHOD@ 100258e0     error_messages.obj
 0002:000038f0       ??_C@_0O@MHNCFNDK@INVALID_COUNT@ 100258f0     error_messages.obj
 0002:00003900       ??_C@_0BD@EHLJKCDN@JDWP_ERROR_unknown@ 10025900     error_messages.obj
 0002:00003914       ??_C@_0DD@FOCDBFMB@DEBUGGING?3?5JDWP?5pause?5for?5PID?5?$CF@ 10025914     error_messages.obj
 0002:00003948       ??_C@_0DI@FMKFEDPB@DEBUGGING?3?5JDWP?5pause?5got?5tired@ 10025948     error_messages.obj
 0002:00003980       ??_C@_0DI@GJAHDGCJ@s?2src?2jdk?4jdwp?4agent?2share?2nati@ 10025980     eventFilter.obj
 0002:000039b8       ??_C@_0BB@GAFCOFIH@GetVersionNumber@ 100259b8     eventFilter.obj
 0002:000039cc       ??_C@_0BB@BEKNDEAI@GetLocalInstance@ 100259cc     eventFilter.obj
 0002:000039e0       ??_C@_0BB@FFOAPJHA@IsAssignableFrom@ 100259e0     eventFilter.obj
 0002:000039f4       ??_C@_0N@JPGMCHOC@IsInstanceOf@ 100259f4     eventFilter.obj
 0002:00003a04       ??_C@_0BK@BBNCBBEI@filter?9?$DOu?4Count?4count?5?$DO?50@ 10025a04     eventFilter.obj
 0002:00003a20       ??_C@_0BI@BDIJIJG@Invalid?5filter?5modifier@ 10025a20     eventFilter.obj
 0002:00003a38       ??_C@_03KPOLBBFN@LOC@      10025a38     eventFilter.obj
 0002:00003a3c       ??_C@_0DB@GIOMMMKK@SetBreakpoint?5at?5location?3?5meth@ 10025a3c     eventFilter.obj
 0002:00003a70       ??_C@_0O@OBFGDNOO@SetBreakpoint@ 10025a70     eventFilter.obj
 0002:00003a80       ??_C@_0DD@BOLIJEFD@ClearBreakpoint?5at?5location?3?5me@ 10025a80     eventFilter.obj
 0002:00003ab4       ??_C@_0BA@KALLGBAH@ClearBreakpoint@ 10025ab4     eventFilter.obj
 0002:00003ac4       ??_C@_0BE@BNFCJLBG@SetFieldAccessWatch@ 10025ac4     eventFilter.obj
 0002:00003ad8       ??_C@_0BK@LOHLKOFB@SetFieldModificationWatch@ 10025ad8     eventFilter.obj
 0002:00003af4       ??_C@_0BG@IELHINIE@ClearFieldAccessWatch@ 10025af4     eventFilter.obj
 0002:00003b0c       ??_C@_0BM@BCBGEJEO@ClearFieldModificationWatch@ 10025b0c     eventFilter.obj
 0002:00003b28       ??_C@_0DJ@IALHBKPF@s?2src?2jdk?4jdwp?4agent?2share?2nati@ 10025b28     eventHandler.obj
 0002:00003b64       ??_C@_0BG@HNCJHGFL@bad?5index?5for?5handler@ 10025b64     eventHandler.obj
 0002:00003b7c       ??_C@_0BH@GJLAODLP@iterator?5function?5NULL@ 10025b7c     eventHandler.obj
 0002:00003b98       ??_C@_0EP@MEMOEFKL@Co?9located?5breakpoint?5event?5fou@ 10025b98     eventHandler.obj
 0002:00003be8       ??_C@_0EL@CHJDLPBE@event?5report?5being?5skipped?3?5ei?$DN@ 10025be8     eventHandler.obj
 0002:00003c34       ??_C@_0BB@EIEOGLKK@eventBag?5?$CB?$DN?5NULL@ 10025c34     eventHandler.obj
 0002:00003c48       ??_C@_0BI@NCLCAKI@event_callback?$CI?$CJ?3?5ei?$DN?$CFs@ 10025c48     eventHandler.obj
 0002:00003c60       ??_C@_0BB@GKNNLBLP@event_callback?$CI?$CJ@ 10025c60     eventHandler.obj
 0002:00003c74       ??_C@_0BG@HHJEAHIC@handler?5function?5NULL@ 10025c74     eventHandler.obj
 0002:00003c8c       ??_C@_0CK@GFKKNCOE@Can?8t?5get?5jclass?5for?5a?5methodID@ 10025c8c     eventHandler.obj
 0002:00003cb8       ??_C@_0BI@OKNNPEIC@cbSingleStep?3?5thread?$DN?$CFp@ 10025cb8     eventHandler.obj
 0002:00003cd0       ??_C@_0CD@FPLFBNDA@Problems?5tracking?5active?5callba@ 10025cd0     eventHandler.obj
 0002:00003cf4       ??_C@_0BB@HHEIIDE@END?5cbSingleStep@ 10025cf4     eventHandler.obj
 0002:00003d08       ??_C@_0BI@INKCIGJH@cbBreakpoint?3?5thread?$DN?$CFp@ 10025d08     eventHandler.obj
 0002:00003d20       ??_C@_0BB@MLFPCDPM@END?5cbBreakpoint@ 10025d20     eventHandler.obj
 0002:00003d34       ??_C@_0BG@DJEPKKOO@cbFramePop?3?5thread?$DN?$CFp@ 10025d34     eventHandler.obj
 0002:00003d4c       ??_C@_0P@OGOCKOP@END?5cbFramePop@ 10025d4c     eventHandler.obj
 0002:00003d5c       ??_C@_0BH@OOFFIBDG@cbException?3?5thread?$DN?$CFp@ 10025d5c     eventHandler.obj
 0002:00003d74       ??_C@_0BA@JBFNAOBA@END?5cbException@ 10025d74     eventHandler.obj
 0002:00003d84       ??_C@_0BJ@DNMCHIHH@cbThreadStart?3?5thread?$DN?$CFp@ 10025d84     eventHandler.obj
 0002:00003da0       ??_C@_0BC@HNAGBODM@END?5cbThreadStart@ 10025da0     eventHandler.obj
 0002:00003db4       ??_C@_0BH@CLNHMLJ@cbThreadEnd?3?5thread?$DN?$CFp@ 10025db4     eventHandler.obj
 0002:00003dcc       ??_C@_0BA@PMEDEDIF@END?5cbThreadEnd@ 10025dcc     eventHandler.obj
 0002:00003ddc       ??_C@_0BK@KPCGMFCD@cbClassPrepare?3?5thread?$DN?$CFp@ 10025ddc     eventHandler.obj
 0002:00003df8       ??_C@_0BD@NJBOMDHE@END?5cbClassPrepare@ 10025df8     eventHandler.obj
 0002:00003e0c       ??_C@_0BK@DBGEMJPF@cbGarbageCollectionFinish@ 10025e0c     eventHandler.obj
 0002:00003e28       ??_C@_0BO@NFODBOGB@END?5cbGarbageCollectionFinish@ 10025e28     eventHandler.obj
 0002:00003e48       ??_C@_0BH@OAIHEEJM@cbClassLoad?3?5thread?$DN?$CFp@ 10025e48     eventHandler.obj
 0002:00003e60       ??_C@_0BA@OJJLNIBG@END?5cbClassLoad@ 10025e60     eventHandler.obj
 0002:00003e70       ??_C@_0BJ@NDKLILBO@cbFieldAccess?3?5thread?$DN?$CFp@ 10025e70     eventHandler.obj
 0002:00003e8c       ??_C@_0BC@PHEEKBJC@END?5cbFieldAccess@ 10025e8c     eventHandler.obj
 0002:00003ea0       ??_C@_0BP@NOJMIFFP@cbFieldModification?3?5thread?$DN?$CFp@ 10025ea0     eventHandler.obj
 0002:00003ec0       ??_C@_0BI@JFPADOMO@END?5cbFieldModification@ 10025ec0     eventHandler.obj
 0002:00003ed8       ??_C@_0BM@FNPGHFD@cbExceptionCatch?3?5thread?$DN?$CFp@ 10025ed8     eventHandler.obj
 0002:00003ef4       ??_C@_0BF@KCHHGDCL@END?5cbExceptionCatch@ 10025ef4     eventHandler.obj
 0002:00003f0c       ??_C@_0BJ@BDJJHIIJ@cbMethodEntry?3?5thread?$DN?$CFp@ 10025f0c     eventHandler.obj
 0002:00003f28       ??_C@_0BC@ODEOLGDB@END?5cbMethodEntry@ 10025f28     eventHandler.obj
 0002:00003f3c       ??_C@_0BI@DMPAEBFP@cbMethodExit?3?5thread?$DN?$CFp@ 10025f3c     eventHandler.obj
 0002:00003f54       ??_C@_0BB@DDLCHFPG@END?5cbMethodExit@ 10025f54     eventHandler.obj
 0002:00003f68       ??_C@_0CD@MLINJBLL@cbMonitorContendedEnter?3?5thread@ 10025f68     eventHandler.obj
 0002:00003f8c       ??_C@_0BM@FCFEADJF@END?5cbMonitorContendedEnter@ 10025f8c     eventHandler.obj
 0002:00003fa8       ??_C@_0CF@PHEBGJDK@cbMonitorContendedEntered?3?5thre@ 10025fa8     eventHandler.obj
 0002:00003fd0       ??_C@_0BO@NKLCNKNJ@END?5cbMonitorContendedEntered@ 10025fd0     eventHandler.obj
 0002:00003ff0       ??_C@_0BJ@DBNLPCK@cbMonitorWait?3?5thread?$DN?$CFp@ 10025ff0     eventHandler.obj
 0002:0000400c       ??_C@_0BC@HCJEOKMD@END?5cbMonitorWait@ 1002600c     eventHandler.obj
 0002:00004020       ??_C@_0BL@EDMNBHDO@cbMonitorWaited?3?5thread?$DN?$CFp@ 10026020     eventHandler.obj
 0002:0000403c       ??_C@_0BE@OPIFFKBH@END?5cbMonitorWaited@ 1002603c     eventHandler.obj
 0002:00004050       ??_C@_08JPFKMCJM@cbVMInit@ 10026050     eventHandler.obj
 0002:0000405c       ??_C@_0N@CGBLLPFL@END?5cbVMInit@ 1002605c     eventHandler.obj
 0002:0000406c       ??_C@_09FKPIGOCC@cbVMDeath@ 1002606c     eventHandler.obj
 0002:00004078       ??_C@_0CI@BDMPOPOL@Can?8t?5clear?5event?5callbacks?5on?5@ 10026078     eventHandler.obj
 0002:000040a0       ??_C@_0O@FPEBHIEM@END?5cbVMDeath@ 100260a0     eventHandler.obj
 0002:000040b0       ??_C@_0BD@GLFAIKMG@JDWP?5Callback?5Lock@ 100260b0     eventHandler.obj
 0002:000040c4       ??_C@_0BE@MNAKHAMD@JDWP?5Callback?5Block@ 100260c4     eventHandler.obj
 0002:000040d8       ??_C@_0BI@FOIPGHII@JDWP?5Event?5Handler?5Lock@ 100260d8     eventHandler.obj
 0002:000040f0       ??_C@_0BM@MPBGMHFO@Can?8t?5enable?5vm?5init?5events@ 100260f0     eventHandler.obj
 0002:0000410c       ??_C@_0BN@JOALGOKL@Can?8t?5enable?5vm?5death?5events@ 1002610c     eventHandler.obj
 0002:0000412c       ??_C@_0CB@JOBGHMA@Can?8t?5enable?5thread?5start?5event@ 1002612c     eventHandler.obj
 0002:00004150       ??_C@_0BP@FDDGJEME@Can?8t?5enable?5thread?5end?5events@ 10026150     eventHandler.obj
 0002:00004170       ??_C@_0CC@OGPPHNDL@Can?8t?5enable?5class?5prepare?5even@ 10026170     eventHandler.obj
 0002:00004194       ??_C@_0CO@BHGAKFIC@Can?8t?5enable?5garbage?5collection@ 10026194     eventHandler.obj
 0002:000041c4       ??_C@_0BK@PHMDAOAK@Can?8t?5set?5event?5callbacks@ 100261c4     eventHandler.obj
 0002:000041e0       ??_C@_0DA@KKIKEDIE@enqueueCommand?$CI?$CJ?3?5HelperCommand@ 100261e0     eventHelper.obj
 0002:00004210       ??_C@_0CF@LMNBMKHE@enqueueCommand?$CI?$CJ?3?5HelperCommand@ 10026210     eventHelper.obj
 0002:00004238       ??_C@_0CO@HANEHINJ@completeCommand?$CI?$CJ?3?5HelperComman@ 10026238     eventHelper.obj
 0002:00004268       ??_C@_0DI@GNPLLKOC@s?2src?2jdk?4jdwp?4agent?2share?2nati@ 10026268     eventHelper.obj
 0002:000042a0       ??_C@_0CJ@KNNNNIJI@dequeueCommand?$CI?$CJ?3?5command?5being@ 100262a0     eventHelper.obj
 0002:000042cc       ??_C@_0CK@HMEDCJBG@dequeueCommand?$CI?$CJ?3?5command?5sessi@ 100262cc     eventHelper.obj
 0002:000042f8       ??_C@_0BE@OLGJGEIN@unknown?5event?5index@ 100262f8     eventHelper.obj
 0002:0000430c       ??_C@_0BF@EBMLONF@Event?5Helper?5Command@ 1002630c     eventHelper.obj
 0002:00004324       ??_C@_0BK@IAKHDCAG@Begin?5command?5loop?5thread@ 10026324     eventHelper.obj
 0002:00004340       ??_C@_0CF@IHKNBMKL@commandLoop?$CI?$CJ?3?5command?5being?5ha@ 10026340     eventHelper.obj
 0002:00004368       ??_C@_0CA@PBIKJLAJ@JDWP?5Event?5Helper?5Queue?5Monitor@ 10026368     eventHelper.obj
 0002:00004388       ??_C@_0CF@DAMBCHBM@JDWP?5Event?5Helper?5Completion?5Mo@ 10026388     eventHelper.obj
 0002:000043b0       ??_C@_0CF@PDAKBDPJ@JDWP?5Event?5Block?5CommandLoop?5Mo@ 100263b0     eventHelper.obj
 0002:000043d8       ??_C@_0CC@JBOJCKEK@JDWP?5VM_DEATH?5CommandLoop?5Monit@ 100263d8     eventHelper.obj
 0002:000043fc       ??_C@_0BJ@MHCAKDHO@JDWP?5Event?5Helper?5Thread@ 100263fc     eventHelper.obj
 0002:00004418       ??_C@_0CP@KONMJMJG@exitVmDeathLockOnError?3?5error?5i@ 10026418     eventHelper.obj
 0002:00004448       ??_C@_0BB@POGOAJG@GetCurrentThread@ 10026448     eventHelper.obj
 0002:0000445c       ??_C@_0BB@BFBJHKBE@bagAdd?$CIeventBag?$CJ@ 1002645c     eventHelper.obj
 0002:00004470       ??_C@_0BI@GCGOKABC@err?5?$DN?$DN?5JVMTI_ERROR_NONE@ 10026470     eventHelper.obj
 0002:00004488       ??_C@_0O@LKPPNPDK@HelperCommand@ 10026488     eventHelper.obj
 0002:00004498       ??_C@_0P@FHCDPAEP@HelperCommmand@ 10026498     eventHelper.obj
 0002:000044a8       ??_C@_0BF@BPGCNEIM@JDWP?5Invocation?5Lock@ 100264a8     invoker.obj
 0002:000044c0       ??_C@_0CB@NAOIBAAB@Request?5methodSignature?5not?5nul@ 100264c0     invoker.obj
 0002:000044e4       ??_C@_0DE@EFONEHB@s?2src?2jdk?4jdwp?4agent?2share?2nati@ 100264e4     invoker.obj
 0002:00004518       ??_C@_06FJHNOCKE@thread@   10026518     invoker.obj
 0002:00004520       ??_C@_0BO@ICHBCBGF@getting?5thread?5invoke?5request@ 10026520     invoker.obj
 0002:00004540       ??_C@_0BI@MLBHEPJD@GetMethodDeclaringClass@ 10026540     invoker.obj
 0002:00004558       ??_C@_0N@FKNOGHOK@IsSameObject@ 10026558     invoker.obj
 0002:00004568       ??_C@_0BD@GGJIMJB@Request?5clazz?5null@ 10026568     invoker.obj
 0002:0000457c       ??_C@_0L@DEGKKCHL@NewObjectA@ 1002657c     invoker.obj
 0002:00004588       ??_C@_0BI@JEDJKLFO@CallStaticObjectMethodA@ 10026588     invoker.obj
 0002:000045a0       ??_C@_0BG@OLLEIINM@CallStaticByteMethodA@ 100265a0     invoker.obj
 0002:000045b8       ??_C@_0BG@BGEPLKKM@CallStaticCharMethodA@ 100265b8     invoker.obj
 0002:000045d0       ??_C@_0BH@PAMJMCFG@CallStaticFloatMethodA@ 100265d0     invoker.obj
 0002:000045e8       ??_C@_0BI@IBCKJKHM@CallStaticDoubleMethodA@ 100265e8     invoker.obj
 0002:00004600       ??_C@_0BF@JPBMCNAM@CallStaticIntMethodA@ 10026600     invoker.obj
 0002:00004618       ??_C@_0BG@FKLMGMON@CallStaticLongMethodA@ 10026618     invoker.obj
 0002:00004630       ??_C@_0BH@JGHONGAL@CallStaticShortMethodA@ 10026630     invoker.obj
 0002:00004648       ??_C@_0BJ@PIJAHNCD@CallStaticBooleanMethodA@ 10026648     invoker.obj
 0002:00004664       ??_C@_0BG@GHMCEOMM@CallStaticVoidMethodA@ 10026664     invoker.obj
 0002:0000467c       ??_C@_0BJ@NJKAEDMC@Invalid?5method?5signature@ 1002667c     invoker.obj
 0002:00004698       ??_C@_0BG@LMEMBPGM@Request?5instance?5null@ 10026698     invoker.obj
 0002:000046b0       ??_C@_0BC@DPOBDBNG@CallObjectMethodA@ 100266b0     invoker.obj
 0002:000046c4       ??_C@_0BA@PKCJIMNA@CallByteMethodA@ 100266c4     invoker.obj
 0002:000046d4       ??_C@_0BA@HNCLOKA@CallCharMethodA@ 100266d4     invoker.obj
 0002:000046e4       ??_C@_0BB@PJGOBDHJ@CallFloatMethodA@ 100266e4     invoker.obj
 0002:000046f8       ??_C@_0BC@CKPCAAPE@CallDoubleMethodA@ 100266f8     invoker.obj
 0002:0000470c       ??_C@_0P@DBDHNNH@CallIntMethodA@ 1002670c     invoker.obj
 0002:0000471c       ??_C@_0BA@ELCBGIOB@CallLongMethodA@ 1002671c     invoker.obj
 0002:0000472c       ??_C@_0BB@JPNJAHCE@CallShortMethodA@ 1002672c     invoker.obj
 0002:00004740       ??_C@_0BD@BLFIKOKL@CallBooleanMethodA@ 10026740     invoker.obj
 0002:00004754       ??_C@_0BA@HGFPEKMA@CallVoidMethodA@ 10026754     invoker.obj
 0002:00004764       ??_C@_0BM@GJKAAPAH@CallNonvirtualObjectMethodA@ 10026764     invoker.obj
 0002:00004780       ??_C@_0BK@GCNLPHID@CallNonvirtualByteMethodA@ 10026780     invoker.obj
 0002:0000479c       ??_C@_0BK@JPCAMFPD@CallNonvirtualCharMethodA@ 1002679c     invoker.obj
 0002:000047b8       ??_C@_0BL@LJEOBEM@CallNonvirtualFloatMethodA@ 100267b8     invoker.obj
 0002:000047d4       ??_C@_0BM@HMLDDOCF@CallNonvirtualDoubleMethodA@ 100267d4     invoker.obj
 0002:000047f0       ??_C@_0BJ@CDEIJCJF@CallNonvirtualIntMethodA@ 100267f0     invoker.obj
 0002:0000480c       ??_C@_0BK@NDNDBDLC@CallNonvirtualLongMethodA@ 1002680c     invoker.obj
 0002:00004828       ??_C@_0BL@GNCDPFBB@CallNonvirtualShortMethodA@ 10026828     invoker.obj
 0002:00004844       ??_C@_0BN@OKNKANNH@CallNonvirtualBooleanMethodA@ 10026844     invoker.obj
 0002:00004864       ??_C@_0BK@OOKNDBJD@CallNonvirtualVoidMethodA@ 10026864     invoker.obj
 0002:00004880       ??_C@_0BB@EDABLKKF@request?9?$DOpending@ 10026880     invoker.obj
 0002:00004894       ??_C@_0BB@JHNKMJKL@request?9?$DOstarted@ 10026894     invoker.obj
 0002:000048a8       ??_C@_0BI@OKOEINGF@methodSignature?5is?5NULL@ 100268a8     invoker.obj
 0002:000048c0       ??_C@_07ENHGAJCI@request@  100268c0     invoker.obj
 0002:000048c8       ??_C@_09CMKFMIAO@?$CFs?2?$CFs?4dll@ 100268c8     linker_md.obj
 0002:000048d4       ??_C@_0DI@JPDHMHMH@s?2src?2jdk?4jdwp?4agent?2windows?2na@ 100268d4     linker_md.obj
 0002:00004910       ??_C@_0GB@EFLPCEDF@One?5or?5more?5of?5the?5library?5path@ 10026910     linker_md.obj
 0002:00004974       ??_C@_06DAJAKOAL@?$CFs?4dll@ 10026974     linker_md.obj
 0002:0000497c       ??_C@_0BP@KMBPCJLM@Can?8t?5find?5dependent?5libraries@ 1002697c     linker_md.obj
 0002:0000499c       ??_C@_0M@ILCKPJLM@?$CFd?4?$CFm?4?$CFY?5?$CFT@ 1002699c     log_messages.obj
 0002:000049a8       ??_C@_02HOGMBHDI@?$CFZ@    100269a8     log_messages.obj
 0002:000049ac       ??_C@_04FHKNIFPB@?$CF?43d@ 100269ac     log_messages.obj
 0002:000049b4       ??_C@_0L@LMNAMKMD@?$CFs?4?$CF?43s?5?$CFs@ 100269b4     log_messages.obj
 0002:000049c0       ??_C@_07CIFAGBMG@unknown@  100269c0     log_messages.obj
 0002:000049c8       ??_C@_0M@JJMNGIAI@?$CFs?3?$CC?$CFs?$CC?3?$CFd?$DL@ 100269c8     log_messages.obj
 0002:000049d4       ??_C@_0BM@BMLHDEI@?$FL?$CD?$HM?$CFs?$HM?$CFs?$HM?$CFs?$HM?$CFs?$HM?$CFs?$HM?$CFs?3?$CFs?$HM?$CD?$FN?6@ 100269d4     log_messages.obj
 0002:000049f0       ??_C@_01NOFIACDB@w@        100269f0     log_messages.obj
 0002:000049f4       ??_C@_06JGDLHNPI@FINEST@   100269f4     log_messages.obj
 0002:000049fc       ??_C@_07NPAANBDA@J2SE1?45@ 100269fc     log_messages.obj
 0002:00004a04       ??_C@_04CAJKAAHJ@jdwp@     10026a04     log_messages.obj
 0002:00004a0c       ??_C@_0BH@HINFEDE@LOC?$DN?$CFs?$DLPID?$DN?$CFd?$DLTHR?$DNt?$EA?$CFd@ 10026a0c     log_messages.obj
 0002:00004a24       ??_C@_05NINEKCGD@?$CFs?4?$CFd@ 10026a24     log_messages.obj
 0002:00004a2c       ??_C@_0DG@EGMOAHHB@s?2src?2jdk?4jdwp?4agent?2share?2nati@ 10026a2c     outStream.obj
 0002:00004a64       ??_C@_0BB@JPLDOFMC@Invalid?5type?5key@ 10026a64     outStream.obj
 0002:00004a78       ??_C@_0CA@OJHGJLHC@outStream_setError?5error?$DN?$CFs?$CI?$CFd?$CJ@ 10026a78     outStream.obj
 0002:00004a98       ??_C@_0BE@DHHKMLKH@isArrayTag?$CItypeKey?$CJ@ 10026a98     signature.obj
 0002:00004aac       ??_C@_0DG@EOHOCBDN@s?2src?2jdk?4jdwp?4agent?2share?2nati@ 10026aac     signature.obj
 0002:00004ae4       ??_C@_06BHPCHHEB@tagPtr@   10026ae4     signature.obj
 0002:00004aec       ??_C@_0CF@NLOPLAKC@signature?$FL0?$FN?5?$DN?$DN?5SIGNATURE_BEGIN@ 10026aec     signature.obj
 0002:00004b14       ??_C@_0DA@CGCGEBGH@Should?5never?5call?5handleGarbage@ 10026b14     standardHandlers.obj
 0002:00004b44       ??_C@_0DN@BIHCGFFE@s?2src?2jdk?4jdwp?4agent?2share?2nati@ 10026b44     standardHandlers.obj
 0002:00004b84       ??_C@_0CJ@EJBINECN@Unable?5to?5install?5VM?5Death?5even@ 10026b84     standardHandlers.obj
 0002:00004bb0       ??_C@_0DI@LNANLGGM@s?2src?2jdk?4jdwp?4agent?2share?2nati@ 10026bb0     stepControl.obj
 0002:00004be8       ??_C@_0BE@MKGOBEGB@getting?5frame?5count@ 10026be8     stepControl.obj
 0002:00004bfc       ??_C@_04MOOLDHHD@STEP@     10026bfc     stepControl.obj
 0002:00004c04       ??_C@_0BK@NIDDNIOA@enableStepping?3?5thread?$DN?$CFp@ 10026c04     stepControl.obj
 0002:00004c20       ??_C@_0BF@CCJDHFEH@enabling?5single?5step@ 10026c20     stepControl.obj
 0002:00004c38       ??_C@_0BL@EHDJHHNF@disableStepping?3?5thread?$DN?$CFp@ 10026c38     stepControl.obj
 0002:00004c54       ??_C@_0BG@LEFCIDGN@disabling?5single?5step@ 10026c54     stepControl.obj
 0002:00004c6c       ??_C@_0P@IEFLKDKM@NotifyFramePop@ 10026c6c     stepControl.obj
 0002:00004c7c       ??_C@_0BG@OKKJJMAC@initState?$CI?$CJ?3?5frame?$DN?$CFd@ 10026c7c     stepControl.obj
 0002:00004c94       ??_C@_0BN@LKIHPCMO@initState?$CI?$CJ?3?5Begin?5line?5step@ 10026c94     stepControl.obj
 0002:00004cb4       ??_C@_0BF@FOPEDPHN@getting?5step?5request@ 10026cb4     stepControl.obj
 0002:00004ccc       ??_C@_0DJ@BEIBIGEH@handleFramePopEvent?3?5BEGIN?5from@ 10026ccc     stepControl.obj
 0002:00004d08       ??_C@_0DG@IPJGEBF@handleFramePopEvent?3?5starting?5s@ 10026d08     stepControl.obj
 0002:00004d40       ??_C@_0FK@PCMGCGNB@handleFramePopEvent?3?5starting?5s@ 10026d40     stepControl.obj
 0002:00004d9c       ??_C@_0CF@MGOMDHJC@step?9?$DOdepth?5?$DN?$DN?5JDWP_STEP_DEPTH?$CI@ 10026d9c     stepControl.obj
 0002:00004dc8       ??_C@_0HJ@MEDPAGIL@handleFramePopEvent?3?5starting?5s@ 10026dc8     stepControl.obj
 0002:00004e48       ??_C@_0HH@NFEOAAP@handleFramePopEvent?3?5starting?5s@ 10026e48     stepControl.obj
 0002:00004ec0       ??_C@_0BO@EJIOKDML@handleFramePopEvent?3?5finished@ 10026ec0     stepControl.obj
 0002:00004ee0       ??_C@_0DJ@FFHBGECC@handleExceptionCatchEvent?3?5from@ 10026ee0     stepControl.obj
 0002:00004f1c       ??_C@_0CC@GMNCKPDI@handleMethodEnterEvent?3?5thread?$DN@ 10026f1c     stepControl.obj
 0002:00004f40       ??_C@_0BI@ONNFECIM@completeStep?3?5thread?$DN?$CFp@ 10026f40     stepControl.obj
 0002:00004f58       ??_C@_0BI@POGAKJLC@initializing?5step?5state@ 10026f58     stepControl.obj
 0002:00004f70       ??_C@_0CC@JMCHFEAK@stepControl_handleStep?3?5thread?$DN@ 10026f70     stepControl.obj
 0002:00004f94       ??_C@_0CM@NNBPEOLN@stepControl_handleStep?3?5complet@ 10026f94     stepControl.obj
 0002:00004fc0       ??_C@_0DA@FOFCMEJP@stepControl_handleStep?3?5complet@ 10026fc0     stepControl.obj
 0002:00004ff0       ??_C@_0EB@JJDJIOHA@stepControl_handleStep?3?5complet@ 10026ff0     stepControl.obj
 0002:00005038       ??_C@_0FM@PAKAGCBL@stepControl_handleStep?3?5complet@ 10027038     stepControl.obj
 0002:00005094       ??_C@_0CG@MFJECOCG@installing?5event?5method?5enter?5h@ 10027094     stepControl.obj
 0002:000050c0       ??_C@_0EG@INCGEIIO@stepControl_handleStep?3?5NotifyF@ 100270c0     stepControl.obj
 0002:00005108       ??_C@_0BM@IPAAJJGN@setting?5up?5notify?5frame?5pop@ 10027108     stepControl.obj
 0002:00005128       ??_C@_0EH@PDNBFMBE@stepControl_handleStep?3?5complet@ 10027128     stepControl.obj
 0002:00005170       ??_C@_0BH@BJILJMJK@getting?5frame?5location@ 10027170     stepControl.obj
 0002:00005188       ??_C@_0CP@KIJNJAEA@stepControl_handleStep?3?5checkin@ 10027188     stepControl.obj
 0002:000051b8       ??_C@_0CK@BMELMNFO@stepControl_handleStep?3?5checkin@ 100271b8     stepControl.obj
 0002:000051e8       ??_C@_0FC@HLIPCJAI@stepControl_handleStep?3?5complet@ 100271e8     stepControl.obj
 0002:00005240       ??_C@_0EL@JOGIECCM@stepControl_handleStep?3?5complet@ 10027240     stepControl.obj
 0002:0000528c       ??_C@_0CB@DMEMPEEG@stepControl_handleStep?3?5finishe@ 1002728c     stepControl.obj
 0002:000052b0       ??_C@_0BH@NFDHFKGE@JDWP?5Step?5Handler?5Lock@ 100272b0     stepControl.obj
 0002:000052c8       ??_C@_0CE@GBBAGAOP@stepControl_resetRequest?3?5threa@ 100272c8     stepControl.obj
 0002:000052ec       ??_C@_0CC@POHINOEB@step?9?$DOframePopHandlerNode?5?$DN?$DN?5NU@ 100272ec     stepControl.obj
 0002:00005310       ??_C@_0BP@KCAAPAME@installing?5step?5event?5handlers@ 10027310     stepControl.obj
 0002:00005330       ??_C@_0DC@LKPPLDLN@stepControl_beginStep?3?5thread?$DN?$CF@ 10027330     stepControl.obj
 0002:00005364       ??_C@_0CN@MHELALJG@stepControl_beginStep?3?5cannot?5s@ 10027364     stepControl.obj
 0002:00005394       ??_C@_0BP@INDEPPPG@stepControl_endStep?3?5thread?$DN?$CFp@ 10027394     stepControl.obj
 0002:000053b4       ??_C@_0CE@EJEIFKKI@stepControl_clearRequest?3?5threa@ 100273b4     stepControl.obj
 0002:000053d8       ??_C@_0DK@MIIMOJNB@s?2src?2jdk?4jdwp?4agent?2share?2nati@ 100273d8     threadControl.obj
 0002:00005414       ??_C@_0P@BHNPMDOE@GetThreadState@ 10027414     threadControl.obj
 0002:00005424       ??_C@_0BG@OHKNBDMG@SetThreadLocalStorage@ 10027424     threadControl.obj
 0002:0000543c       ??_C@_0CA@BNIMIHGG@cannot?5set?5thread?5local?5storage@ 1002743c     threadControl.obj
 0002:0000545c       ??_C@_0BG@BCPLMKIH@GetThreadLocalStorage@ 1002745c     threadControl.obj
 0002:00005474       ??_C@_0CA@LOCGOKPD@cannot?5get?5thread?5local?5storage@ 10027474     threadControl.obj
 0002:00005494       ??_C@_0BD@NHJKPLLD@thread?5table?5entry@ 10027494     threadControl.obj
 0002:000054a8       ??_C@_0CH@CFIIJJMO@findThread?$CIdest?0?5node?9?$DOthread?$CJ?5@ 100274a8     threadControl.obj
 0002:000054d0       ??_C@_0ED@OAECAMKM@cannot?5process?5deferred?5thread?5@ 100274d0     threadControl.obj
 0002:00005514       ??_C@_0BB@EFDALKHP@JDWP?5Thread?5Lock@ 10027514     threadControl.obj
 0002:00005528       ??_C@_0BK@CAIODGML@no?5java?4lang?4thread?5class@ 10027528     threadControl.obj
 0002:00005544       ??_C@_0BF@OPEELAAF@cannot?5resume?5thread@ 10027544     threadControl.obj
 0002:0000555c       ??_C@_0BI@IPGEEFGE@getting?5method?5location@ 1002755c     threadControl.obj
 0002:00005574       ??_C@_0BF@KAINFNPD@getting?5thread?5state@ 10027574     threadControl.obj
 0002:0000558c       ??_C@_0BM@BDKKJJIL@node?9?$DOresumeFrameDepth?5?$DN?$DN?50@ 1002758c     threadControl.obj
 0002:000055a8       ??_C@_0N@BJJFBAKB@thread?5table@ 100275a8     threadControl.obj
 0002:000055b8       ??_C@_0BE@PLBAIHPP@thread?$DN?$CFp?5suspended@ 100275b8     threadControl.obj
 0002:000055cc       ??_C@_0O@HMJOGGOE@SuspendThread@ 100275cc     threadControl.obj
 0002:000055dc       ??_C@_0BC@DNHNKGGE@thread?$DN?$CFp?5resumed@ 100275dc     threadControl.obj
 0002:000055f0       ??_C@_0N@JPHIGJOE@ResumeThread@ 100275f0     threadControl.obj
 0002:00005600       ??_C@_0BE@PGDPIDGL@resume?5request?5list@ 10027600     threadControl.obj
 0002:00005614       ??_C@_0M@FIFGDPKA@resume?5list@ 10027614     threadControl.obj
 0002:00005620       ??_C@_0BB@FPIEDMNB@ResumeThreadList@ 10027620     threadControl.obj
 0002:00005634       ??_C@_0CG@OGGIDGFO@missing?5entry?5in?5running?5thread@ 10027634     threadControl.obj
 0002:0000565c       ??_C@_0CC@EENAOFCJ@thread?$DN?$CFp?5resumed?5as?5part?5of?5li@ 1002765c     threadControl.obj
 0002:00005680       ??_C@_0N@JJLGEDON@request?5list@ 10027680     threadControl.obj
 0002:00005690       ??_C@_0BF@BGHKIDKG@suspend?5list?5results@ 10027690     threadControl.obj
 0002:000056a8       ??_C@_0BC@GFPPJMEE@SuspendThreadList@ 100276a8     threadControl.obj
 0002:000056bc       ??_C@_0BP@JBJIEHDD@missing?5entry?5in?5thread?5tables@ 100276bc     threadControl.obj
 0002:000056dc       ??_C@_0CE@BDMKGMJL@thread?$DN?$CFp?5suspended?5as?5part?5of?5@ 100276dc     threadControl.obj
 0002:00005700       ??_C@_0BO@IJHNAMAJ@threadControl_suspendThread?$CI?$CJ@ 10027700     threadControl.obj
 0002:00005720       ??_C@_0BN@GKLHJPIH@threadControl_resumeThread?$CI?$CJ@ 10027720     threadControl.obj
 0002:00005740       ??_C@_0BL@CGJFPBGG@threadControl_suspendAll?$CI?$CJ@ 10027740     threadControl.obj
 0002:0000575c       ??_C@_0BK@KAONLLJF@threadControl_resumeAll?$CI?$CJ@ 1002775c     threadControl.obj
 0002:00005778       ??_C@_0BJ@CHKMKGNA@JDWP?5PopFrame?5Event?5Lock@ 10027778     threadControl.obj
 0002:00005794       ??_C@_0BL@NLADKEIC@JDWP?5PopFrame?5Proceed?5Lock@ 10027794     threadControl.obj
 0002:000057b0       ??_C@_0BG@BDPIMKHA@entry?5in?5thread?5table@ 100277b0     threadControl.obj
 0002:000057c8       ??_C@_08PALMFDC@PopFrame@  100277c8     threadControl.obj
 0002:000057d4       ??_C@_0CB@FDGFBJBH@thread?$DN?$CFp?5resumed?5in?5popOneFram@ 100277d4     threadControl.obj
 0002:000057f8       ??_C@_0CD@CBFJIOGD@thread?$DN?$CFp?5suspended?5in?5popOneFr@ 100277f8     threadControl.obj
 0002:0000581c       ??_C@_0BK@HGCCNNPL@threadControl_popFrames?$CI?$CJ@ 1002781c     threadControl.obj
 0002:00005838       ??_C@_0BO@BMDHOIKK@thread?5start?5during?5pop?5frame@ 10027838     threadControl.obj
 0002:00005858       ??_C@_0CE@DLABLPCM@threadControl_onEventHandlerEnt@ 10027858     threadControl.obj
 0002:0000587c       ??_C@_0BA@PNKGFJII@InterruptThread@ 1002787c     threadControl.obj
 0002:0000588c       ??_C@_0L@FBFPPEII@StopThread@ 1002788c     threadControl.obj
 0002:00005898       ??_C@_0CD@DBNMOEOD@threadControl_onEventHandlerExi@ 10027898     threadControl.obj
 0002:000058bc       ??_C@_0BG@EPAAPLLF@thread?5list?5corrupted@ 100278bc     threadControl.obj
 0002:000058d4       ??_C@_0CI@GCOAEGE@threadControl_applicationThread@ 100278d4     threadControl.obj
 0002:000058fc       ??_C@_0BK@BIOOONKE@threadControl_interrupt?$CI?$CJ@ 100278fc     threadControl.obj
 0002:00005918       ??_C@_0BF@NHLBNOB@threadControl_stop?$CI?$CJ@ 10027918     threadControl.obj
 0002:00005930       ??_C@_0BL@KPAJNPJE@otherThreads?4first?5?$DN?$DN?5NULL@ 10027930     threadControl.obj
 0002:0000594c       ??_C@_0DG@DKBGPIDI@s?2src?2jdk?4jdwp?4agent?2share?2nati@ 1002794c     transport.obj
 0002:00005984       ??_C@_0BH@DPMJLMBJ@transport?5error?5?$CFd?3?5?$CFs@ 10027984     transport.obj
 0002:0000599c       ??_C@_07NFANNNEC@UNKNOWN@  1002799c     transport.obj
 0002:000059a4       ??_C@_0BJ@JEKDFBOP@_jdwpTransport_OnLoad?$EA16@ 100279a4     transport.obj
 0002:000059c0       ??_C@_0BF@FOBNBFPM@jdwpTransport_OnLoad@ 100279c0     transport.obj
 0002:000059d8       ??_C@_0BG@FMJOLAEE@library?5name?5is?5empty@ 100279d8     transport.obj
 0002:000059f0       ??_C@_0CI@LAKGPIH@internal?5error?3?5info?5should?5not@ 100279f0     transport.obj
 0002:00005a18       ??_C@_0CP@KHDMANEH@Java?5property?5sun?4boot?4library?4@ 10027a18     transport.obj
 0002:00005a48       ??_C@_0CA@EHDNLIPG@transport?5library?5not?5found?3?5?$CFs@ 10027a48     transport.obj
 0002:00005a68       ??_C@_0CL@KNFBHFGD@transport?5library?5missing?5onLoa@ 10027a68     transport.obj
 0002:00005a94       ??_C@_09KFMAMAFK@GetJavaVM@ 10027a94     transport.obj
 0002:00005aa0       ??_C@_0CP@JIHKFCKD@insufficient?5memory?5to?5complete@ 10027aa0     transport.obj
 0002:00005ad0       ??_C@_0EB@ONKBAHBP@transport?5doesn?8t?5recognize?5all@ 10027ad0     transport.obj
 0002:00005b14       ??_C@_0DA@LIDKNCMN@transport?5doesn?8t?5support?5multi@ 10027b14     transport.obj
 0002:00005b44       ??_C@_0CF@BGANCHCG@unrecognized?5error?5?$CFd?5from?5tran@ 10027b44     transport.obj
 0002:00005b6c       ??_C@_0BJ@IFDFBAP@sun?4jdwp?4listenerAddress@ 10027b6c     transport.obj
 0002:00005b88       ??_C@_0BE@JKJABKEE@Begin?5accept?5thread@ 10027b88     transport.obj
 0002:00005b9c       ??_C@_0CK@GLGDCAJA@could?5not?5connect?0?5timeout?5or?5f@ 10027b9c     transport.obj
 0002:00005bc8       ??_C@_0BC@NENNJKEM@End?5accept?5thread@ 10027bc8     transport.obj
 0002:00005bdc       ??_C@_0BE@BNNAEGLJ@Begin?5attach?5thread@ 10027bdc     transport.obj
 0002:00005bf0       ??_C@_0BC@FDJNMGLB@End?5attach?5thread@ 10027bf0     transport.obj
 0002:00005c04       ??_C@_0CA@PPOAMFKF@JDWP?5Transport?5Listener?5Monitor@ 10027c04     transport.obj
 0002:00005c24       ??_C@_0BM@EOHCCJHG@JDWP?5Transport?5Send?5Monitor@ 10027c24     transport.obj
 0002:00005c40       ??_C@_01CLKCMJKC@?5@       10027c40     transport.obj
 0002:00005c44       ??_C@_0DO@LDLIIPAI@Allow?5parameter?5is?5specified?5bu@ 10027c44     transport.obj
 0002:00005c84       ??_C@_01JLIPDDHJ@?3@       10027c84     transport.obj
 0002:00005c88       ??_C@_0BK@NKDBJPAM@JDWP?5Transport?5Listener?3?5@ 10027c88     transport.obj
 0002:00005ca4       ??_C@_0CK@NABHANCN@Listening?5for?5transport?5?$CFs?5at?5a@ 10027ca4     transport.obj
 0002:00005cd0       ??_C@_0BJ@NDKKCKOJ@UTF?5ERROR?5?$FL?$CC?$CFs?$CC?3?$CFd?$FN?3?5?$CFs?6@ 10027cd0     utf_util.obj
 0002:00005cec       ??_C@_0BH@PGKNPGMC@ASSERT?5ERROR?5i?$DN?$DNlength@ 10027cec     utf_util.obj
 0002:00005d04       ??_C@_0DF@HFLPGPCA@s?2src?2jdk?4jdwp?4agent?2share?2nati@ 10027d04     utf_util.obj
 0002:00005d3c       ??_C@_0BK@HADMOKCE@ASSERT?5ERROR?5j?$DN?$DNnewLength@ 10027d3c     utf_util.obj
 0002:00005d58       ??_C@_0BN@ILDOBJEF@Can?8t?5get?5WIDE?5string?5length@ 10027d58     utf_util.obj
 0002:00005d78       ??_C@_0BJ@LFBNLHDK@Can?8t?5malloc?$CI?$CJ?5any?5space@ 10027d78     utf_util.obj
 0002:00005d94       ??_C@_0BG@OELEGHKP@Can?8t?5get?5WIDE?5string@ 10027d94     utf_util.obj
 0002:00005dac       ??_C@_0BC@FAJHJFKN@ASSERT?5ERROR?5utf8@ 10027dac     utf_util.obj
 0002:00005dc0       ??_C@_0BE@MONHEHKE@ASSERT?5ERROR?5output@ 10027dc0     utf_util.obj
 0002:00005dd4       ??_C@_0BG@IGPBKLGM@ASSERT?5ERROR?5len?5?$DO?$DN?50@ 10027dd4     utf_util.obj
 0002:00005dec       ??_C@_0CB@NCJBKIBF@ASSERT?5ERROR?5outputBufSize?5?$DO?5le@ 10027dec     utf_util.obj
 0002:00005e10       ??_C@_0BB@LBCDKBGH@ASSERT?5ERROR?5str@ 10027e10     utf_util.obj
 0002:00005e24       ??_C@_0CI@EJHCPIBO@Can?8t?5convert?5WIDE?5string?5to?5mu@ 10027e24     utf_util.obj
 0002:00005e4c       ??_C@_0DB@OKLBDJGC@s?2src?2jdk?4jdwp?4agent?2share?2nati@ 10027e4c     util.obj
 0002:00005e80       ??_C@_0BD@FDGEFMPC@saveGlobalRef?5pobj@ 10027e80     util.obj
 0002:00005e94       ??_C@_0BE@HPCONGOG@saveGlobalRef?5?$CKpobj@ 10027e94     util.obj
 0002:00005ea8       ??_C@_0BC@DCADFAHL@saveGlobalRef?5env@ 10027ea8     util.obj
 0002:00005ebc       ??_C@_0BC@LCNDBECG@saveGlobalRef?5obj@ 10027ebc     util.obj
 0002:00005ed0       ??_C@_0BD@EBGPHOMG@tossGlobalRef?5pobj@ 10027ed0     util.obj
 0002:00005ee4       ??_C@_0BC@IOMIDECC@tossGlobalRef?5env@ 10027ee4     util.obj
 0002:00005ef8       ??_C@_0BC@OBIHAHP@tossGlobalRef?5obj@ 10027ef8     util.obj
 0002:00005f0c       ??_C@_0O@IHOLADDN@findClass?5env@ 10027f0c     util.obj
 0002:00005f1c       ??_C@_0P@HPKFFFCG@findClass?5name@ 10027f1c     util.obj
 0002:00005f2c       ??_C@_09MBLIIDDK@FindClass@ 10027f2c     util.obj
 0002:00005f38       ??_C@_0BJ@HIODLEDE@JDWP?5Can?8t?5find?5class?5?$CFs@ 10027f38     util.obj
 0002:00005f54       ??_C@_0CJ@HHGLKNAH@JDWP?5Exception?5occurred?5finding@ 10027f54     util.obj
 0002:00005f80       ??_C@_0O@GPBJKDDD@getMethod?5env@ 10027f80     util.obj
 0002:00005f90       ??_C@_0BA@FGFFFLNK@getMethod?5clazz@ 10027f90     util.obj
 0002:00005fa0       ??_C@_0P@JIPFIKIB@getMethod?5name@ 10027fa0     util.obj
 0002:00005fb0       ??_C@_0BE@CCFOHHKE@getMethod?5signature@ 10027fb0     util.obj
 0002:00005fc4       ??_C@_0M@BBNOPHHB@GetMethodID@ 10027fc4     util.obj
 0002:00005fd0       ??_C@_0CM@BOMIIGLD@JDWP?5Can?8t?5find?5method?5?$CFs?5with?5@ 10027fd0     util.obj
 0002:00005ffc       ??_C@_0DM@IMIOOKLN@JDWP?5Exception?5occurred?5finding@ 10027ffc     util.obj
 0002:00006038       ??_C@_0BE@PJAHCBJI@getStaticMethod?5env@ 10028038     util.obj
 0002:0000604c       ??_C@_0BG@BIBAEKOK@getStaticMethod?5clazz@ 1002804c     util.obj
 0002:00006064       ??_C@_0BF@NJGHOOGD@getStaticMethod?5name@ 10028064     util.obj
 0002:0000607c       ??_C@_0BK@NDPLJBJF@getStaticMethod?5signature@ 1002807c     util.obj
 0002:00006098       ??_C@_0BC@MJDCJNCH@GetStaticMethodID@ 10028098     util.obj
 0002:000060ac       ??_C@_0BA@JJLOPNCP@java?1lang?1Class@ 100280ac     util.obj
 0002:000060bc       ??_C@_0BB@NOKBFPFO@java?1lang?1Thread@ 100280bc     util.obj
 0002:000060d0       ??_C@_0BG@FMEDAMPL@java?1lang?1ThreadGroup@ 100280d0     util.obj
 0002:000060e8       ??_C@_0BG@HADLBHEN@java?1lang?1ClassLoader@ 100280e8     util.obj
 0002:00006100       ??_C@_0BB@FLFAIHG@java?1lang?1String@ 10028100     util.obj
 0002:00006114       ??_C@_0BB@NAICLKDB@java?1lang?1System@ 10028114     util.obj
 0002:00006128       ??_C@_0BF@JMMLIHKH@java?1util?1Properties@ 10028128     util.obj
 0002:00006140       ??_C@_0CN@EFABAIOP@?$CILjava?1lang?1ThreadGroup?$DLLjava?1l@ 10028140     util.obj
 0002:00006170       ??_C@_06FALKBLGB@?$DMinit?$DO@ 10028170     util.obj
 0002:00006178       ??_C@_04LHKBAEFM@?$CIZ?$CJV@ 10028178     util.obj
 0002:00006180       ??_C@_09GMGCGCNB@setDaemon@ 10028180     util.obj
 0002:0000618c       ??_C@_03GAEACAIP@?$CI?$CJV@ 1002818c     util.obj
 0002:00006190       ??_C@_06PLELHCEK@resume@   10028190     util.obj
 0002:00006198       ??_C@_0CH@NCPCFFHJ@?$CILjava?1lang?1String?$DL?$CJLjava?1lang?1@ 10028198     util.obj
 0002:000061c0       ??_C@_0M@NBNLNHMA@getProperty@ 100281c0     util.obj
 0002:000061cc       ??_C@_0DJ@BABOCAJP@?$CILjava?1lang?1String?$DLLjava?1lang?1S@ 100281cc     util.obj
 0002:00006208       ??_C@_0M@NOMFABED@setProperty@ 10028208     util.obj
 0002:00006214       ??_C@_0BO@CMFEIIEP@Can?8t?5get?5system?5thread?5group@ 10028214     util.obj
 0002:00006234       ??_C@_0N@KAKDDEJA@java?4version@ 10028234     util.obj
 0002:00006244       ??_C@_0N@FFLEMEAC@java?4vm?4name@ 10028244     util.obj
 0002:00006254       ??_C@_0N@EJENAPCP@java?4vm?4info@ 10028254     util.obj
 0002:00006264       ??_C@_0BA@BKCDAGON@java?4class?4path@ 10028264     util.obj
 0002:00006274       ??_C@_0BG@HAHGGNHO@sun?4boot?4library?4path@ 10028274     util.obj
 0002:0000628c       ??_C@_0P@GNCHJOPK@path?4separator@ 1002828c     util.obj
 0002:0000629c       ??_C@_08IOMDCONK@user?4dir@ 1002829c     util.obj
 0002:000062a8       ??_C@_0BK@DKBCNDAC@jdk?1internal?1vm?1VMSupport@ 100282a8     util.obj
 0002:000062c4       ??_C@_0BJ@BIOCMJG@?$CI?$CJLjava?1util?1Properties?$DL@ 100282c4     util.obj
 0002:000062e0       ??_C@_0BD@KIFIICML@getAgentProperties@ 100282e0     util.obj
 0002:000062f4       ??_C@_0BH@FMELKLIP@CallStaticObjectMethod@ 100282f4     util.obj
 0002:0000630c       ??_C@_0DI@CNPAJEKH@Exception?5occurred?5calling?5VMSu@ 1002830c     util.obj
 0002:00006344       ??_C@_0P@NGFPBMPI@GetObjectField@ 10028344     util.obj
 0002:00006354       ??_C@_0N@PICDCNEH@GetByteField@ 10028354     util.obj
 0002:00006364       ??_C@_0N@DKHIINEE@GetCharField@ 10028364     util.obj
 0002:00006374       ??_C@_0O@ENLNECGO@GetFloatField@ 10028374     util.obj
 0002:00006384       ??_C@_0P@MGBEMHIL@GetDoubleField@ 10028384     util.obj
 0002:00006394       ??_C@_0M@LAAAOMAB@GetIntField@ 10028394     util.obj
 0002:000063a0       ??_C@_0N@EDNEBKMF@GetLongField@ 100283a0     util.obj
 0002:000063b0       ??_C@_0O@GJMDLMFF@GetShortField@ 100283b0     util.obj
 0002:000063c0       ??_C@_0BA@BNOCBIGH@GetBooleanField@ 100283c0     util.obj
 0002:000063d0       ??_C@_0BF@IIMAGDFM@GetStaticObjectField@ 100283d0     util.obj
 0002:000063e8       ??_C@_0BD@HKPDDFOM@GetStaticByteField@ 100283e8     util.obj
 0002:000063fc       ??_C@_0BD@LIKIJFOP@GetStaticCharField@ 100283fc     util.obj
 0002:00006410       ??_C@_0BE@MDLOIBG@GetStaticFloatField@ 10028410     util.obj
 0002:00006424       ??_C@_0BF@JIILLICP@GetStaticDoubleField@ 10028424     util.obj
 0002:0000643c       ??_C@_0BC@GIOMIGFH@GetStaticIntField@ 1002843c     util.obj
 0002:00006450       ??_C@_0BD@MBAEACGO@GetStaticLongField@ 10028450     util.obj
 0002:00006464       ??_C@_0BE@CIEFBGCN@GetStaticShortField@ 10028464     util.obj
 0002:00006478       ??_C@_0BG@MMAHOAOJ@GetStaticBooleanField@ 10028478     util.obj
 0002:00006490       ??_C@_0BC@OMFJHBGB@GetFieldModifiers@ 10028490     util.obj
 0002:000064a4       ??_C@_0BD@MKDIHAMO@GetMethodModifiers@ 100284a4     util.obj
 0002:000064b8       ??_C@_0BC@IEPBNALO@GetMethodLocation@ 100284b8     util.obj
 0002:000064cc       ??_C@_0O@GILEHKFL@GetMethodName@ 100284cc     util.obj
 0002:000064dc       ??_C@_0N@NGLPCACC@GetFieldName@ 100284dc     util.obj
 0002:000064f0       ??_C@_0EH@KPFCNOHP@JDWP?5Unable?5to?5get?5JNI?51?42?5envi@ 100284f0     util.obj
 0002:00006538       ??_C@_0BI@LAHADAN@Spawning?5new?5thread?3?5?$CFs@ 10028538     util.obj
 0002:00006550       ??_C@_09FKAPGGP@NewObject@ 10028550     util.obj
 0002:0000655c       ??_C@_0P@ICNACBEG@CallVoidMethod@ 1002855c     util.obj
 0002:0000656c       ??_C@_0P@DJOFCLII@RunAgentThread@ 1002856c     util.obj
 0002:0000657c       ??_C@_0BA@OPKACKGF@GetCapabilities@ 1002857c     util.obj
 0002:0000658c       ??_C@_0CE@HHNFGJJN@on?5getting?5the?5JVMTI?5version?5nu@ 1002858c     util.obj
 0002:000065b0       ??_C@_0BI@ENBJCOLA@GetSourceDebugExtension@ 100285b0     util.obj
 0002:000065c8       ??_C@_0BN@EMLFDJOM@VM_DEAD?0?5in?5debugMonitor?$CK?$CI?$CJ?$DP@ 100285c8     util.obj
 0002:000065e8       ??_C@_0BA@LGEBNIEA@RawMonitorEnter@ 100285e8     util.obj
 0002:000065f8       ??_C@_0BF@HPIHFHIM@on?5raw?5monitor?5enter@ 100285f8     util.obj
 0002:00006610       ??_C@_0P@KLKLHGFP@RawMonitorExit@ 10028610     util.obj
 0002:00006620       ??_C@_0BE@GBAEDMCM@on?5raw?5monitor?5exit@ 10028620     util.obj
 0002:00006634       ??_C@_0P@JMJKKKKI@RawMonitorWait@ 10028634     util.obj
 0002:00006644       ??_C@_0BE@FGDFOANL@on?5raw?5monitor?5wait@ 10028644     util.obj
 0002:00006658       ??_C@_0BK@CEEJLKMK@on?5raw?5monitor?5timed?5wait@ 10028658     util.obj
 0002:00006674       ??_C@_0BB@BADFPBLM@RawMonitorNotify@ 10028674     util.obj
 0002:00006688       ??_C@_0BG@ICCOLJKI@on?5raw?5monitor?5notify@ 10028688     util.obj
 0002:000066a0       ??_C@_0BE@DMHNDKAM@RawMonitorNotifyAll@ 100286a0     util.obj
 0002:000066b4       ??_C@_0BK@IADPLGNI@on?5raw?5monitor?5notify?5all@ 100286b4     util.obj
 0002:000066d0       ??_C@_0BB@JDINKLEG@CreateRawMonitor@ 100286d0     util.obj
 0002:000066e4       ??_C@_0BN@LOANNDKM@on?5creation?5of?5a?5raw?5monitor@ 100286e4     util.obj
 0002:00006704       ??_C@_0BC@BGDFMCKH@DestroyRawMonitor@ 10028704     util.obj
 0002:00006718       ??_C@_0BO@BEIEAEKF@on?5destruction?5of?5raw?5monitor@ 10028718     util.obj
 0002:00006738       ??_C@_0BE@EADHGNCO@getting?5all?5threads@ 10028738     util.obj
 0002:0000674c       ??_C@_0BD@NCBLAKCF@GetThreadGroupInfo@ 1002874c     util.obj
 0002:00006760       ??_C@_0BN@CIHPHBI@on?5getting?5thread?5group?5info@ 10028760     util.obj
 0002:00006780       ??_C@_0BC@KKCEBIKL@GetClassSignature@ 10028780     util.obj
 0002:00006794       ??_C@_0BI@DOAGCGDM@on?5getting?5class?5status@ 10028794     util.obj
 0002:000067ac       ??_C@_0N@MDOILCOK@IsArrayClass@ 100287ac     util.obj
 0002:000067bc       ??_C@_0BP@KJLIJLJN@on?5checking?5for?5an?5array?5class@ 100287bc     util.obj
 0002:000067dc       ??_C@_0M@MIKDFOKN@IsInterface@ 100287dc     util.obj
 0002:000067e8       ??_C@_0BN@DEKKBCOO@on?5checking?5for?5an?5interface@ 100287e8     util.obj
 0002:00006808       ??_C@_0BB@GDNGBOGG@IsFieldSynthetic@ 10028808     util.obj
 0002:0000681c       ??_C@_0BC@CNKKCFND@IsMethodSynthetic@ 1002881c     util.obj
 0002:00006830       ??_C@_0P@MGFNMOMF@IsMethodNative@ 10028830     util.obj
 0002:00006840       ??_C@_0CD@EMIAHINC@on?5checking?5for?5a?5native?5interf@ 10028840     util.obj
 0002:00006864       ??_C@_0BJ@MOLBHIDD@GetImplementedInterfaces@ 10028864     util.obj
 0002:00006880       ??_C@_0BB@GNCMCKG@GetLoadedClasses@ 10028880     util.obj
 0002:00006894       ??_C@_0BG@MKDAPNKD@GetClassLoaderClasses@ 10028894     util.obj
 0002:000068ac       ??_C@_0P@KJBCCNJH@PushLocalFrame@ 100288ac     util.obj
 0002:000068bc       ??_C@_0CJ@GCEOKHEO@PushLocalFrame?3?5Unable?5to?5push?5@ 100288bc     util.obj
 0002:000068e8       ??_C@_0BC@GGHEKHNA@GetSystemProperty@ 100288e8     util.obj
 0002:000068fc       ??_C@_0CF@NNJAIEKP@JDWP?5Can?8t?5get?5property?5value?5f@ 100288fc     util.obj
 0002:00006924       ??_C@_0BB@CBHJBEJP@IsMethodObsolete@ 10028924     util.obj
 0002:00006938       ??_C@_08PEJFBAGK@Allocate@ 10028938     util.obj
 0002:00006944       ??_C@_0BM@ODCKHMNI@Can?8t?5allocate?5jvmti?5memory@ 10028944     util.obj
 0002:00006960       ??_C@_0L@KKLFJCNC@Deallocate@ 10028960     util.obj
 0002:0000696c       ??_C@_0BO@BLAPEFNH@Can?8t?5deallocate?5jvmti?5memory@ 1002896c     util.obj
 0002:0000698c       ??_C@_0P@IBCMMHME@bad?5EventIndex@ 1002898c     util.obj
 0002:0000699c       ??_C@_01OGPIMHDM@?$DP@     1002899c     util.obj
 0002:000069a0       ??_C@_0DE@JMACMIEC@?$CFs?3?5debugee?3?5thread?$DN?$CFp?$CI?$CFs?30x?$CFx?$CJ@ 100289a0     util.obj
 0002:000069d4       ??_C@_0BB@GFEELDOE@FollowReferences@ 100289d4     util.obj
 0002:000069e8       ??_C@_0BD@BPILAJHK@GetObjectsWithTags@ 100289e8     util.obj
 0002:000069fc       ??_C@_0BH@NKLJCIAP@ForceGarbageCollection@ 100289fc     util.obj
 0002:00006a14       ??_C@_0BD@FIHAEDOF@IterateThroughHeap@ 10028a14     util.obj
 0002:00006a30       __xmm@00000033000000320000004a00000049 10028a30     util.obj
 0002:00006a40       __xmm@0000003a0000003d0000003e0000003c 10028a40     util.obj
 0002:00006a50       __xmm@0000003b000000400000003f00000037 10028a50     util.obj
 0002:00006a60       __xmm@0000004c0000004b0000004200000041 10028a60     util.obj
 0002:00006a70       __xmm@00000052000000380000003500000034 10028a70     util.obj
 0002:00006a80       __pDefaultRawDllMain       10028a80     MSVCRT:dll_dllmain.obj
 0002:00006a80       __pRawDllMain              10028a80     MSVCRT:dll_dllmain.obj
 0002:00006b00       __load_config_used         10028b00     MSVCRT:loadcfg.obj
 0002:00006bb8       ___safe_se_handler_table   10028bb8     <linker-defined>
 0002:00006e40       ___rtc_iaa                 10028e40     MSVCRT:initsect.obj
 0002:00006e44       ___rtc_izz                 10028e44     MSVCRT:initsect.obj
 0002:00006e48       ___rtc_taa                 10028e48     MSVCRT:initsect.obj
 0002:00006e4c       ___rtc_tzz                 10028e4c     MSVCRT:initsect.obj
 0002:00006f7c       __IMPORT_DESCRIPTOR_KERNEL32 10028f7c     kernel32:KERNEL32.dll
 0002:00006f90       __IMPORT_DESCRIPTOR_VCRUNTIME140 10028f90     vcruntime:VCRUNTIME140.dll
 0002:00006fa4       __IMPORT_DESCRIPTOR_api-ms-win-crt-stdio-l1-1-0 10028fa4     ucrt:api-ms-win-crt-stdio-l1-1-0.dll
 0002:00006fb8       __IMPORT_DESCRIPTOR_api-ms-win-crt-string-l1-1-0 10028fb8     ucrt:api-ms-win-crt-string-l1-1-0.dll
 0002:00006fcc       __IMPORT_DESCRIPTOR_api-ms-win-crt-runtime-l1-1-0 10028fcc     ucrt:api-ms-win-crt-runtime-l1-1-0.dll
 0002:00006fe0       __IMPORT_DESCRIPTOR_api-ms-win-crt-convert-l1-1-0 10028fe0     ucrt:api-ms-win-crt-convert-l1-1-0.dll
 0002:00006ff4       __IMPORT_DESCRIPTOR_api-ms-win-crt-environment-l1-1-0 10028ff4     ucrt:api-ms-win-crt-environment-l1-1-0.dll
 0002:00007008       __IMPORT_DESCRIPTOR_api-ms-win-crt-filesystem-l1-1-0 10029008     ucrt:api-ms-win-crt-filesystem-l1-1-0.dll
 0002:0000701c       __IMPORT_DESCRIPTOR_api-ms-win-crt-time-l1-1-0 1002901c     ucrt:api-ms-win-crt-time-l1-1-0.dll
 0002:00007030       __IMPORT_DESCRIPTOR_api-ms-win-crt-heap-l1-1-0 10029030     ucrt:api-ms-win-crt-heap-l1-1-0.dll
 0002:00007044       __NULL_IMPORT_DESCRIPTOR   10029044     kernel32:KERNEL32.dll
 0003:00000000       _ArrayReference_CmdSet     1002a000     ArrayReferenceImpl.obj
 0003:0000000c       _ArrayReference_Commands   1002a00c     ArrayReferenceImpl.obj
 0003:00000024       _ArrayType_CmdSet          1002a024     ArrayTypeImpl.obj
 0003:00000030       _ArrayType_Commands        1002a030     ArrayTypeImpl.obj
 0003:00000038       _ClassLoaderReference_CmdSet 1002a038     ClassLoaderReferenceImpl.obj
 0003:00000044       _ClassLoaderReference_Commands 1002a044     ClassLoaderReferenceImpl.obj
 0003:0000004c       _ClassObjectReference_CmdSet 1002a04c     ClassObjectReferenceImpl.obj
 0003:00000058       _ClassObjectReference_Commands 1002a058     ClassObjectReferenceImpl.obj
 0003:00000060       _ClassType_CmdSet          1002a060     ClassTypeImpl.obj
 0003:0000006c       _ClassType_Commands        1002a06c     ClassTypeImpl.obj
 0003:0000008c       _EventRequest_CmdSet       1002a08c     EventRequestImpl.obj
 0003:00000098       _EventRequest_Commands     1002a098     EventRequestImpl.obj
 0003:000000b0       _Field_CmdSet              1002a0b0     FieldImpl.obj
 0003:000000bc       _InterfaceType_CmdSet      1002a0bc     InterfaceTypeImpl.obj
 0003:000000c8       _InterfaceType_Commands    1002a0c8     InterfaceTypeImpl.obj
 0003:000000d0       _Method_CmdSet             1002a0d0     MethodImpl.obj
 0003:000000dc       _Method_Commands           1002a0dc     MethodImpl.obj
 0003:00000104       _ModuleReference_CmdSet    1002a104     ModuleReferenceImpl.obj
 0003:00000110       _ModuleReference_Commands  1002a110     ModuleReferenceImpl.obj
 0003:00000120       _ObjectReference_CmdSet    1002a120     ObjectReferenceImpl.obj
 0003:00000130       _ObjectReference_Commands  1002a130     ObjectReferenceImpl.obj
 0003:00000180       _ReferenceType_CmdSet      1002a180     ReferenceTypeImpl.obj
 0003:00000190       _ReferenceType_Commands    1002a190     ReferenceTypeImpl.obj
 0003:00000228       _StackFrame_CmdSet         1002a228     StackFrameImpl.obj
 0003:00000234       _StackFrame_Commands       1002a234     StackFrameImpl.obj
 0003:00000254       _StringReference_CmdSet    1002a254     StringReferenceImpl.obj
 0003:00000260       _StringReference_Commands  1002a260     StringReferenceImpl.obj
 0003:00000268       _ThreadGroupReference_CmdSet 1002a268     ThreadGroupReferenceImpl.obj
 0003:00000274       _ThreadGroupReference_Commands 1002a274     ThreadGroupReferenceImpl.obj
 0003:00000290       _ThreadReference_CmdSet    1002a290     ThreadReferenceImpl.obj
 0003:000002a0       _ThreadReference_Commands  1002a2a0     ThreadReferenceImpl.obj
 0003:00000310       _VirtualMachine_CmdSet     1002a310     VirtualMachineImpl.obj
 0003:00000320       _VirtualMachine_Commands   1002a320     VirtualMachineImpl.obj
 0003:00000424       __fltused                  1002a424     MSVCRT:fltused.obj
 0003:00000428       ___security_cookie_complement 1002a428     MSVCRT:gs_cookie.obj
 0003:0000042c       ___security_cookie         1002a42c     MSVCRT:gs_cookie.obj
 0003:00000430       ___scrt_native_dllmain_reason 1002a430     MSVCRT:utility.obj
 0003:00000434       ___isa_enabled             1002a434     MSVCRT:cpu_disp.obj
 0003:00000440       ___scrt_ucrt_dll_is_in_use 1002a440     MSVCRT:ucrt_stubs.obj
 0003:000009b8       _gdata                     1002a9b8     util.obj
 0003:00000a24       ___scrt_current_native_startup_state 1002aa24     MSVCRT:utility.obj
 0003:00000a28       ___scrt_native_startup_lock 1002aa28     MSVCRT:utility.obj
 0003:00000d6c       ___isa_available           1002ad6c     MSVCRT:cpu_disp.obj
 0003:00000d70       ___favor                   1002ad70     MSVCRT:cpu_disp.obj
 0003:00000d74       ___scrt_debugger_hook_flag 1002ad74     MSVCRT:utility_desktop.obj
 0003:00000d78       ?__type_info_root_node@@3U__type_info_node@@A 1002ad78     MSVCRT:tncleanup.obj
 0003:00000d80       ?_OptionsStorage@?1??__local_stdio_scanf_options@@9@4_KA 1002ad80     MSVCRT:default_local_stdio_options.obj
 0003:00000d88       _deletedSignatures         1002ad88     <common>
 0003:00000d90       ?_OptionsStorage@?1??__local_stdio_printf_options@@9@9 1002ad90     <common>
 0003:00000d98       ___dyn_tls_init_callback   1002ad98     <common>

 entry point at        0001:000201aa

 Static symbols

 0000:fffd0000       .debug$S                   10000000     jdwp.exp
 0000:fffd0000       .debug$S                   10000000     vcruntime:VCRUNTIME140.dll
 0000:fffd0000       .debug$S                   10000000     vcruntime:VCRUNTIME140.dll
 0000:fffd0000       .debug$S                   10000000     vcruntime:VCRUNTIME140.dll
 0000:fffd0000       .debug$S                   10000000     vcruntime:VCRUNTIME140.dll
 0000:fffd0000       .debug$S                   10000000     vcruntime:VCRUNTIME140.dll
 0000:fffd0000       .debug$S                   10000000     vcruntime:VCRUNTIME140.dll
 0000:fffd0000       .debug$S                   10000000     vcruntime:VCRUNTIME140.dll
 0000:fffd0000       .debug$S                   10000000     vcruntime:VCRUNTIME140.dll
 0000:fffd0000       .debug$S                   10000000     vcruntime:VCRUNTIME140.dll
 0000:fffd0000       .debug$S                   10000000     vcruntime:VCRUNTIME140.dll
 0000:fffd0000       .debug$S                   10000000     ucrt:api-ms-win-crt-convert-l1-1-0.dll
 0000:fffd0000       .debug$S                   10000000     ucrt:api-ms-win-crt-convert-l1-1-0.dll
 0000:fffd0000       .debug$S                   10000000     ucrt:api-ms-win-crt-convert-l1-1-0.dll
 0000:fffd0000       .debug$S                   10000000     ucrt:api-ms-win-crt-environment-l1-1-0.dll
 0000:fffd0000       .debug$S                   10000000     ucrt:api-ms-win-crt-filesystem-l1-1-0.dll
 0000:fffd0000       .debug$S                   10000000     ucrt:api-ms-win-crt-heap-l1-1-0.dll
 0000:fffd0000       .debug$S                   10000000     ucrt:api-ms-win-crt-heap-l1-1-0.dll
 0000:fffd0000       .debug$S                   10000000     ucrt:api-ms-win-crt-runtime-l1-1-0.dll
 0000:fffd0000       .debug$S                   10000000     ucrt:api-ms-win-crt-runtime-l1-1-0.dll
 0000:fffd0000       .debug$S                   10000000     ucrt:api-ms-win-crt-runtime-l1-1-0.dll
 0000:fffd0000       .debug$S                   10000000     ucrt:api-ms-win-crt-runtime-l1-1-0.dll
 0000:fffd0000       .debug$S                   10000000     ucrt:api-ms-win-crt-runtime-l1-1-0.dll
 0000:fffd0000       .debug$S                   10000000     ucrt:api-ms-win-crt-runtime-l1-1-0.dll
 0000:fffd0000       .debug$S                   10000000     ucrt:api-ms-win-crt-runtime-l1-1-0.dll
 0000:fffd0000       .debug$S                   10000000     ucrt:api-ms-win-crt-runtime-l1-1-0.dll
 0000:fffd0000       .debug$S                   10000000     ucrt:api-ms-win-crt-runtime-l1-1-0.dll
 0000:fffd0000       .debug$S                   10000000     ucrt:api-ms-win-crt-runtime-l1-1-0.dll
 0000:fffd0000       .debug$S                   10000000     ucrt:api-ms-win-crt-runtime-l1-1-0.dll
 0000:fffd0000       .debug$S                   10000000     ucrt:api-ms-win-crt-runtime-l1-1-0.dll
 0000:fffd0000       .debug$S                   10000000     ucrt:api-ms-win-crt-runtime-l1-1-0.dll
 0000:fffd0000       .debug$S                   10000000     ucrt:api-ms-win-crt-runtime-l1-1-0.dll
 0000:fffd0000       .debug$S                   10000000     ucrt:api-ms-win-crt-runtime-l1-1-0.dll
 0000:fffd0000       .debug$S                   10000000     ucrt:api-ms-win-crt-runtime-l1-1-0.dll
 0000:fffd0000       .debug$S                   10000000     ucrt:api-ms-win-crt-runtime-l1-1-0.dll
 0000:fffd0000       .debug$S                   10000000     ucrt:api-ms-win-crt-stdio-l1-1-0.dll
 0000:fffd0000       .debug$S                   10000000     ucrt:api-ms-win-crt-stdio-l1-1-0.dll
 0000:fffd0000       .debug$S                   10000000     ucrt:api-ms-win-crt-stdio-l1-1-0.dll
 0000:fffd0000       .debug$S                   10000000     ucrt:api-ms-win-crt-stdio-l1-1-0.dll
 0000:fffd0000       .debug$S                   10000000     ucrt:api-ms-win-crt-stdio-l1-1-0.dll
 0000:fffd0000       .debug$S                   10000000     ucrt:api-ms-win-crt-stdio-l1-1-0.dll
 0000:fffd0000       .debug$S                   10000000     ucrt:api-ms-win-crt-stdio-l1-1-0.dll
 0000:fffd0000       .debug$S                   10000000     ucrt:api-ms-win-crt-string-l1-1-0.dll
 0000:fffd0000       .debug$S                   10000000     ucrt:api-ms-win-crt-string-l1-1-0.dll
 0000:fffd0000       .debug$S                   10000000     ucrt:api-ms-win-crt-string-l1-1-0.dll
 0000:fffd0000       .debug$S                   10000000     ucrt:api-ms-win-crt-string-l1-1-0.dll
 0000:fffd0000       .debug$S                   10000000     ucrt:api-ms-win-crt-string-l1-1-0.dll
 0000:fffd0000       .debug$S                   10000000     ucrt:api-ms-win-crt-string-l1-1-0.dll
 0000:fffd0000       .debug$S                   10000000     ucrt:api-ms-win-crt-string-l1-1-0.dll
 0000:fffd0000       .debug$S                   10000000     ucrt:api-ms-win-crt-string-l1-1-0.dll
 0000:fffd0000       .debug$S                   10000000     ucrt:api-ms-win-crt-time-l1-1-0.dll
 0000:fffd0000       .debug$S                   10000000     ucrt:api-ms-win-crt-time-l1-1-0.dll
 0000:fffd0000       .debug$S                   10000000     ucrt:api-ms-win-crt-time-l1-1-0.dll
 0000:fffd0000       .debug$S                   10000000     kernel32:KERNEL32.dll
 0000:fffd0000       .debug$S                   10000000     kernel32:KERNEL32.dll
 0000:fffd0000       .debug$S                   10000000     kernel32:KERNEL32.dll
 0000:fffd0000       .debug$S                   10000000     kernel32:KERNEL32.dll
 0000:fffd0000       .debug$S                   10000000     kernel32:KERNEL32.dll
 0000:fffd0000       .debug$S                   10000000     kernel32:KERNEL32.dll
 0000:fffd0000       .debug$S                   10000000     kernel32:KERNEL32.dll
 0000:fffd0000       .debug$S                   10000000     kernel32:KERNEL32.dll
 0000:fffd0000       .debug$S                   10000000     kernel32:KERNEL32.dll
 0000:fffd0000       .debug$S                   10000000     kernel32:KERNEL32.dll
 0000:fffd0000       .debug$S                   10000000     kernel32:KERNEL32.dll
 0000:fffd0000       .debug$S                   10000000     kernel32:KERNEL32.dll
 0000:fffd0000       .debug$S                   10000000     kernel32:KERNEL32.dll
 0000:fffd0000       .debug$S                   10000000     kernel32:KERNEL32.dll
 0000:fffd0000       .debug$S                   10000000     kernel32:KERNEL32.dll
 0000:fffd0000       .debug$S                   10000000     kernel32:KERNEL32.dll
 0000:fffd0000       .debug$S                   10000000     kernel32:KERNEL32.dll
 0000:fffd0000       .debug$S                   10000000     kernel32:KERNEL32.dll
 0000:fffd0000       .debug$S                   10000000     kernel32:KERNEL32.dll
 0000:fffd0000       .debug$S                   10000000     kernel32:KERNEL32.dll
 0000:fffd0000       .debug$S                   10000000     kernel32:KERNEL32.dll
 0000:fffd0000       .debug$S                   10000000     kernel32:KERNEL32.dll
 0000:fffd0000       .debug$S                   10000000     kernel32:KERNEL32.dll
 0000:fffd0000       .debug$S                   10000000     kernel32:KERNEL32.dll
 0000:fffd0000       .debug$S                   10000000     kernel32:KERNEL32.dll
 0000:fffd0000       .debug$S                   10000000     kernel32:KERNEL32.dll
 0001:00000000       _length                    10001000 f   ArrayReferenceImpl.obj
 0001:00000072       _getValues                 10001072 f   ArrayReferenceImpl.obj
 0001:00000293       _setValues                 10001293 f   ArrayReferenceImpl.obj
 0001:000004b5       _isReferenceTag            100014b5 f   ArrayReferenceImpl.obj
 0001:000004b5       _isReferenceTag            100014b5 f   ArrayTypeImpl.obj
 0001:000004b5       _isReferenceTag            100014b5 f   eventHelper.obj
 0001:000004b5       _isReferenceTag            100014b5 f   invoker.obj
 0001:000004b5       _isReferenceTag            100014b5 f   util.obj
 0001:0000051c       _jdwpTag                   1000151c f   ArrayReferenceImpl.obj
 0001:0000051c       _jdwpTag                   1000151c f   ArrayTypeImpl.obj
 0001:0000051c       _jdwpTag                   1000151c f   util.obj
 0001:00000576       _newComponents             10001576 f   ArrayReferenceImpl.obj
 0001:000005b4       _readBooleanComponents     100015b4 f   ArrayReferenceImpl.obj
 0001:00000640       _readByteComponents        10001640 f   ArrayReferenceImpl.obj
 0001:000006cc       _readCharComponents        100016cc f   ArrayReferenceImpl.obj
 0001:0000075b       _readComponents            1000175b f   ArrayReferenceImpl.obj
 0001:00000962       _readDoubleComponents      10001962 f   ArrayReferenceImpl.obj
 0001:000009f3       _readFloatComponents       100019f3 f   ArrayReferenceImpl.obj
 0001:00000a7f       _readIntComponents         10001a7f f   ArrayReferenceImpl.obj
 0001:00000b0b       _readLongComponents        10001b0b f   ArrayReferenceImpl.obj
 0001:00000ba0       _readObjectComponents      10001ba0 f   ArrayReferenceImpl.obj
 0001:00000c5d       _readShortComponents       10001c5d f   ArrayReferenceImpl.obj
 0001:00000cec       _writeBooleanComponents    10001cec f   ArrayReferenceImpl.obj
 0001:00000d75       _writeByteComponents       10001d75 f   ArrayReferenceImpl.obj
 0001:00000dfe       _writeCharComponents       10001dfe f   ArrayReferenceImpl.obj
 0001:00000e87       _writeComponents           10001e87 f   ArrayReferenceImpl.obj
 0001:00000fb4       _writeDoubleComponents     10001fb4 f   ArrayReferenceImpl.obj
 0001:00001048       _writeFloatComponents      10002048 f   ArrayReferenceImpl.obj
 0001:000010da       _writeIntComponents        100020da f   ArrayReferenceImpl.obj
 0001:00001164       _writeLongComponents       10002164 f   ArrayReferenceImpl.obj
 0001:000011f3       _writeObjectComponents     100021f3 f   ArrayReferenceImpl.obj
 0001:00001308       _writeShortComponents      10002308 f   ArrayReferenceImpl.obj
 0001:00001394       _newInstance               10002394 f   ArrayTypeImpl.obj
 0001:00001456       _getComponentClass         10002456 f   ArrayTypeImpl.obj
 0001:00001578       _writeNewObjectArray       10002578 f   ArrayTypeImpl.obj
 0001:000016da       _writeNewPrimitiveArray    100026da f   ArrayTypeImpl.obj
 0001:00001a23       _visibleClasses            10002a23 f   ClassLoaderReferenceImpl.obj
 0001:00001b16       _reflectedType             10002b16 f   ClassObjectReferenceImpl.obj
 0001:00001b65       _superclass                10002b65 f   ClassTypeImpl.obj
 0001:00001c1b       _setValues                 10002c1b f   ClassTypeImpl.obj
 0001:00001d20       _invokeStatic              10002d20 f   ClassTypeImpl.obj
 0001:00001d20       _invokeStatic              10002d20 f   InterfaceTypeImpl.obj
 0001:00001d20       _invokeInstance            10002d20 f   ObjectReferenceImpl.obj
 0001:00001d25       _readStaticFieldValue      10002d25 f   ClassTypeImpl.obj
 0001:0000217d       _setCommand                1000317d f   EventRequestImpl.obj
 0001:0000227d       _clearCommand              1000327d f   EventRequestImpl.obj
 0001:000022f7       _clearAllBreakpoints       100032f7 f   EventRequestImpl.obj
 0001:0000231c       _readAndSetFilters         1000331c f   EventRequestImpl.obj
 0001:000026dc       $LN49                      100036dc     EventRequestImpl.obj
 0001:0000275e       _lineTable                 1000375e f   MethodImpl.obj
 0001:000028d4       _variableTable             100038d4 f   MethodImpl.obj
 0001:000028e7       _variableTableWithGenerics 100038e7 f   MethodImpl.obj
 0001:000028fa       _bytecodes                 100038fa f   MethodImpl.obj
 0001:000029d8       _isObsolete                100039d8 f   MethodImpl.obj
 0001:00002a30       _doVariableTable           10003a30 f   MethodImpl.obj
 0001:00002c1f       _getName                   10003c1f f   ModuleReferenceImpl.obj
 0001:00002d53       _getClassLoader            10003d53 f   ModuleReferenceImpl.obj
 0001:00002dfa       _referenceType             10003dfa f   ObjectReferenceImpl.obj
 0001:00002ecb       _getValues                 10003ecb f   ObjectReferenceImpl.obj
 0001:00002ee0       _setValues                 10003ee0 f   ObjectReferenceImpl.obj
 0001:00003070       _monitorInfo               10004070 f   ObjectReferenceImpl.obj
 0001:000031b8       _disableCollection         100041b8 f   ObjectReferenceImpl.obj
 0001:000031ff       _enableCollection          100041ff f   ObjectReferenceImpl.obj
 0001:00003246       _isCollected               10004246 f   ObjectReferenceImpl.obj
 0001:000032ae       _referringObjects          100042ae f   ObjectReferenceImpl.obj
 0001:000033da       _readFieldValue            100043da f   ObjectReferenceImpl.obj
 0001:00003834       _signature                 10004834 f   ReferenceTypeImpl.obj
 0001:0000389f       _signatureWithGeneric      1000489f f   ReferenceTypeImpl.obj
 0001:0000392e       _getClassLoader            1000492e f   ReferenceTypeImpl.obj
 0001:0000398f       _getModule                 1000498f f   ReferenceTypeImpl.obj
 0001:00003a03       _modifiers                 10004a03 f   ReferenceTypeImpl.obj
 0001:00003a9e       _methods                   10004a9e f   ReferenceTypeImpl.obj
 0001:00003ab1       _methodsWithGeneric        10004ab1 f   ReferenceTypeImpl.obj
 0001:00003ac4       _instances                 10004ac4 f   ReferenceTypeImpl.obj
 0001:00003be4       _getClassVersion           10004be4 f   ReferenceTypeImpl.obj
 0001:00003c94       _getConstantPool           10004c94 f   ReferenceTypeImpl.obj
 0001:00003d5f       _fields                    10004d5f f   ReferenceTypeImpl.obj
 0001:00003d72       _fieldsWithGeneric         10004d72 f   ReferenceTypeImpl.obj
 0001:00003d85       _getValues                 10004d85 f   ReferenceTypeImpl.obj
 0001:00003d9a       _sourceFile                10004d9a f   ReferenceTypeImpl.obj
 0001:00003e3b       _sourceDebugExtension      10004e3b f   ReferenceTypeImpl.obj
 0001:00003e9f       _nestedTypes               10004e9f f   ReferenceTypeImpl.obj
 0001:00003f94       _getClassStatus            10004f94 f   ReferenceTypeImpl.obj
 0001:00003fd4       _interfaces                10004fd4 f   ReferenceTypeImpl.obj
 0001:000040b2       _classObject               100050b2 f   ReferenceTypeImpl.obj
 0001:000040eb       _fields1                   100050eb f   ReferenceTypeImpl.obj
 0001:000041d6       _methods1                  100051d6 f   ReferenceTypeImpl.obj
 0001:000042c1       _writeFieldInfo            100052c1 f   ReferenceTypeImpl.obj
 0001:0000439b       _writeMethodInfo           1000539b f   ReferenceTypeImpl.obj
 0001:000044db       _assureFileTableSize       100054db f   SDE.obj
 0001:0000458c       _assureLineTableSize       1000558c f   SDE.obj
 0001:0000463a       _assureStratumTableSize    1000563a f   SDE.obj
 0001:0000482f       _createJavaStratum         1000582f f   SDE.obj
 0001:00004878       _decode                    10005878 f   SDE.obj
 0001:0000496b       _defaultStratumTableIndex  1000596b f   SDE.obj
 0001:0000498c       _fileSection               1000598c f   SDE.obj
 0001:000049e5       _ignoreLine                100059e5 f   SDE.obj
 0001:00004a06       _ignoreWhite               10005a06 f   SDE.obj
 0001:00004a1c       _lineLine                  10005a1c f   SDE.obj
 0001:00004ab6       _loadDebugInfo             10005ab6 f   SDE.obj
 0001:00004bb7       _readLine                  10005bb7 f   SDE.obj
 0001:00004c11       _readNumber                10005c11 f   SDE.obj
 0001:00004c42       _sdePeek                   10005c42 f   SDE.obj
 0001:00004c59       _sdeRead                   10005c59 f   SDE.obj
 0001:00004cc2       _searchOneSourceName       10005cc2 f   SDE.obj
 0001:00004d7e       _storeFile                 10005d7e f   SDE.obj
 0001:00004db4       _storeLine                 10005db4 f   SDE.obj
 0001:00004dff       _storeStratum              10005dff f   SDE.obj
 0001:00004e6f       _stratumTableIndex         10005e6f f   SDE.obj
 0001:00004eb9       _syntax                    10005eb9 f   SDE.obj
 0001:00004f18       _getValues                 10005f18 f   StackFrameImpl.obj
 0001:0000503b       _setValues                 1000603b f   StackFrameImpl.obj
 0001:00005146       _thisObject                10006146 f   StackFrameImpl.obj
 0001:00005325       _popFrames                 10006325 f   StackFrameImpl.obj
 0001:000053c8       _readVariableValue         100063c8 f   StackFrameImpl.obj
 0001:00005763       _validateThreadFrame       10006763 f   StackFrameImpl.obj
 0001:000057a2       _writeVariableValue        100067a2 f   StackFrameImpl.obj
 0001:00005c15       _value                     10006c15 f   StringReferenceImpl.obj
 0001:00005d18       _name                      10006d18 f   ThreadGroupReferenceImpl.obj
 0001:00005dcc       _parent                    10006dcc f   ThreadGroupReferenceImpl.obj
 0001:00005e72       _children                  10006e72 f   ThreadGroupReferenceImpl.obj
 0001:00005fe5       _name                      10006fe5 f   ThreadReferenceImpl.obj
 0001:00006107       _suspend                   10007107 f   ThreadReferenceImpl.obj
 0001:0000616c       _resume                    1000716c f   ThreadReferenceImpl.obj
 0001:000061d1       _status                    100071d1 f   ThreadReferenceImpl.obj
 0001:0000625a       _threadGroup               1000725a f   ThreadReferenceImpl.obj
 0001:00006381       _frames                    10007381 f   ThreadReferenceImpl.obj
 0001:00006637       _getFrameCount             10007637 f   ThreadReferenceImpl.obj
 0001:000066f9       _ownedMonitors             100076f9 f   ThreadReferenceImpl.obj
 0001:00006866       _currentContendedMonitor   10007866 f   ThreadReferenceImpl.obj
 0001:000069a1       _stop                      100079a1 f   ThreadReferenceImpl.obj
 0001:00006a24       _interrupt                 10007a24 f   ThreadReferenceImpl.obj
 0001:00006a86       _suspendCount              10007a86 f   ThreadReferenceImpl.obj
 0001:00006afb       _ownedMonitorsWithStackDepth 10007afb f   ThreadReferenceImpl.obj
 0001:00006c8f       _forceEarlyReturn          10007c8f f   ThreadReferenceImpl.obj
 0001:000070c5       _validateSuspendedThread   100080c5 f   ThreadReferenceImpl.obj
 0001:0000710c       _version                   1000810c f   VirtualMachineImpl.obj
 0001:000071f2       _classesForSignature       100081f2 f   VirtualMachineImpl.obj
 0001:0000740f       _allModules                1000840f f   VirtualMachineImpl.obj
 0001:00007530       _allClasses                10008530 f   VirtualMachineImpl.obj
 0001:00007543       _allClassesWithGeneric     10008543 f   VirtualMachineImpl.obj
 0001:00007556       _instanceCounts            10008556 f   VirtualMachineImpl.obj
 0001:000076d4       _redefineClasses           100086d4 f   VirtualMachineImpl.obj
 0001:000078b0       _setDefaultStratum         100088b0 f   VirtualMachineImpl.obj
 0001:000078f5       _getAllThreads             100088f5 f   VirtualMachineImpl.obj
 0001:000079c5       _topLevelThreadGroups      100089c5 f   VirtualMachineImpl.obj
 0001:00007ae0       _dispose                   10008ae0 f   VirtualMachineImpl.obj
 0001:00007ae3       _idSizes                   10008ae3 f   VirtualMachineImpl.obj
 0001:00007b17       _suspend                   10008b17 f   VirtualMachineImpl.obj
 0001:00007b53       _resume                    10008b53 f   VirtualMachineImpl.obj
 0001:00007b8f       _doExit                    10008b8f f   VirtualMachineImpl.obj
 0001:00007c0a       _createString              10008c0a f   VirtualMachineImpl.obj
 0001:00007d51       _capabilities              10008d51 f   VirtualMachineImpl.obj
 0001:00007e38       _capabilitiesNew           10008e38 f   VirtualMachineImpl.obj
 0001:0000802f       _classPaths                1000902f f   VirtualMachineImpl.obj
 0001:00008079       _disposeObjects            10009079 f   VirtualMachineImpl.obj
 0001:000080fb       _holdEvents                100090fb f   VirtualMachineImpl.obj
 0001:00008103       _releaseEvents             10009103 f   VirtualMachineImpl.obj
 0001:0000810b       _allClasses1               1000910b f   VirtualMachineImpl.obj
 0001:000082e5       _writePaths                100092e5 f   VirtualMachineImpl.obj
 0001:0000852a       _cbTrackingObjectFree@12   1000952a f   classTrack.obj
 0001:00008931       _cleanDeleted              10009931 f   classTrack.obj
 0001:00008940       _setupEvents               10009940 f   classTrack.obj
 0001:000090c6       _createNode                1000a0c6 f   commonRef.obj
 0001:000092c0       _deleteNode                1000a2c0 f   commonRef.obj
 0001:000093de       _deleteNodeByID            1000a3de f   commonRef.obj
 0001:000094b4       _findNodeByID              1000a4b4 f   commonRef.obj
 0001:000094e8       _findNodeByRef             1000a4e8 f   commonRef.obj
 0001:0000954c       _hashIn                    1000a54c f   commonRef.obj
 0001:00009579       _initializeObjectsByID     1000a579 f   commonRef.obj
 0001:000095cc       _newCommonRef              1000a5cc f   commonRef.obj
 0001:0000965f       _strengthenNode            1000a65f f   commonRef.obj
 0001:0000976c       _weakenNode                1000a76c f   commonRef.obj
 0001:00009e50       _add_to_options            1000ae50 f   debugInit.obj
 0001:00009ea1       _atexit_finish_logging     1000aea1 f   debugInit.obj
 0001:00009ea6       _cbEarlyException@40       1000aea6 f   debugInit.obj
 0001:0000a1f2       _cbEarlyVMDeath@8          1000b1f2 f   debugInit.obj
 0001:0000a2c5       _cbEarlyVMInit@12          1000b2c5 f   debugInit.obj
 0001:0000a396       _checkAddress              1000b396 f   debugInit.obj
 0001:0000a3e7       _compatible_versions       1000b3e7 f   debugInit.obj
 0001:0000a6ee       _disposeEnvironment        1000b6ee f   debugInit.obj
 0001:0000a7a5       _getFirstTransport         1000b7a5 f   debugInit.obj
 0001:0000a7b2       _get_boolean               1000b7b2 f   debugInit.obj
 0001:0000a822       _get_tok                   1000b822 f   debugInit.obj
 0001:0000a870       _initialize                1000b870 f   debugInit.obj
 0001:0000ac76       _jniFatalError             1000bc76 f   debugInit.obj
 0001:0000ad6c       _parseOptions              1000bd6c f   debugInit.obj
 0001:0000b5eb       _printUsage                1000c5eb f   debugInit.obj
 0001:0000b603       _set_event_notification    1000c603 f   debugInit.obj
 0001:0000b6cf       _signalInitComplete        1000c6cf f   debugInit.obj
 0001:0000b72a       _startTransport            1000c72a f   debugInit.obj
 0001:0000ba91       _enqueue                   1000ca91 f   debugLoop.obj
 0001:0000bb3b       _lastCommand               1000cb3b f   debugLoop.obj
 0001:0000bb56       _notifyTransportError      1000cb56 f   debugLoop.obj
 0001:0000bb82       _reader@12                 1000cb82 f   debugLoop.obj
 0001:0000be3b       $LN22                      1000ce3b     error_messages.obj
 0001:0000c4f7       $LN87                      1000d4f7     error_messages.obj
 0001:0000c587       $LN86                      1000d587     error_messages.obj
 0001:0000c643       _vprint_message            1000d643 f   error_messages.obj
 0001:0000c6ec       _clearBreakpoint           1000d6ec f   eventFilter.obj
 0001:0000c7ac       _clearFilters              1000d7ac f   eventFilter.obj
 0001:0000c83c       $LN27                      1000d83c     eventFilter.obj
 0001:0000c860       _clearWatchpoint           1000d860 f   eventFilter.obj
 0001:0000c93a       _disableEvents             1000d93a f   eventFilter.obj
 0001:0000c9bc       _enableEvents              1000d9bc f   eventFilter.obj
 0001:0000ce9a       $LN79                      1000de9a     eventFilter.obj
 0001:0000d440       _eventInstance             1000e440 f   eventFilter.obj
 0001:0000d575       _findFilter                1000e575 f   eventFilter.obj
 0001:0000d5d2       _isVersionGte12x           1000e5d2 f   eventFilter.obj
 0001:0000d64a       _matchBreakpoint           1000e64a f   eventFilter.obj
 0001:0000d6b8       _matchThread               1000e6b8 f   eventFilter.obj
 0001:0000d6d3       _matchWatchpoint           1000e6d3 f   eventFilter.obj
 0001:0000d720       _patternStringMatch        1000e720 f   eventFilter.obj
 0001:0000d787       _requestThread             1000e787 f   eventFilter.obj
 0001:0000d7ab       _setBreakpoint             1000e7ab f   eventFilter.obj
 0001:0000d86b       _setWatchpoint             1000e86b f   eventFilter.obj
 0001:0000d945       _cbBreakpoint@24           1000e945 f   eventHandler.obj
 0001:0000daca       _cbClassLoad@16            1000eaca f   eventHandler.obj
 0001:0000dc37       _cbClassPrepare@16         1000ec37 f   eventHandler.obj
 0001:0000dda4       _cbException@40            1000eda4 f   eventHandler.obj
 0001:0000df4f       _cbExceptionCatch@28       1000ef4f f   eventHandler.obj
 0001:0000e0da       _cbFieldAccess@36          1000f0da f   eventHandler.obj
 0001:0000e271       _cbFieldModification@48    1000f271 f   eventHandler.obj
 0001:0000e41a       _cbFramePop@20             1000f41a f   eventHandler.obj
 0001:0000e59d       _cbGarbageCollectionFinish@4 1000f59d f   eventHandler.obj
 0001:0000e603       _cbMethodEntry@16          1000f603 f   eventHandler.obj
 0001:0000e77c       _cbMethodExit@28           1000f77c f   eventHandler.obj
 0001:0000e90b       _cbMonitorContendedEnter@16 1000f90b f   eventHandler.obj
 0001:0000eaf0       _cbMonitorContendedEntered@16 1000faf0 f   eventHandler.obj
 0001:0000ecd5       _cbMonitorWait@24          1000fcd5 f   eventHandler.obj
 0001:0000eec3       _cbMonitorWaited@20        1000fec3 f   eventHandler.obj
 0001:0000f0a9       _cbSingleStep@24           100100a9 f   eventHandler.obj
 0001:0000f22e       _cbThreadEnd@12            1001022e f   eventHandler.obj
 0001:0000f395       _cbThreadStart@12          10010395 f   eventHandler.obj
 0001:0000f4fc       _cbVMDeath@8               100104fc f   eventHandler.obj
 0001:0000f680       _cbVMInit@12               10010680 f   eventHandler.obj
 0001:0000f7e6       _createInternal            100107e6 f   eventHandler.obj
 0001:0000f874       _deferEventReport          10010874 f   eventHandler.obj
 0001:00010031       _event_callback            10011031 f   eventHandler.obj
 0001:00010371       _freeHandler               10011371 f   eventHandler.obj
 0001:000103c5       _getHandlerChain           100113c5 f   eventHandler.obj
 0001:0001049b       _getObjectClass            1001149b f   eventHandler.obj
 0001:000104e4       _installHandler            100114e4 f   eventHandler.obj
 0001:0001056d       _reportEvents              1001156d f   eventHandler.obj
 0001:0001067c       _skipEventReport           1001167c f   eventHandler.obj
 0001:00010704       _synthesizeUnloadEvent     10011704 f   eventHandler.obj
 0001:00010829       _commandLoop@12            10011829 f   eventHelper.obj
 0001:00010a60       _completeCommand           10011a60 f   eventHelper.obj
 0001:00010aae       _dequeueCommand            10011aae f   eventHelper.obj
 0001:00010b72       _enqueueCommand            10011b72 f   eventHelper.obj
 0001:00010c7e       _enumForCombinedSuspendPolicy 10011c7e f   eventHelper.obj
 0001:00010cc2       _enumForCopyingSingles     10011cc2 f   eventHelper.obj
 0001:00010ceb       _enumForVMDeath            10011ceb f   eventHelper.obj
 0001:00011311       _handleCommand             10012311 f   eventHelper.obj
 0001:000113cd       _handleEventCommandSingle  100123cd f   eventHelper.obj
 0001:00011507       _handleFrameEventCommandSingle 10012507 f   eventHelper.obj
 0001:000115b9       _handleReportEventCompositeCommand 100125b9 f   eventHelper.obj
 0001:0001170b       _handleReportVMInitCommand 1001270b f   eventHelper.obj
 0001:000117d0       _saveEventInfoRefs         100127d0 f   eventHelper.obj
 0001:0001192f       _tossEventInfoRefs         1001292f f   eventHelper.obj
 0001:000119e7       _writeClassEvent           100129e7 f   eventHelper.obj
 0001:00011aac       _writeExceptionEvent       10012aac f   eventHelper.obj
 0001:00011b06       _writeFieldAccessEvent     10012b06 f   eventHelper.obj
 0001:00011b7a       _writeFieldModificationEvent 10012b7a f   eventHelper.obj
 0001:00011bfd       _writeMonitorEvent         10012bfd f   eventHelper.obj
 0001:00011d2a       _deleteRef                 10012d2a f   inStream.obj
 0001:000122f2       _readBytes                 100132f2 f   inStream.obj
 0001:00012340       _check_methodClass         10013340 f   invoker.obj
 0001:00012438       _createGlobalRefs          10013438 f   invoker.obj
 0001:00012723       _deleteGlobalArgumentRefs  10013723 f   invoker.obj
 0001:00012820       _fillInvokeRequest         10013820 f   invoker.obj
 0001:000128f0       _invokeConstructor         100138f0 f   invoker.obj
 0001:0001297e       _invokeNonvirtual          1001397e f   invoker.obj
 0001:00012de8       _invokeStatic              10013de8 f   invoker.obj
 0001:0001320f       _invokeVirtual             1001420f f   invoker.obj
 0001:00013f17       _dll_build_name            10014f17 f   linker_md.obj
 0001:00014019       _fill_location_stamp       10015019 f   log_messages.obj
 0001:000140ab       _get_time_stamp            100150ab f   log_messages.obj
 0001:000142f9       _commonInit                100152f9 f   outStream.obj
 0001:000143ea       _outStream_send            100153ea f   outStream.obj
 0001:00014af9       _releaseID                 10015af9 f   outStream.obj
 0001:00014b13       _writeBytes                10015b13 f   outStream.obj
 0001:00014ea9       _genericHandler            10015ea9 f   standardHandlers.obj
 0001:00014ec5       _handleClassPrepare        10015ec5 f   standardHandlers.obj
 0001:00014eff       _handleFrameEvent          10015eff f   standardHandlers.obj
 0001:00014f9b       _handleGarbageCollectionFinish 10015f9b f   standardHandlers.obj
 0001:00014ff4       $LN11                      10015ff4     standardHandlers.obj
 0001:00015008       $LN10                      10016008     standardHandlers.obj
 0001:00015079       _clearStep                 10016079 f   stepControl.obj
 0001:000150ca       _completeStep              100160ca f   stepControl.obj
 0001:0001516e       _disableStepping           1001616e f   stepControl.obj
 0001:000151f4       _enableStepping            100161f4 f   stepControl.obj
 0001:0001527a       _getFrameCount             1001627a f   stepControl.obj
 0001:00015311       _getFrameLocation          10016311 f   stepControl.obj
 0001:00015389       _getLineNumberTable        10016389 f   stepControl.obj
 0001:00015405       _handleExceptionCatchEvent 10016405 f   stepControl.obj
 0001:00015506       _handleFramePopEvent       10016506 f   stepControl.obj
 0001:0001572f       _handleMethodEnterEvent    1001672f f   stepControl.obj
 0001:0001586b       _hasLineNumbers            1001686b f   stepControl.obj
 0001:0001589a       _initEvents                1001689a f   stepControl.obj
 0001:000159b2       _initState                 100169b2 f   stepControl.obj
 0001:00016528       _addDeferredEventMode      10017528 f   threadControl.obj
 0001:00016584       _addNode                   10017584 f   threadControl.obj
 0001:000165bd       _checkForPopFrameEvents    100175bd f   threadControl.obj
 0001:0001667d       $LN16                      1001767d     threadControl.obj
 0001:00016691       $LN15                      10017691     threadControl.obj
 0001:0001669f       _clearThread               1001769f f   threadControl.obj
 0001:000166fc       _commonResumeList          100176fc f   threadControl.obj
 0001:0001694a       _commonSuspend             1001794a f   threadControl.obj
 0001:000169bb       _commonSuspendByNode       100179bb f   threadControl.obj
 0001:00016a47       _commonSuspendList         10017a47 f   threadControl.obj
 0001:00016cb7       _detachHelper              10017cb7 f   threadControl.obj
 0001:00016cc8       _doPendingTasks            10017cc8 f   threadControl.obj
 0001:00016df0       _enumerateOverThreadList   10017df0 f   threadControl.obj
 0001:00016e1f       _findThread                10017e1f f   threadControl.obj
 0001:00016e8c       _getLocks                  10017e8c f   threadControl.obj
 0001:00016eb2       _getPopFrameEvent          10017eb2 f   threadControl.obj
 0001:00016f36       _getPopFrameProceed        10017f36 f   threadControl.obj
 0001:00016fba       _getResumee                10017fba f   threadControl.obj
 0001:00017018       _getStackDepth             10018018 f   threadControl.obj
 0001:000170b5       _getThreadLocalStorage     100180b5 f   threadControl.obj
 0001:0001715e       _handleAppResumeBreakpoint 1001815e f   threadControl.obj
 0001:0001719c       _handleAppResumeCompletion 1001819c f   threadControl.obj
 0001:000171f6       _insertThread              100181f6 f   threadControl.obj
 0001:00017316       _moveNode                  10018316 f   threadControl.obj
 0001:0001736c       _newArray                  1001836c f   threadControl.obj
 0001:00017395       _nonTlsSearch              10018395 f   threadControl.obj
 0001:000173c2       _notifyAppResumeComplete   100183c2 f   threadControl.obj
 0001:00017409       _pendingAppResume          10018409 f   threadControl.obj
 0001:000174a8       _popFrameCompleteEvent     100184a8 f   threadControl.obj
 0001:00017519       _popOneFrame               10018519 f   threadControl.obj
 0001:0001769c       _preSuspend                1001869c f   threadControl.obj
 0001:000176ec       _processDeferredEventModes 100186ec f   threadControl.obj
 0001:000177d1       _releaseLocks              100187d1 f   threadControl.obj
 0001:000177f6       _removeNode                100187f6 f   threadControl.obj
 0001:00017839       _removeResumed             10018839 f   threadControl.obj
 0001:00017869       _removeThread              10018869 f   threadControl.obj
 0001:00017898       _resetHelper               10018898 f   threadControl.obj
 0001:00017941       _resumeCopyHelper          10018941 f   threadControl.obj
 0001:0001799d       _resumeCountHelper         1001899d f   threadControl.obj
 0001:000179c2       _resumeHelper              100189c2 f   threadControl.obj
 0001:000179cd       _resumeThreadByNode        100189cd f   threadControl.obj
 0001:00017ab6       _setPopFrameEvent          10018ab6 f   threadControl.obj
 0001:00017b4d       _setPopFrameProceed        10018b4d f   threadControl.obj
 0001:00017bd6       _setPopFrameThread         10018bd6 f   threadControl.obj
 0001:00017c61       _setThreadLocalStorage     10018c61 f   threadControl.obj
 0001:00017d02       _suspendAllHelper          10018d02 f   threadControl.obj
 0001:00017d5f       _suspendThreadByNode       10018d5f f   threadControl.obj
 0001:00018767       _threadControl_removeDebugThread 10019767 f   threadControl.obj
 0001:00018d47       _threadSetEventNotificationMode 10019d47 f   threadControl.obj
 0001:00018db7       _threadState               10019db7 f   threadControl.obj
 0001:00018e07       _trackAppResume            10019e07 f   threadControl.obj
 0001:00018f2c       _acceptThread@12           10019f2c f   transport.obj
 0001:00019028       _attachThread@12           1001a028 f   transport.obj
 0001:0001909e       _connectionInitiated       1001a09e f   transport.obj
 0001:0001911f       _freeTransportInfo         1001a11f f   transport.obj
 0001:0001914a       _launch                    1001a14a f   transport.obj
 0001:00019215       _loadTransport             1001a215 f   transport.obj
 0001:000194f7       _loadTransportLibrary      1001a4f7 f   transport.obj
 0001:00019586       _printLastError            1001a586 f   transport.obj
 0001:00019ad0       _getCodepage               1001aad0 f   utf_util.obj
 0001:00019b2d       _getWideString             1001ab2d f   utf_util.obj
 0001:0001a23b       _utfError                  1001b23b f   utf_util.obj
 0001:0001a7ca       _cbObjectCounter@28        1001b7ca f   util.obj
 0001:0001a812       _cbObjectCounterFromRef@48 1001b812 f   util.obj
 0001:0001a8af       _cbObjectTagInstance@48    1001b8af f   util.obj
 0001:0001a8eb       _cbObjectTagReferrer@48    1001b8eb f   util.obj
 0001:0001bf73       _getPropertyUTF8           1001cf73 f   util.obj
 0001:0001c126       _getPropertyValue          1001d126 f   util.obj
 0001:0001c3c7       _getStaticMethod           1001d3c7 f   util.obj
 0001:0001c6a5       _handleInterrupt           1001d6a5 f   util.obj
 0001:0001c6c5       _ignore_vm_death           1001d6c5 f   util.obj
 0001:0001c79b       _isArrayClass              1001d79b f   util.obj
 0001:0001c943       _isInterface               1001d943 f   util.obj
 0001:0001cc8b       _is_a_nested_class         1001dc8b f   util.obj
 0001:0001cfa6       _jvmtiVersion              1001dfa6 f   util.obj
 0001:0001d497       $LN65                      1001e497     util.obj
 0001:0001d57f       $LN64                      1001e57f     util.obj
 0001:0001f29a       _writeFieldValue           1002029a f   util.obj
 0001:0001f719       _writeStaticFieldValue     10020719 f   util.obj
 0001:0001fb50       ?find_pe_section@@YAPAU_IMAGE_SECTION_HEADER@@QAEI@Z 10020b50 f   MSVCRT:utility.obj
 0001:0001fe6a       ?dllmain_crt_dispatch@@YGHQAUHINSTANCE__@@KQAX@Z 10020e6a f   MSVCRT:dll_dllmain.obj
 0001:0001febd       ?dllmain_crt_process_attach@@YAHQAUHINSTANCE__@@QAX@Z 10020ebd f   MSVCRT:dll_dllmain.obj
 0001:0001ffc4       ?dllmain_crt_process_detach@@YAH_N@Z 10020fc4 f   MSVCRT:dll_dllmain.obj
 0001:00020074       ?dllmain_dispatch@@YAHQAUHINSTANCE__@@KQAX@Z 10021074 f   MSVCRT:dll_dllmain.obj
 0001:0002017f       ?dllmain_raw@@YGHQAUHINSTANCE__@@KQAX@Z 1002117f f   MSVCRT:dll_dllmain.obj
 0001:000205f0       $$000000                   100215f0     MSVCRT:sehprolg4.obj
 0001:00020677       ___get_entropy             10021677 f   MSVCRT:gs_support.obj
 0002:00006a84       _GS_ExceptionPointers      10028a84     MSVCRT:gs_report.obj
 0002:00006e50       __sehtable$___scrt_is_nonwritable_in_current_image 10028e50     MSVCRT:utility.obj
 0002:00006e70       __sehtable$?dllmain_crt_process_attach@@YAHQAUHINSTANCE__@@QAX@Z 10028e70     MSVCRT:dll_dllmain.obj
 0002:00006e90       __sehtable$?dllmain_crt_process_detach@@YAH_N@Z 10028e90     MSVCRT:dll_dllmain.obj
 0002:00006eb8       __sehtable$?dllmain_dispatch@@YAHQAUHINSTANCE__@@KQAX@Z 10028eb8     MSVCRT:dll_dllmain.obj
 0002:00006ee0       .edata                     10028ee0     jdwp.exp
 0002:00006f08       rgpv                       10028f08     jdwp.exp
 0002:00006f14       rgszName                   10028f14     jdwp.exp
 0002:00006f20       rgwOrd                     10028f20     jdwp.exp
 0002:00006f26       szName                     10028f26     jdwp.exp
 0002:00006f2f       $N00001                    10028f2f     jdwp.exp
 0002:00006f40       $N00002                    10028f40     jdwp.exp
 0002:00006f52       $N00003                    10028f52     jdwp.exp
 0002:0000737c       .idata$6                   1002937c     kernel32:KERNEL32.dll
 0002:00007402       .idata$6                   10029402     vcruntime:VCRUNTIME140.dll
 0002:00007638       .idata$6                   10029638     ucrt:api-ms-win-crt-stdio-l1-1-0.dll
 0002:00007658       .idata$6                   10029658     ucrt:api-ms-win-crt-string-l1-1-0.dll
 0002:0000767a       .idata$6                   1002967a     ucrt:api-ms-win-crt-runtime-l1-1-0.dll
 0002:0000769c       .idata$6                   1002969c     ucrt:api-ms-win-crt-convert-l1-1-0.dll
 0002:000076be       .idata$6                   100296be     ucrt:api-ms-win-crt-environment-l1-1-0.dll
 0002:000076e4       .idata$6                   100296e4     ucrt:api-ms-win-crt-filesystem-l1-1-0.dll
 0002:0000770a       .idata$6                   1002970a     ucrt:api-ms-win-crt-time-l1-1-0.dll
 0002:0000772a       .idata$6                   1002972a     ucrt:api-ms-win-crt-heap-l1-1-0.dll
 0003:000003d0       _versionName               1002a3d0     VirtualMachineImpl.obj
 0003:000003d4       _initOnStartup             1002a3d4     debugInit.obj
 0003:000003d5       _suspendOnInit             1002a3d5     debugInit.obj
 0003:000003d8       _nof_compatible_versions   1002a3d8     debugInit.obj
 0003:000003dc       _compatible_versions_list  1002a3dc     debugInit.obj
 0003:0000040c       _p                         1002a40c     error_messages.obj
 0003:00000410       _maxQueueSize              1002a410     eventHelper.obj
 0003:00000414       _transportVersion          1002a414     transport.obj
 0003:00000418       _callback                  1002a418     transport.obj
 0003:00000420       ?intCodePage@?1??getCodepage@@9@9 1002a420     utf_util.obj
 0003:00000448       ?method@?1??getName@@9@9   1002a448     ModuleReferenceImpl.obj
 0003:0000044c       ?method@?1??getClassLoader@@9@9 1002a44c     ModuleReferenceImpl.obj
 0003:00000450       _globalDefaultStratumId    1002a450     SDE.obj
 0003:00000454       _defaultStratumId          1002a454     SDE.obj
 0003:00000458       _cachedClass               1002a458     SDE.obj
 0003:0000045c       _fileTable                 1002a45c     SDE.obj
 0003:00000460       _lineTable                 1002a460     SDE.obj
 0003:00000464       _stratumTable              1002a464     SDE.obj
 0003:00000468       _fileTableSize             1002a468     SDE.obj
 0003:0000046c       _lineTableSize             1002a46c     SDE.obj
 0003:00000470       _stratumTableSize          1002a470     SDE.obj
 0003:00000474       _fileIndex                 1002a474     SDE.obj
 0003:00000478       _lineIndex                 1002a478     SDE.obj
 0003:0000047c       _stratumIndex              1002a47c     SDE.obj
 0003:00000480       _currentFileId             1002a480     SDE.obj
 0003:00000484       _defaultStratumIndex       1002a484     SDE.obj
 0003:00000488       _baseStratumIndex          1002a488     SDE.obj
 0003:0000048c       _sdePos                    1002a48c     SDE.obj
 0003:00000490       _jplsFilename              1002a490     SDE.obj
 0003:00000494       _NullString                1002a494     SDE.obj
 0003:00000498       _sourceDebugExtension      1002a498     SDE.obj
 0003:0000049c       _sourceMapIsValid          1002a49c     SDE.obj
 0003:000004a0       _jmp_buf_env               1002a4a0     SDE.obj
 0003:000004e0       _trackingEnv               1002a4e0     classTrack.obj
 0003:000004e4       _classTrackLock            1002a4e4     classTrack.obj
 0003:000004e8       _cmdSetsArray              1002a4e8     debugDispatch.obj
 0003:000004f0       _vmInitialized             1002a4f0     debugInit.obj
 0003:000004f1       _initComplete              1002a4f1     debugInit.obj
 0003:000004f2       _currentSessionID          1002a4f2     debugInit.obj
 0003:000004f3       _isServer                  1002a4f3     debugInit.obj
 0003:000004f4       _initMonitor               1002a4f4     debugInit.obj
 0003:000004f8       _isStrict                  1002a4f8     debugInit.obj
 0003:000004f9       _useStandardAlloc          1002a4f9     debugInit.obj
 0003:000004fa       _initOnUncaught            1002a4fa     debugInit.obj
 0003:000004fb       _dopause                   1002a4fb     debugInit.obj
 0003:000004fc       _transports                1002a4fc     debugInit.obj
 0003:00000500       _initOnException           1002a500     debugInit.obj
 0003:00000504       _launchOnInit              1002a504     debugInit.obj
 0003:00000508       _docoredump                1002a508     debugInit.obj
 0003:00000509       _allowStartViaJcmd         1002a509     debugInit.obj
 0003:0000050a       _startedViaJcmd            1002a50a     debugInit.obj
 0003:0000050c       _logfile                   1002a50c     debugInit.obj
 0003:00000510       _logflags                  1002a510     debugInit.obj
 0003:00000514       _names                     1002a514     debugInit.obj
 0003:00000518       ?s@?1??get_gdata@@9@9      1002a518     debugInit.obj
 0003:00000658       _cmdQueue                  1002a658     debugLoop.obj
 0003:0000065c       _cmdQueueLock              1002a65c     debugLoop.obj
 0003:00000660       _vmDeathLock               1002a660     debugLoop.obj
 0003:00000664       _transportError            1002a664     debugLoop.obj
 0003:00000665       ?got_version@?1??eventInstance@@9@9 1002a665     eventFilter.obj
 0003:00000666       ?is_version_gte_12x@?1??eventInstance@@9@9 1002a666     eventFilter.obj
 0003:00000668       _requestIdCounter          1002a668     eventHandler.obj
 0003:0000066c       _currentSessionID          1002a66c     eventHandler.obj
 0003:0000066d       _vm_death_callback_active  1002a66d     eventHandler.obj
 0003:00000670       _active_callbacks          1002a670     eventHandler.obj
 0003:00000674       _callbackLock              1002a674     eventHandler.obj
 0003:00000678       _callbackBlock             1002a678     eventHandler.obj
 0003:0000067c       _handlerLock               1002a67c     eventHandler.obj
 0003:00000680       ___handlers                1002a680     eventHandler.obj
 0003:000006d0       _garbageCollected          1002a6d0     eventHandler.obj
 0003:000006d4       _commandQueue              1002a6d4     eventHelper.obj
 0003:000006dc       _commandQueueLock          1002a6dc     eventHelper.obj
 0003:000006e0       _commandCompleteLock       1002a6e0     eventHelper.obj
 0003:000006e4       _blockCommandLoopLock      1002a6e4     eventHelper.obj
 0003:000006e8       _vmDeathLock               1002a6e8     eventHelper.obj
 0003:000006ec       _commandLoopEnteredVmDeathLock 1002a6ec     eventHelper.obj
 0003:000006ed       _holdEvents                1002a6ed     eventHelper.obj
 0003:000006ee       ?vmDeathReported@?1??enqueueCommand@@9@9 1002a6ee     eventHelper.obj
 0003:000006ef       _blockCommandLoop          1002a6ef     eventHelper.obj
 0003:000006f0       _currentQueueSize          1002a6f0     eventHelper.obj
 0003:000006f4       _currentSessionID          1002a6f4     eventHelper.obj
 0003:000006f8       _invokerLock               1002a6f8     invoker.obj
 0003:00000700       _logging                   1002a700     log_messages.obj
 0003:00000704       _log_file                  1002a704     log_messages.obj
 0003:00000708       _logging_filename          1002a708     log_messages.obj
 0003:00000810       _location_stamp            1002a810     log_messages.obj
 0003:00000938       _processPid                1002a938     log_messages.obj
 0003:0000093c       _open_count                1002a93c     log_messages.obj
 0003:00000940       _stepLock                  1002a940     stepControl.obj
 0003:00000948       _suspendAllCount           1002a948     threadControl.obj
 0003:0000094c       _popFrameEventLock         1002a94c     threadControl.obj
 0003:00000950       _popFrameProceedLock       1002a950     threadControl.obj
 0003:00000954       _threadLock                1002a954     threadControl.obj
 0003:00000958       _resumeLocation            1002a958     threadControl.obj
 0003:00000960       _breakpointHandlerNode     1002a960     threadControl.obj
 0003:00000964       _framePopHandlerNode       1002a964     threadControl.obj
 0003:00000968       _catchHandlerNode          1002a968     threadControl.obj
 0003:0000096c       _runningThreads            1002a96c     threadControl.obj
 0003:00000970       _otherThreads              1002a970     threadControl.obj
 0003:00000974       _debugThreadCount          1002a974     threadControl.obj
 0003:00000978       _debugThreads              1002a978     threadControl.obj
 0003:000009a0       _deferredEventModes        1002a9a0     threadControl.obj
 0003:000009a8       _transport                 1002a9a8     transport.obj
 0003:000009ac       _listenerLock              1002a9ac     transport.obj
 0003:000009b0       _sendLock                  1002a9b0     transport.obj
 0003:000009bc       ?currentID@?1??uniqueID@@9@9 1002a9bc     util.obj
 0003:000009c0       _index2jvmti               1002a9c0     util.obj
 0003:00000a10       _index2jdwp                1002aa10     util.obj
 0003:00000a2c       ?is_initialized_as_dll@@3_NA 1002aa2c     MSVCRT:utility.obj
 0003:00000a2d       ?module_local_atexit_table_initialized@@3_NA 1002aa2d     MSVCRT:utility.obj
 0003:00000a30       ?module_local_atexit_table@@3U_onexit_table_t@@A 1002aa30     MSVCRT:utility.obj
 0003:00000a3c       ?module_local_at_quick_exit_table@@3U_onexit_table_t@@A 1002aa3c     MSVCRT:utility.obj
 0003:00000a48       ?__proc_attached@@3HA      1002aa48     MSVCRT:dll_dllmain.obj
 0003:00000a50       _GS_ExceptionRecord        1002aa50     MSVCRT:gs_report.obj
 0003:00000aa0       _GS_ContextRecord          1002aaa0     MSVCRT:gs_report.obj
 0004:00000060       $R000000                   1002b060     jdwp.dll.res
